:020000040000FA
:040000006FD00400B9
:101000006F00907E00000000000000009020002093
:10101000AA220020A9BDF9F56C23002000000000E1
:10102000000000006C230020902000200000000041
:101030000000000090200020000000009020002010
:101040000000000090200020902000209020002030
:101050009020002090200020582F00209424002071
:101060000000000090200020902000201E2400207E
:1010700090200020D22300209020002090200020EB
:101080009020002090200020902000209020002020
:101090009020002001A04111B7170040985F3AC688
:1010A000945F3247E39CE6FE3245410182800111A4
:1010B00013078008F337078093F787083EC20100C3
:1010C0000100B7170040930570052380B70413068D
:1010D00080FA2380C7040100010083C6B70493F699
:1010E000F60DA385D704238007049246F3A6068055
:1010F0000100010093760502D5CEF336078093F602
:10110000860836C4010001002380B7042380C70489
:1011100001000100B70614007D89558D88C70100C4
:1011200001000100010023800704A246F3A6068007
:101130000100010073370780137787083AC6010062
:1011400001002380B7042380C704010001000100CF
:1011500001003727004093061005A303D7802380A2
:101160000704B247F3A70780010001009307800836
:10117000F3B7078093F787083ECE01000100B71749
:101180000040130770052380E704130780FA2380CB
:10119000E7040100010003C7B70413670708A3852C
:1011A000E70423800704F247F3A70780010001004A
:1011B0000561828093760504BDC6F336078093F6F9
:1011C000860836C8010001002380B7042380C704C5
:1011D00001000100B7061400938606047D89558D31
:1011E00088C7010001000100010023800704C246F6
:1011F000F3A6068001000100733707801377870884
:101200003ACA010001002380B7042380C70401000B
:1012100001003727004093062005A303D7802380D1
:101220000704D24781B773370780137787083ACC12
:10123000010001002380B7042380C70401000100DE
:1012400098471367070C98C723800704E24719BF24
:101250000111814601468145114506CE97000000E7
:10126000E780605893078008F3B7078093F78708F3
:101270003EC601000100B717004013077005238028
:10128000E704130780FA2380E7040100010003C785
:101290006704136717002383E70423800704B2471A
:1012A000F3A7078001000100F2400561828041112F
:1012B000814601468145114597000000E780A05214
:1012C00013078008F337078093F787083EC40100AF
:1012D0000100B7170040130670052380C70493066A
:1012E00080FA2380D70401000100FD552396B70240
:1012F00023800704A245F3A5058001000100733790
:101300000780137787083AC6010001002380C704CD
:101310002380D7040100010003C767041367170087
:101320002383E70423800704B247F3A70780010063
:10133000010001A0BD473305F50201007D1575FDD3
:101340008280411122C426C206C6AA8401446317C2
:101350009400B24022449244410182800504130566
:10136000803E420497000000E78000FD4180C5B741
:101370009305000273A04580824573901534924016
:101380002242B2424243D2436244F2440255925551
:101390002256B2564257D2576258F25806499649D9
:1013A000264AB64A464BD64B664CF64C065D965DD1
:1013B000265EB65E465FD65F09617300203041113C
:1013C000B7170040985F3AC6945F3247E39CE6FE49
:1013D000324541018280B71700401307000323887C
:1013E000E702854717170000232EF74673002030C9
:1013F000411122C42D6426C24AC006C637190040D6
:101400001304A4AAB704002023208900977000E0E9
:10141000E780C0819C408297977000E0E780008160
:10142000E5B737370040834747009146BD8B639E41
:10143000D702B73600401306F00F973500009385AA
:10144000E51E9737000083D7672E03C7A6001377E2
:10145000F70F1DE3B7E70400BC4F09468945171590
:1014600000000345A5F7829731A099466394D70001
:10147000834757007300203003C786001377F70FA8
:10148000E365F6FC13851700AE9717380000231F9D
:10149000A8282380E70075B7B787004003C7670017
:1014A000098B6309071003C77700930600031377BE
:1014B0000703630DD70817380000034878781736FC
:1014C00000001306E6740547B30606012380E60014
:1014D00083C577001737000013078775429793F588
:1014E000F50F2300B70003C58700973500009385EB
:1014F0002573C2951375F50F2380A50003470700D8
:1015000089451377F703630CB70C63E7E50A6306B5
:10151000071A8545630CB7129737000083C75772C7
:101520003307F600034707001377F70F19CB85073A
:1015300093F7F70F3D476363F71A17370000A301CE
:10154000F770B787004009472383E700B78700405B
:1015500083C77700E207E18763DE0704973700005F
:1015600083C7176E173700001307876A3E978546B3
:101570002300D700173700001307876B3E979306A9
:1015800000032300D70017370000130767693E9751
:10159000A14685072300D70093F7F70F3D47636403
:1015A000F71417370000A30DF768B7870040094705
:1015B0002383E70073002030930610026300D70EE8
:1015C000930620026305D70693060002E316D7F4BC
:1015D00003C727021377C70F13672700D5A803C7D0
:1015E00067001377070465CB03C7A702173800000D
:1015F00013088843173500001305C53A1347070839
:101600002385E70203C7A7021377370F1367870005
:101610002385E702814713070004B305F5008C41D9
:10162000B306F80091078CC2E399E7FEF5B503C74E
:10163000A702134707042385E70203C7A70213770E
:10164000C70F136727002385E702F9B503C76700B3
:101650001377070449C303C767021738000013084C
:101660006830173500001305A527134707082383A3
:10167000E70203C767021377370F136787002383D7
:10168000E702814713070004B305F5008C41B30658
:10169000F80091078CC2E399E7FEBDBD03C767025E
:1016A000134707042383E70203C767021377C70FB3
:1016B000136727002383E70285B503C76700137705
:1016C000070411CB03C727021377370F136787006F
:1016D0002381E70291B5238006003DBD97370000C6
:1016E000A3800756B9BD97370000A38B075475BD7B
:1016F0002303048015472303E48001002302A48010
:10170000828083076480E3CE07FE23030480828007
:1017100083076480E3CE07FE03454480828083070D
:101720006480E3CE07FE2302A4808280411126C498
:101730004AC24EC006C61377F50BAD47AA892E895B
:101740009544630CF700194597000000E78080FA84
:1017500097000000E78020FB8D444E859700000035
:10176000E78040F9FD59FD1463983401B240A2446A
:101770001249824941018280135509011375F50F01
:1017800097000000E780E0F92209F1BF011126CCA3
:1017900006CEB704080097000000E780C0F61545A4
:1017A00097000000E78000F597000000E78080F6D2
:1017B00097000000E78000F62AC697000000E78047
:1017C00080F432459377150089EB13651500137586
:1017D000F50FF240E24405618280FD14E9F0014515
:1017E000CDBF397126DC4ADA4ED852D656D45AD2F9
:1017F0005ED006DE62CE66CCB7E700E07D5783AAF6
:10180000070022C603AA470023A0E71823A2E7186F
:10181000B7170040130770052380E704130780FA09
:101820002380E70483C74704930B75FFB684E20760
:1018300093FBFB0F8546AA892E8B32893724004003
:10184000E187015763FA76016308D50089461307DB
:1018500000026313D5000157D98F93F7F70FB71C18
:1018600000402382FC0411472303E4801305F00F9A
:1018700097000000E78000E8094C97000000E7802F
:1018800080E863657C15B7050700DA9537870700A0
:10189000795563FEE504B3879500636AF704370B57
:1018A0000800A94733EB65016395F90881E8814495
:1018B00097000000E78020E5268515A8DA85094510
:1018C00097000000E780C0E605090345F9FFFD1415
:1018D000050B97000000E780C0E481C49377FB0FFD
:1018E000E5F797000000E780A0EA69F17D55B7179A
:1018F0000040130770052380E704130780FA238054
:10190000E70403C74704418B2382E704F250B7E79B
:1019100000E023A0571123A24711E2543244525948
:10192000C259325AA25A125B825B724CE24C21615C
:101930008280A547639BF90685691309F00FB306FA
:101940009900B3742B01B6941349F9FFB37499004D
:10195000856B33796901416B9387F9FFB3F72701F1
:1019600099E363FC340193D94900C147E3E637FFAB
:101970003DBF0569C1697D19D9B71305800D63881D
:101980006901130500026384790113051008CA85F3
:1019900097000000E780C0D997000000E78040DF93
:1019A00031D54E99B38434416DBFDA852D4597000A
:1019B0000000E780E0D7CA94E30B99EE0509970091
:1019C0000000E78020D5A30FA9FEFDB79387F9FF9C
:1019D00093F7F70F636DFC0C83C71C0413073008E3
:1019E0006315F706370708006361EB06B3079B0032
:1019F000B706100063FBD704334BEB0089476399AC
:101A0000F9068980D549E38404EADA850945970017
:101A10000000E780E0D111090327C9FF9147232087
:101A2000E48003076480E34E07FE23033481FD173F
:101A3000EDFBFD14110B81C49377FB0FE9FF9700B9
:101A40000000E780E0D461F155B5B717004003C747
:101A50005704B70708001377070219E3B787070091
:101A60007955E376FBE833079B00E3F9E7F841B5E6
:101A70008547E380F9F0DA852D4597000000E7807F
:101A800020CB9389F4FFE38404E297000000E78011
:101A900060C893F7390091EB83260480032709007F
:101AA00093074900E396E6E03E89CE84D9BFB54767
:101AB0006399F9001305900B97000000E78080C33D
:101AC000FDB3B1471305B00AE388F9FE9947639760
:101AD000F904B7050800B365BB002D459700000069
:101AE000E78000C581448D4BA14997000000E78045
:101AF00060C263967401832704802320F900850463
:101B0000E39534FF8327048013172B0163550700E7
:101B10002312F90069BB2322F90051BB9D47639F43
:101B2000F90281451305B00497000000E78040C02A
:101B3000BD442320090023220900FD59970000001D
:101B4000E78040BD93F77400CA9703C70700FD14F0
:101B5000398D2380A700E39334FF91BBA14763979E
:101B6000F90697000000E780A0C28144630D0B00D6
:101B70008D479304C0036308FB00930400056304CE
:101B80008B01930440041375C507E30295D21945F0
:101B900097000000E78000B697000000E780A0B63D
:101BA000054597000000E780E0B426859700000017
:101BB000E78020B7094597000000E78080B69700CE
:101BC0000000E780E0BCE31405CE0DB39147639FAE
:101BD000F9001305600697000000E780A0B19700A8
:101BE0000000E78040B213059009F9B5E38109CC04
:101BF000F1547DB9BD6601471736000013068630E3
:101C0000938606A685458347060093F7F70F91C391
:101C100082800507E3F9E6FE973700002384B72E9C
:101C2000DDB77D166206618693178601E18763D46E
:101C3000070001458280931726003307F500AE9711
:101C400018439C4363E7E7007D16E37FF7FC7D556F
:101C5000828005458280FD15E205E18513978501A7
:101C6000618793F7F50F63480700FD15139725006B
:101C70002A97584365D713851700620561858280CE
:101C80003308B5021C4283A80600B335B502C297DB
:101C900033B50701AE98469585486367B5006394F0
:101CA000A50063E3070181480C43C6950CC388C2B5
:101CB0001CC2828081471397870161876343B70005
:101CC0008280139727002A97232007008507E5B70E
:101CD0008147014793968701E18663C5B6001335B6
:101CE0001700828093962700AA9694428507558F05
:101CF000D5B793D755408A07AA979C430545331516
:101D0000B5007D8D828017F3FFDFE702833D2A84D3
:101D100097000000E78060F405C5931725003E9406
:101D20000327C4FF814711EB7D1516053E9542053B
:101D3000418517F3FFDF6700033D05838507E5B79E
:101D40000145C5BF81471397870161876343C7007A
:101D5000828013972700B386E50094422A9785076F
:101D600014C3D5B77D1662066186014793178601B5
:101D7000E18763D50700133517008280931726008B
:101D8000B306F500AE9794429C437D16B58F5D8FE8
:101D9000F1BF8A05AA9501476363B500828083A6D7
:101DA000C5FFF11593D71600D98F9CC11397F60183
:101DB000E5B72A830148014701456343D700828084
:101DC000B387050183A80700B30706019C43C697A4
:101DD000AA976384F80033B517010507B308030118
:101DE000620723A0F80061871108C1BF2A83014759
:101DF0008147014563C3D70082803388E50083288B
:101E00000800330EE600032E0E003388A840330886
:101E1000C8416384080133B508018507B308E300AE
:101E2000E20723A00801E1871107E9B717F3FFDFF5
:101E3000E702232B0111B286B2842E86AA850A8579
:101E400097000000E780C0FA2A84A6850A859700DB
:101E50000000E78020E833348000060413351500C5
:101E6000018D056117F3FFDF6700E32917F3FFDF3B
:101E7000E702A3244111AA89AE8A328BB68402C23A
:101E800002C402C60144131C8401135C8C416349E3
:101E90009C02939B1400FD1B0549138CF4FFF15C1D
:101EA00033048901620461846340740792478E049D
:101EB000CE9423AEF4FE410117F3FFDF67006323E6
:101EC00013192400B30B2B01014A93172A00D6974C
:101ED00083A50B0088437800340050009700000071
:101EE000E78040DA050A93178A01E187F11BE35E78
:101EF000FCFC92474E9905042320F900A2473EC2FC
:101F0000B24702C63EC441B7131A8901135A8A4127
:101F1000131D240093178A01E18763CF970092472E
:101F20000A044E941CC0A24705091379F90F3EC25A
:101F3000B24702C63EC4ADB7B3079A0313152A00D1
:101F400056950841780034005000050AEA97DA9760
:101F50008C4397000000E780E0D26DBF197106C284
:101F600012C416C61AC81ECA22CC26CE2AD02ED219
:101F700032D436D63AD83EDA42DC46DECAC0CEC2C9
:101F8000D2C4D6C6DAC8DECAE2CCE6CEEAD0EED2F9
:101F9000F2D4F6D6FAD8FEDA971500009385058CB0
:101FA0008841E700050092402242B2424243D243B8
:101FB0006244F244025592552256B2564257D257C5
:101FC0006258F25806499649264AB64A464BD64BBD
:101FD000664CF64C065D965D265EB65E465FD65F45
:101FE0000961730020300000972100209381810156
:101FF000175100201301018117F5FFFF1305C500DC
:102000009705002093850500171600201306C6FDCE
:1020100063FAC5008322050023A055001105910530
:10202000E3EAC5FE170502001305053C97150020DD
:102030009385C5FB171600201306C66563FAC50015
:102040008322050023A0550011059105E3EAC5FE92
:1020500017150020130505649745002093858536E4
:102060006377B500232005001105E36DB5FEFD4241
:10207000739002BC8D4273904280B722000093821D
:10208000828873900230970200209382A2F793E235
:10209000320073905230975200009382E2AF7390F7
:1020A00012346FB0F47573002030397101436EC67D
:1020B00019A0397141536AC866CA62CC5ECE19A0B4
:1020C000397101535AD056D252D44ED64AD826DA54
:1020D00022DC06DE33016140828241114AC026C201
:1020E00022C406C68282B24D4101024D924C224C5E
:1020F000B24B4101024B924A224AB2494101024984
:1021000092442244B240410182803D432A87637356
:10211000C3029377F700BDEFADE5937606FF3D8AE6
:10212000BA960CC34CC30CC74CC74107E36BD7FE30
:1021300011E28280B306C3408A0697020000969699
:102140006780A6002307B700A306B7002306B700E1
:10215000A305B7002305B700A304B7002304B70005
:10216000A303B7002303B700A302B7002302B700FD
:10217000A301B7002301B700A300B7002300B700F5
:10218000828093F5F50F93968500D58D9396050182
:10219000D58D61B7939627009702000096968682A8
:1021A000E78086FA9680C1171D8F3E96E374C3F8C8
:1021B000A5B73367B500FD530D8B79E7B7877F7FF0
:1021C0009387F7F710419441B372F6003363F6003A
:1021D000BE92B3E262006397720C6318D606504158
:1021E000D441B372F6003363F600BE92B3E26200EC
:1021F0006398720A631BD60410459445B372F600C7
:102200003363F600BE92B3E262006391720A631E0A
:10221000D6025045D445B372F6003363F600BE9241
:10222000B3E26200639A72086311D60210499449BE
:10223000B372F6003363F600BE92B3E262006393BA
:1022400072085105D105E30FD6F6131706019397CF
:102250000601631CF7001357060193D706013305E7
:10226000F7409375F50F91E982804183C18333056F
:10227000F7409375F50F91E182801377F70F93F78D
:10228000F70F3305F74082800346050083C605003B
:10229000050585056313D60065FA3305D6408280AF
:1022A00011059105E312D6FE014582802105A105A5
:1022B000E31CD6FC014582803105B105E316D6FC4E
:1022C000014582804105C105E310D6FC01458280AD
:1022D000B717004003C777051377E70FA38BE70411
:1022E000130700F8A38DE7043D47238CE704130789
:1022F0005003A38CE70403C7A7051377D70F238DDB
:10230000E7048280B717004003C7E7020D89411137
:102310001377C70F498F93068008F3B6068093F6AC
:10232000860836C601000100930670052380D70495
:10233000930680FA2380D704010001002387E70277
:1023400023800704B247F3A7078001000100410181
:10235000828041112A83014E930E407E130F001993
:10236000930F400663E56E129308001913034006AD
:10237000B3781503854E0D4FA14F337365020D8958
:102380001335150063EFBE121308F6FF79467298F5
:102390004208135808013307C70213D61700BE07B7
:1023A00032976146B3F6C60213068070B386C60242
:1023B0003697A166F58F42075D8FB716004083C739
:1023C000F60293F70708A303F1000346710083C7E1
:1023D000F60293F70708E394C7FE83477100B71628
:1023E000004093F7F70F6388071293078008F3B74D
:1023F000078093F787083EC401000100B71700402B
:10240000930670052380D704930680FA2380D704AF
:102410000100010023AA070383C6170393E60608F9
:10242000A388D70223800704A247F3A707800100EF
:1024300001001166B71700407D16D45BC85F938515
:102440004703A98EF18EF5FA93068008F3B606804D
:1024500093F6860836C601000100930670052380B6
:10246000D704930680FA2380D7040100010098C1A5
:1024700003C7170313670704A388E7022380070431
:10248000B247F3A7078001000100410182807D135C
:102490003368E3039308E016630E08003368F30320
:1024A0009308D016630808009378330093B8180097
:1024B0009388D81633081E01131E0801135E0E01FF
:1024C00055B56393E5030548638608000148630337
:1024D00003002A8871087298FD15131E0801C205B1
:1024E000135E0E01C18179BD13F8150063F4BF00BE
:1024F0007908D5B713381800E5BF83C7F60293F7FC
:102500000708A303F1000346710083C7F60293F79F
:102510000708E394C7FE8347710093F7F70FF1DFD5
:10252000E9B531714AD966CB06DF22DD26DB4ED70D
:1025300052D556D35AD15ECF62CD6AC96EC7AA8C26
:1025400002D897100000E78020B12A8993078008FD
:10255000F3B7078093F787083EDA01000100B71749
:102560000040130770052380E704130780FA2380D7
:10257000E7040100010003C7F7021377770FA38771
:10258000E70203C7F70213678700A387E7022380E8
:102590000704D257F3A70780010001000545970003
:1025A0000000E78060D6130780C13347E902116A53
:1025B00093070AE893065002BD69930BA004814A71
:1025C000014B13048008930470057D1AB347F90288
:1025D0003307D7023EC0FD873ECC938709A69309F7
:1025E000803E3347F7023AC27D873AC43347390306
:1025F0008549B399990193D93940B306D702B30BF2
:102600007703B3C6F602B3CBFB0236C6FD8636C8E7
:1026100093D6FB4136CEB7460F0093860624334946
:10262000D9028566938606FAB3969601B389E902C4
:10263000130760553309D90293060010B389E902E4
:102640003349D902B3C9F9029316390036CA37198A
:102650000040FD8636D0930D090493D7F9413ED250
:10266000F336048093F6860836DC010001009307F8
:1026700070052380FD00930680FA2380DD000100B1
:1026800001008346390593F6860FA309D9048346D2
:10269000390593E61600A309D90423800D00E256FC
:1026A000F3A6068001000100130C80FA116DF336C9
:1026B000048093F6860836DE01000100930770055A
:1026C0002380FD0023808D01010001008346390530
:1026D000216693E60602A309D90483560905B3E6E9
:1026E000A6012318D90483560905D18E2318D904CD
:1026F00023800D00F256F3A60680010001008346F8
:10270000390593F606026381061A03463905218AC4
:102710006DDE081897100000E7800098733604807B
:1027200013768608B2C20100010023809D00238039
:102730008D0101000100B717004003C6370513766D
:10274000F60DA389C70403C6370513660602A389DD
:10275000C704835609052166B3E6A6012318D904E8
:1027600083560905D18E2318D90423800D0096467F
:10277000F3A60680010001008346390593F60602A0
:10278000638B061483463905A18AEDFE970000206D
:10279000E7806090AA8636D497000020E780A08F5B
:1027A000A256E30AD5FE835609054255B3E6A601B3
:1027B0002318D90497100000E780C08F834639059D
:1027C000A18AEDDE03560905834629058247337643
:1027D000CA00B306DA0293D5F641B296B388F64042
:1027E000E24733B8C6002E983308F840A247B3B684
:1027F00016013308D84063C70701631DF8009247EC
:1028000063FA1701C247634FF80E63950701B24799
:1028100063EAF80E894663E9660FF24693151800DD
:1028200013D3F8015E8613951800B365B30042D642
:1028300046D497C00100E78020213258050B137B56
:10284000FB0F63470001631A0838A25863870838F2
:1028500013081500B336A800B69513D6F5013298C3
:10286000B336C800AE9613581800FE06B3E606014C
:102870007336048013768608B2C6010001002380F7
:102880009D0023808D01010001000356C902B2960C
:10289000C206C1822316D90223800D00B646F3A6D4
:1028A00006800100010021B5F336048093F6860806
:1028B000B6C00100010023809D0023808D0101002E
:1028C00001008346390593E60602A309D904238053
:1028D0000D0086460DB5F336048093F68608B6C41F
:1028E0000100010023809D0023808D010100010073
:1028F0008346390593E60602A309D90423800D0017
:10290000A646BDB5E30B0BF0F336048093F68608BC
:10291000B6C801000100930680FA23809D00238041
:10292000DD00010001008346390593F5FC0F93F6A5
:10293000860FA309D90483463905CD8EA309D9048E
:1029400023800D00C646F3A6068001000100130592
:1029500080FA03463905930639051D8A631C9629BA
:102960007336048013768608B2CC0100010013068A
:1029700080FA23809D002380CD000100010003C662
:1029800006001376F60D2380C60003C60600136604
:1029900006022380C600835609051166D18E2318CE
:1029A000D904835609052166D18E2318D9042380C2
:1029B0000D00E646F3A6068001000100130680FA2A
:1029C0008346390593F60602638006268346390559
:1029D000130C3905A18AFDDA081897000000E7807A
:1029E000A06BF336048093F68608B6D00100010090
:1029F000930680FA23809D002380DD000100010002
:102A000083460C00116693F6F60D2300DC00834626
:102A10000C0093E606022300DC0083560905D18EE4
:102A20002318D904835609052166D18E2318D904A9
:102A300023800D008656F3A60680010001001306D0
:102A400080FA8346390593F60602638A0620834698
:102A50003905A18AEDFE97F0FF1FE780C0632A8C3D
:102A600097F0FF1FE7802063E30C85FF835609057D
:102A700011664255D18E2318D90497000000E780D3
:102A800060638346390513063905A18AFDDAF336FA
:102A9000048093F68608B6D401000100930680FAFC
:102AA00023809D002380DD00010001008346060095
:102AB00093F6F60D2300D60023800D00A656F3A64C
:102AC0000680010001008356090503462905D24707
:102AD000B376DA003306CA021305800C9355F6412B
:102AE0003696330DF6408257333CD6002E9C333653
:102AF000A601330CFC40330CCC40330885039256BE
:102B00004E86B335A5033305A503C29597C00100D2
:102B1000E78080F363468001631E0C16630C0D167C
:102B2000130615003335A6002E959356F5013696FB
:102B3000B335D600AA959396F50105828585D18E89
:102B40006346B000639D051A638B061A0356C902DB
:102B500015823305D6003336C500B2956348B00000
:102B6000639105241306F00F637DA622894663F363
:102B7000561593078008F3B7078093F78708BED6EA
:102B80000100010037170040930770052300F70488
:102B9000930780FA2300F704010001008356C7025F
:102BA00089678117D58FC207C1832316F7022300D7
:102BB0000704B657F3A7078001000100FA506A54D2
:102BC000DA544A59BA592A5A9A5A0A5BFA4B6A4C49
:102BD000DA4C4A4DBA4D296182801308F5FF33352E
:102BE000A800FD152E951356F5013298B336C8008E
:102BF000AA9695B9F336048093F68608B6CA010002
:102C0000010023809D002380AD0001000100834668
:102C10003905CD8EA309D90423800D00D646F3A62D
:102C200006800100010035B3F336048093F6860870
:102C3000B6CE0100010023809D002380CD0001005D
:102C400001008346390593E60602A309D9042380CF
:102C50000D00F646F3A606800100010095B3F33699
:102C6000048093F68608B6D20100010023809D00FF
:102C70002380CD00010001008346390593E606025A
:102C8000A309D90423800D009656F3A606800100FF
:102C9000010045BB9306F5FF33B5A600FD152E9543
:102CA0009355F501AE96B3B5B600AA951396F50106
:102CB000858269B5F336048093F68608B6D801009C
:102CC0000100930680FA23809D002380DD0001002F
:102CD00001008356C9020566011693F6F60FD18EE0
:102CE000C206C1822316D90223800D00C656F3A660
:102CF000068001000100850A93FAFA0F95B233E6C7
:102D0000B60045C20356C9023305D0403338A0008F
:102D1000B305B040B385054115826345B000D1E1EC
:102D20006371A608894663F0560593078008F3B7D8
:102D3000078093F78708BEDA01000100B71700404B
:102D4000130770052380E704130780FA2380E70444
:102D50000100010003D7C7027D8B2396E702238081
:102D60000704D65781BDF336048093F68608B6DC97
:102D700001000100930680FA23809D002380DD007E
:102D8000010001008356C9020566011693F6F60F8D
:102D9000D18EC206C1822316D90223800D00E656C9
:102DA000B9B793078008F3B7078093F78708BEDEAB
:102DB0000100010037170040930770052300F70456
:102DC000930780FA2300F704010001000356C702AD
:102DD00093975600B297C207C1832316F7022300C8
:102DE0000704F657C1BB914763EEB70217D701003E
:102DF000130787638A05BA959C41BA978287B717EC
:102E0000004003A7470B1345F5FF698F23AAE70A84
:102E100003A7070B698F23A8E70A03A7070A798D81
:102E200023A0A70A8280B717004083A6470B134749
:102E3000F5FFF98E23AAD70A83A6070B558D23A881
:102E4000A70A83A6070A758F23A0E70A8280B7170F
:102E5000004003A7470B498F23AAE70A03A7070BE4
:102E60001345F5FF45BFB717004083A6470B13472F
:102E7000F5FF758F23AAE70A03A7070A598D4DB7F7
:102E8000B717004003A7470B498FEDB7914763EE93
:102E9000B70217D701001307675A8A05BA959C41F4
:102EA000BA978287B717004003A7470D1345F5FF70
:102EB000698F23AAE70C03A7070D698F23A8E70CE6
:102EC00003A7070C798D23A0A70C8280B7170040B9
:102ED00083A6470D1347F5FFF98E23AAD70C83A6C7
:102EE000070D558D23A8A70C83A6070C758F23A06B
:102EF000E70C8280B717004003A7470D498F23AA2C
:102F0000E70C03A7070D1345F5FF45BFB7170040B2
:102F100083A6470D1347F5FF758F23AAE70C03A778
:102F2000070C598D4DB7B717004003A7470D498FC0
:102F3000EDB7797122D43714004026D24AD0035914
:102F400024028354040206D64209C2044ECE52CC57
:102F500056CA13590901C1802DE11379F9F793F489
:102F6000F49F4209C20413590901C18093078008E4
:102F7000F3B7078093F787083EC401000100930769
:102F800070052300F404930780FA2300F404010081
:102F90000100231124032310940223000404A247F8
:102FA000F3A7078001000100B25022549254025945
:102FB000F249624AD24A45618280B7F507008146EC
:102FC0003000B105194597000020E7808081A247B5
:102FD00013972701E34A07FC1369090893E40440A7
:102FE00093098008F3B7098093F787083EC0010072
:102FF0000100930A700523005405130A80FA230088
:10300000440501000100231124032310940223002E
:1030100004048247F3A7078001000100294597F0C7
:10302000FF1FE7802031F3B9098093F989084EC268
:1030300001000100230054052300440501000100A4
:103040008357040293E707202310F40223000404AB
:103050009247B9B7B7170040884742054181937737
:10306000050491EB9377F5013755E80113050580C9
:103070003345F50282809377050C130700046397AC
:10308000E7009377F50137459C1CCDB72165130503
:1030900005D0828037E700E01C435443A183E20659
:1030A000D58F1CC1FD572320F7182322F7188280E3
:1030B00013178500B7E700E023A0E710618123A282
:1030C000A7108280B7F700E08847CC47828081470D
:1030D00037370040A14663C4C7003285828003456C
:1030E000B740E38EA6FE3385F5000345050085074E
:1030F0002304A740CDB797070020938727EF9C4371
:10310000173700201307072C3E95636EE50017372D
:1031100000201307273F6368A70017070020232715
:10312000A7EC3E858280FD57EDBF8280411122C40D
:1031300006C62A8497000000E78000F22947B307FB
:10314000E502B2408D83B3D7870222449507B3D7F7
:10315000E70237370040C207C1832316F700410159
:103160008280411137150E0006C697000000E780E7
:1031700020FCB7370040130770F82381E7000D47A4
:10318000A381E70013070004A380E7000547238716
:10319000E700B24041018280373700408347270073
:1031A0001A0593F7F703C98F93F7F70F2301F70079
:1031B0008280B737004003C7170019C9D98DA38093
:1031C000B70003C70700136787002380E7008280EA
:1031D00093C5F5FFF98DA380B7008280AE872A875B
:1031E000B736004021463738004089E71703000012
:1031F0006700E3F383C8B600E30916FF05078348B9
:10320000F7FFFD17C20723041801C183F9BF41115D
:1032100022C406C62A8497000000E780E0E329471D
:10322000B307E502B2408D83B3D7870222449507E6
:10323000B3D7E70237370040C207C1832316F740F0
:1032400041018280716541111305052006C6970072
:103250000000E78000FCB7370040130770F82381B7
:10326000E7400D47A381E74013070004A380E74030
:1032700005472387E740B24041018280CC4141119C
:1032800006C6328503C6150083C5050022064D8E8D
:1032900042068D654186138875A2630C0611634B47
:1032A000C804138845A26300060D634AC8009385CD
:1032B00035A26301B6082390060029464DA0138865
:1032C00055A26305060D938565A2E316B6FE8D45EE
:1032D0001D4663E6E5081146198E63F3C7003E8676
:1032E000B7E704002390C600FC4797D501009385FB
:1032F00025179DA0138895A263030611634E060D42
:103300001388A5A263000613938505A5E315B6FAF5
:1033100099451D4663E5E504198E63F3C7003E86B3
:10332000B7E704002390C600FC479705002093856B
:1033300025D61DA09D451D4663E3E5022146198E55
:1033400063F3C7003E86B7E70400FC472390C6003E
:103350009705002093858534BA9582970146B2403F
:10336000328541018280AD451D46E3EAE5FE3146E6
:10337000198E63F3C7003E86B7E704002390C600AA
:10338000FC4797D5010093852510F9B7B1451D4637
:10339000E3E7E5FC3546198E63F3C7003E86B7E7E1
:1033A00004002390C600FC4797D501009385C50E05
:1033B00065B78D451D46E3E4E5FA1146198E63F3C2
:1033C000C7003E86B7E704002390C600FC4797D5A8
:1033D00001009385A50949B78D451D46E3E1E5F850
:1033E0001146198E63F3C7003E86B7E704002390A9
:1033F000C600FC4797D501009385C50BB1BFA54515
:103400001D46E3EEE5F42946198E63F3C7003E86B8
:10341000B7E704002390C600FC4797D501009385C9
:10342000A5051DBFB5451D46E3EBE5F23946198EEE
:1034300063F3C7003E86B7E704002390C600FC474D
:1034400097D501009385C50001BFB7E7040003A32A
:103450000713970600209386A6C24146A545170587
:1034600000201305E5B802832D455DE703C505007F
:103470000947631FE50803A84500411106C6034735
:10348000180032850346080022074168518F9308CF
:1034900028FE6307170563E9E800051863030703BF
:1034A00023900600294591A8130648FE630AC70425
:1034B0001518E31707FF15463E87637BF60015478F
:1034C00001A8130600023E876374F600130700028A
:1034D000B7E704002390E600FC471316070111A884
:1034E0003E8691C30546B7E70400FC472390C6001B
:1034F0004206CC45418282970145B240410182801B
:10350000130600083E87E375F6FC13070008C9B7E9
:103510002390060005458280828041677917630405
:10352000E504411122C406C685472A84639FF5003D
:10353000B7E7040022852244B24003A3871397050E
:1035400000209385E52F4101028389476399F500A7
:10355000B7E7040083A7070B8545829771D9B2406E
:103560002244410182808280797126D252CCAE847D
:103570002A8A97D501009385E5F517D50100130533
:10358000E5F706D63AC622D44AD0368432894ECEE2
:1035900097C00100E7808096A28517D5010013052A
:1035A000E5F697C00100E7806095294597C00100C6
:1035B000E780A09983C7840093F70702F9E383C9E2
:1035C00004008947054532476396F908D44083C70C
:1035D000160083C60600A207D58FC166138616FEA5
:1035E000638CC7028D16638FD7068D6693862690EF
:1035F00029456391D706B7E70400A286225403A3A6
:103600004714B250F2494A86A6850259925452850F
:10361000624A8547456102832D450DEF93070002FD
:10362000354563E98702B7E70400FC47C844130641
:103630000002CA8582978149970700209387072156
:103640009C43014581CB9C4391C74E852286CA8508
:1036500082970145B250225492540259F249624A6B
:10366000456182802D457DF79307700F3545E3E373
:1036700087FEB7E70400FC47C8442286CA858297C4
:1036800065BF2145C1BF411122C437E4040083272F
:10369000841326C2AA84416506C697050020938537
:1036A000251A7D1582978327C40A17050000130584
:1036B00005E78588829795C0032304132244B2400E
:1036C000924497060020938626AE4146C5451705CD
:1036D00000201305659C41010283B24022449244BC
:1036E00001454101828019C59707002023A0A71634
:1036F00001458280454582801147636AA70A97D6B3
:1037000001009386E6DB0A0536951841411106C68D
:103710003697AE87B2850287130700026145639D25
:10372000E700B7E70400FC47130600021705002076
:10373000130545F782970145B24041018280054754
:103740006145E39BE7FEB7E70400FC470546170524
:103750000020130525F7F9BF1307700F6145E39D9E
:10376000E7FCB7E70400FC471306700F17050020BD
:10377000130585F5C1B7130700086145E39EE7FA15
:10378000B7E70400FC4713060008170500201305DF
:1037900025034DB715476145E390E7FAB7E7040005
:1037A000FC471546170500201305C50961B70945F3
:1037B0008280411126C2B7E4040083A7C41322C447
:1037C0004AC006C62E8497050020938565072A897E
:1037D0008297058905C5970700209387E78B83D7D4
:1037E000A70BA28503A3440D2310F4002244B2408A
:1037F00092444A850249014641010283B240224473
:103800009244024949454101828097070020238163
:1038100007049707002023AF0702B717004003A74C
:10382000070CB706C0FFFD16758F23A0E70C03A792
:10383000070DB7064000558F23A8E70C03A7070C18
:103840003D9B23A0E70C03A7070D1367070123A8DF
:10385000E70C8280B717004003A5470C83A7470CED
:10386000598113451500C18B058999E3136525001E
:103870009707002083C7C7FD6380A7029707002032
:103880002388A7FC11C9970700209387A7FC03A3EF
:1038900007006303030002838280114517F3FFFFD3
:1038A000670063C8011122CC06CE3714004026CA37
:1038B0004AC84EC652C483447405034AB4058349BA
:1038C00084050349940597F0FFFFE780A0A0834794
:1038D000A40593F4F40F137AFA0F93E71700230D5E
:1038E000F40493F9F90F1379F90FB717004003C7E0
:1038F000A705058B6DFF03D5C705A38D4705238C51
:103900003705A38C2705A38B9704F2406244D24469
:103910004249B249224A05618280411193970501CB
:1039200022C406C626C2C1872E8463DC0700B7E422
:103930000400FC54829719C1BC5482972165218DE3
:1039400015A893F7150013C515008DE793F725000B
:103950009DC797000000E78020F0B7E70400BC4F48
:103960001306000A894517050020034525EF8297B5
:1039700013452400B240224492444101828093972F
:10398000250163D80702B7E4040083A7C41E829709
:1039900097000000E780A0F0BC4C375607001306E4
:1039A0000630896517050020034545EB82970965B8
:1039B00079B7939715010145E3DE07FA17D50100A2
:1039C0001305C5BC97B00100E780206BB7E7040082
:1039D000BC4F13060064916517050020034505E8F8
:1039E00082971165A9BF1D71A2CC37E404005C5C0D
:1039F000485886CE494697D501009385A5B482974D
:103A000011E917D50100130525B597B00100E7802E
:103A1000C06601A0B7F600E0795798CAFD57DCCA26
:103A20000567B7E700E023A0E7101306F00290C295
:103A300023A0E718010001003707002018471306EC
:103A4000000481459706002023A8E6E04157A38A99
:103A5000E7403C4408088297970700209387877CBB
:103A60003EC8856713870740938757D1231AE10023
:103A70002312F1021307B00F97F7FFFF9387C76474
:103A80002310E1023ED81547970700009387C7E14E
:103A9000B7F50700A30FE1003EDC054797070000DC
:103AA0009387E7DF81463000E10519452301E102F4
:103AB0003EDE97F0FF1FE780C0D218088147994685
:103AC00030003E960346060085070507A30BC70096
:103AD000E398D7FEC24791C70357410185676373D7
:103AE000F70001A0B7E7040083A7470A08088297F8
:103AF000AA8511C917D50100130545A797B0010084
:103B0000E780C03F01A0F6406644256182804111F4
:103B100026C2B7E4040083A7040806C622C417051A
:103B200000001305C5DF829717040020130404D397
:103B30002300A40097000000E780800297000000A7
:103B4000E780E0CC03450400224403A38405B2408F
:103B5000924413060032896541010283797106D6C9
:103B600022D413078008F337078093F787083EC2F3
:103B700001000100B7170040930570052380B704CA
:103B8000130680FA2380C7040100010083C6F702F0
:103B900093F6A60FA387D702238007049246F3A6C5
:103BA00006800100010073370780137787083AC445
:103BB000010001002380B7042380C7040100010035
:103BC00003C7F70213672700A387E70223800704D0
:103BD000A247F3A7078001000100054597E0FFFF1A
:103BE000E780807297000000E78060CB0147814644
:103BF0008147054685451305407E97E0FFFFE78036
:103C0000807537E404003C44680051468145829742
:103C1000B707C0A83EC8B787E803938707D03ECA56
:103C200097E7FF1F9387A7793EC67C586800829765
:103C3000B250225445618280411197D5010093858D
:103C400025F717D501001305658B06C697B001004F
:103C5000E780C02A17D501001305450D97B0010074
:103C6000E780C029B2402945410117B30100670030
:103C7000C32D411197D501009385C5F417D50100D7
:103C80001305C58706C697B00100E780202717D522
:103C900001001305650897B00100E7802026B240B7
:103CA0002945410117B301006700232A411122C4AD
:103CB00006C6834705002A849DC797D501009385D2
:103CC00025F617D501001305658397B00100E7803D
:103CD000E0224C4017D501001305C51A97B001002A
:103CE000E780C0213DA058410DEF97D50100938595
:103CF00025F317D501001305658097B00100E78013
:103D0000E01F17D501001305651997B00100E78082
:103D1000E01E2244B2402945410117B3010067006B
:103D2000C322A1679386D7036313D70297D50100F7
:103D3000938505EF17C501001305457C97B0010079
:103D4000E780C01B17D50100130545167DBFED07A1
:103D500097D501009385C5EC17C501001305057AB9
:103D6000631BF70097B00100E780401917D50100E9
:103D70001305051559BF97B00100E78020184C4086
:103D800017D501001305C51591BF411197D5010045
:103D9000938585E417C501001305457606C697B0DF
:103DA0000100E780A015B2402945410117B3010089
:103DB0006700A319797122D426D24AD02E842A8989
:103DC000B28481457146480006D697E0FFFFE78040
:103DD000003497F7FF1F9387275EDC4783D70700E0
:103DE000231421012313F10097500000E780202DB8
:103DF0008547A305F1009307401F2305A1003EC698
:103E00002686FD57A2854800230AF100975000003E
:103E1000E780C02DB25022549254025945618280ED
:103E20004111814617F6FF1F1306465685451705B3
:103E300000200355252406C697C00000E780C07DFA
:103E400015C997D50100938565DC17C501001305D9
:103E5000E56A97B00100E780600A17D501001305F5
:103E600065FE97B00100E7806009294597B0010021
:103E7000E780A00D97D50100938545D917C50100AE
:103E80001305C56797B00100E780400717D501000B
:103E9000130585FC97B00100E7804006294597B0DF
:103EA0000100E780800A97F7FF1F9387E750DC4700
:103EB000054797D50100938565D52390E70017C581
:103EC00001001305A56397B00100E780200317D513
:103ED00001001305A5F997B00100E7802002B24068
:103EE0002945410117B3010067002306411122C48F
:103EF00097D50100938505D42A8417C501001305C1
:103F0000E55F06C697B00100E78040FF4C4017D53B
:103F100001001305A5F097B00100E78020FE2945B8
:103F200097B00100E7806002034704009307F00F99
:103F3000631FF70297D501009385C5CF17C5010010
:103F40001305C55B97B00100E78040FB4C4017D5D7
:103F500001001305A5ED97B00100E78020FA224487
:103F6000B2402945410117B30100670003FEB2408A
:103F7000224441018280411122C426C22A84AE8497
:103F800017C501001305855797D50100938545C6D0
:103F900006C697B00100E78060F617D5010013054B
:103FA000E5F897B00100E78060F5294597B001007A
:103FB000E780A0F997D50100938585C39707002076
:103FC000239A870A17C5010013054553054497072F
:103FD0000020239F970897070020239C87089717A6
:103FE00000202394977497B00100E78020F1971583
:103FF000002083D5857317D501001305A5F397B06D
:104000000100E780A0EF294597B00100E780E0F3C9
:10401000971700202388876097F7FF1F9387C7397A
:10402000DC47170500200345E58303D70700C16778
:10403000FD17631EF700B7E7040003A38705130607
:10404000000A85452244B240924441010283B7E709
:10405000040003A387051306001493050010DDB7C1
:10406000B1C1411122C417C50100130525492E8491
:1040700097D50100938505B706C697B00100E78084
:10408000E0E7A28517D50100130585E997B0010087
:10409000E780C0E62244B2402945410117B3010040
:1040A0006700A3EA8280011122CC06CE26CA4AC844
:1040B0004EC693F715002E84B5CB97000000E7801D
:1040C00060D6930710F817070020230FF70497070F
:1040D000002083D7E7F917070020A307F7049145CD
:1040E000A183170500201305250417070020230EC0
:1040F000F70297070020A38A070297600000E78075
:1041000040BDB7E70400BC4F130600149305001030
:1041100017F5FF1F03450575829713451400F240FC
:104120006244D2444249B2490561828093F7052036
:1041300081CB97070020238B07FC13C50520C5B74B
:1041400093F70510B1C3054597600000E78060C193
:10415000171500200355655D97600000E780E08C2F
:1041600097200000E780204A9707002083C7570B5D
:1041700089E797600000E78000E397600000E78030
:1041800040E41345041061BF93F72500E9CF1707FA
:1041900000200357E7F769C7AD64B719004093845F
:1041A000A4AA23A09900970600209386A6F694421D
:1041B00097D701009387C7DA17060020034666F5F4
:1041C000814517D501001305A5DA97700000E78037
:1041D000206123A0990097F7FF1F2393A70E2A8938
:1041E00041C197D50100938525A917C50100130585
:1041F000E53097B00100E78060D0CA8517C501009F
:104200001305854797B00100E78040CF294597B057
:104210000100E78080D397070020239B07EE9307D8
:1042200010F8170700202301F7F09707002083D725
:1042300027E417070020A309F7EEA1831707002042
:104240002305F7EE91458D47170500201305C5EDB1
:1042500017070020A30BF7EC97600000E78060A72A
:10426000134524006DBD93F74500D1C397D50100D8
:10427000938585A017C501001305452897B0010057
:10428000E780C0C717C501001305C54097B00100FE
:10429000E780C0C6294597B00100E78000CB9307AF
:1042A00020F8170700202301F7E89707002083D79D
:1042B00067DE17070020A309F7E6A1831707002090
:1042C0002305F7E6854717070020A300F7E6975078
:1042D0000000E780C0F5170500201305E5E49145CF
:1042E00097600000E780E09E134544000DBD93F702
:1042F0008500A9C797D501009385059817C50100CA
:104300001305C51F97B00100E78040BF17C5010026
:104310001305853997B00100E78040BE294597B065
:104320000100E78080C297070020239307DE977083
:104330000000E780C05A13458400D5B393F7050108
:10434000D1C38545170500200355C5D497600100EA
:10435000E780C00F97D501009385059217C501002E
:104360001305C51997B00100E78040B917C50100D2
:104370001305C53497B00100E78040B8294597B0D0
:104380000100E78080BC930730F817070020230D59
:10439000F7D89707002083D7E7CF17070020A3059A
:1043A000F7D817050020130525D8A1838D451707D9
:1043B0000020230CF7D697600000E780809113451A
:1043C0000401B1BB93F70502D1C797D501009385CE
:1043D000A58A17C501001305651297B00100E78093
:1043E000E0B117C501001305A52F97B00100E780C4
:1043F000E0B0294597B00100E78020B5930740F869
:10440000170700202302F7D29707002083D7C7C6DB
:1044100017070020A30AF7D0A1831707002023065F
:10442000F7D0854717070020A301F7D09707002092
:10443000239407C497500000E78060DF1705002031
:10444000130585CE914597600000E780808813456D
:104450000402F1B193F70504FDC397D501009385DC
:10446000A58117C501001305650997B00100E78014
:10447000E0A817C501001305252897B00100E780C3
:10448000E0A7294597B00100E78020AC97070020FE
:1044900083C787C91307700A6386E7061307800A74
:1044A000638CE7081307600A6393E704930760F8D7
:1044B00017070020230AF7C69707002083D7E7C411
:1044C00017070020A302F7C6A18317070020230EB9
:1044D000F7C4854717070020A30DF7C4B14517059A
:1044E0000020130565C497500000E780807E975038
:1044F0000000E780C0D313450404970700202396EB
:1045000007C031B9930770F817070020230EF7C0D2
:104510009707002083D767BF17070020A306F7C0BF
:10452000A183170700202302F7C085471707002043
:10453000A30EF7BE994565B7930780F8F1B793F7D7
:1045400005080145E38D07BC97C501009385C57239
:1045500017C50100130585FA97B00100E780009A9E
:1045600017C501001305C51A97B00100E78000992F
:10457000294597B00100E780409D9307A0F81707F1
:1045800000202303F7BA9707002083D7E7B817075F
:104590000020A30BF7B8A183170700202307F7B863
:1045A000854717070020A302F7B897070020239537
:1045B00007B697500000E78080C717050020130555
:1045C000A5B6914597500000E780A07013450408F8
:1045D000B9B697F7FF1F83C7572917F5FF1F034584
:1045E000E5283D8D220597F7FF1F83C737283D8DAE
:1045F0004605458111C5D1476315F50055458280B3
:1046000005458280411197170020239007129717C4
:1046100000202389070006C6170700200347C7B0FC
:104620009307F00A6315F7029307F0F88945170519
:104630000020130565AF170700202307F7AE970783
:104640000020A38307AE97500000E7808068976042
:104650000000E780409597600000E78080968145E4
:10466000370504009707002023A607AA9707002014
:10467000238107AA97070020239E07A09707002001
:10468000239C079E97070020239107A897070020E7
:10469000239407A897300000E78040FA014597501F
:1046A0000000E780006C97000000E780C0F29707E9
:1046B0000020239FA7A4B7E70400BC4F13060014F3
:1046C000894517F5FF1F0345E519829797C5010036
:1046D0009385055317C50100130545E297B0010006
:1046E000E780C0819705002083D585A217D50100FA
:1046F0001305458597B00100E7804080B240294509
:10470000410117B3010067004384011122CC37E453
:1047100004005C5C06CE26CA354697C50100938529
:10472000256217D501001305E531829711E917C5F8
:104730000100130565E297B00100E780009401A035
:1047400097F7FF1F9387C7123EC4B7F50700856729
:1047500093870780814617F6FF1F1306E610E105D1
:1047600019453EC697E0FF1FE780A0077C44194625
:1047700097F5FF1F9385450F170500201305C59179
:104780008297340017F6FF1F1306060E97D5010017
:10479000938545A617D50100130545A7977000001E
:1047A000E78000D9AA8421C197C501009385C54B34
:1047B00017C50100130585D497A00100E780007498
:1047C000A68517C501001305A55897A00100E7802D
:1047D000E072294597A00100E7802077F24062440B
:1047E000D2440561828097E00000E780203E17C533
:1047F00001001305E54C97600000E78020CD97602D
:104800000100E78060F717F5FF1F130565B7976094
:104810000100E78000E017C501001305654B9760B4
:104820000100E780E0F7AA8497600000E780E033AA
:1048300097100100E78040CF97800100E780606813
:1048400097800000E780C08F97700000E780E0A9A4
:1048500097400100E780A09097C501009385C5406F
:1048600017C50100130585C999C897A00100E78005
:10487000E068A68517C501001305C54FB9B797A015
:104880000100E780A06717C501001305E55097A058
:104890000100E780A066294597A00100E780E06A53
:1048A00097300100E780806C97000100E780408B23
:1048B0006DC585453705040097300000E78000D8B6
:1048C00097C501009385453A17C50100130505C337
:1048D00097A00100E780806217C501001305454DD0
:1048E00097A00100E7808061294597A00100E7803B
:1048F000C06597F7FF1F9387A79B83D707001717FC
:1049000000202314F7E2854717170020230CF7D067
:1049100097F7FF1F938747AADC4703D70700C167B4
:10492000FD176316F70097F0FFFFE780A04F977021
:104930000000E780000B8567938707E33E9597703B
:104940000000E780C00A97200000E780C0CB171561
:104950000020035585DD97500000E780000D0545D8
:1049600097500000E780E03F97500000E7806065C7
:1049700097C501009385452F17C50100130505B89C
:1049800097A00100E780805717C501001305C547B0
:1049900097A00100E78080562DBD97000000E780BA
:1049A00080C397F7FF1F2395A77697C501009385CE
:1049B000A52B17C50100130565B497A00100E7807A
:1049C000E05317C601001306E64097F5FF1F83D595
:1049D000257417C501001305654097A00100E78005
:1049E000E051294597A00100E78020563C4C130672
:1049F000000A894517F5FF1F0345C5E68297014563
:104A000097500000E780E035A5B7411122C437E494
:104A100004008327041A06C6829797500000E78097
:104A200080048327040817F5FFFF130505688297A4
:104A300097F7FF1F2388A7E217F5FF1F1305C597F8
:104A400097500000E78060B52244B240410117034F
:104A500000006700C3CBB7E70400FC471171A2DD7B
:104A6000CAD986DFA6DBCED72E8432892E86AA85C8
:104A700017F5FF1F1305456B829717F7FF1F1307E5
:104A8000A76A83470700930680029387E70793F797
:104A9000F70FE3ECF610BA898A0717C7010013076E
:104AA00027AFBA979C43BA9782878D4797C5010075
:104AB0009385C51D17C50100130545A4630FF400B8
:104AC00097A00100E780804317C501001305C5DAF0
:104AD00097A00100E7808042BDA497A00100E78075
:104AE000E04117C501001305A5DA97A00100E78092
:104AF000E040294597A00100E7802045930720F872
:104B0000114697F5FF1F938525624A8517F7FF1F0A
:104B1000230CF76097F7FF1FA389076097F0FFFF4B
:104B2000E78080292A841DC997C501009385051651
:104B300017C501001305859C97A00100E780003C84
:104B4000A28517C50100130565D897A00100E7806D
:104B5000E03A294597A00100E780203F97C5010072
:104B60009385C51217C501001305459997A001004B
:104B7000E780C03817C50100130585D697A001004E
:104B8000E780C037294597A00100E780003C4165D8
:104B9000930730FA054697F5FF1F9385E5587D1575
:104BA00017F7FF1F2302F75897F0FFFFE780C02099
:104BB0002A841DC997C501009385450D17C50100BD
:104BC0001305C59397A00100E7804033A28517C560
:104BD00001001305A5CF97A00100E78020322945E9
:104BE00097A00100E7806036B7E70400BC4F056678
:104BF000130606C8A14517F5FF1F0345A5C68297F2
:104C0000FE506E54DE544E59BE5911618280914758
:104C10006303F40297C501009385450717C501009A
:104C20001305C58D97A00100E780402D17C5010031
:104C3000130545CE71BDB7E70400FC4F914517F54C
:104C4000FF1F034525C2829797C501009385050480
:104C500017C501001305858A97A00100E780002A87
:104C600017C501001305C5CC97A00100E7800029F6
:104C7000294597A00100E780402D97400000E7807C
:104C8000005B914535A485476303F40297C5010095
:104C90009385C5FF17C501001305458697A0010040
:104CA000E780C02517C50100130505CA15B597F79C
:104CB000FF1F2391273FB7E704000566BC4F13068B
:104CC00006C8C1450DBF8D476303F40297C50100B7
:104CD0009385C5FB17C501001305458297A0010008
:104CE000E780C02117C501001305C5C7D5B39307D9
:104CF00040F8114697F5FF1F938505434A8517F73E
:104D0000FF1F2303F74297F7FF1FA380074297F087
:104D1000FFFFE780600A2A84E30405EE97C50100DF
:104D20009385C5F617B501001305457D97A00100D1
:104D3000E780C01CA28517C50100130525B997A0FF
:104D40000100E780A01B294597A00100E780E01F34
:104D500045BD9147E31CF4F6B7E70400FC4F93050B
:104D6000000217F5FF1F0345E5AF829797C50100C5
:104D70009385C5F117B501001305457897A001008B
:104D8000E780C01717C50100130545BFF1BD89476E
:104D900063E3870297C50100938545EF17B50100CE
:104DA0001305C57597A00100E780401517C50100E0
:104DB000130505BE31BB97F4FF1F83C4043797F773
:104DC000FF1F83C7773697C50100938525ECA204A2
:104DD00017B5010013058572DD8C97A00100E780EF
:104DE000E011A28517C501001305C5BB97A00100FE
:104DF000E780C010C204294597A00100E780E014B5
:104E0000C1849305D4FF93960401C1824A8693F529
:104E1000F50F17F5FF1F1305553197300000E78098
:104E2000A085E35F90DC930750F817F7FF1F230D71
:104E3000F72E83C73900228697F5FF1F9385C52E6D
:104E400085074A8517F7FF1FA301F72E97F0FFFF8D
:104E5000E78080F62A84E30505DA97C5010093858B
:104E6000E5E217B501001305656997A00100E78029
:104E7000E008A28517C5010013058509C9B5894752
:104E800063E3870297C50100938545E017B50100EC
:104E90001305C56697A00100E780400617C501000D
:104EA000130505B235B197400000E7804038A28570
:104EB00017F5FF1F1305452797500000E78060E1B5
:104EC00081B38D476303F40297C50100938505DC28
:104ED00017B501001305856297A00100E780000265
:104EE00017C50100130585AFE5B6B7660200014698
:104EF000B7750200054597E0FF1FE780808E930796
:104F000060F817F7FF1F2301F72297F7FF1FA38E03
:104F100007209307000617F7FF1F2309F72089478B
:104F200017F7FF1FA304F72097F7FF1F2381072020
:104F300097F7FF1FA38D071EC14717F7FF1F230910
:104F4000F71E930720F917F7FF1FA303F71E31463B
:104F500097F7FF1FA38FA71C97F5FF1F9385C51C0D
:104F60004A8597F7FF1F2386071C97F0FFFFE7800E
:104F7000A0E42A84E30605C897C50100938505D1FE
:104F800017B501001305855797A00100E78000F7CA
:104F9000A28517C501001305E5A555B3B147630305
:104FA000F40297C50100938565CE17B5010013057E
:104FB000E55497A00100E78060F417C501001305D0
:104FC00025A539B6B7E70400FC4F9305000417F593
:104FD000FF1F03452589829797400000E780202521
:104FE000B145F9B5914763E3870297C50100938501
:104FF000E5C917B501001305655097A00100E780CA
:10500000E0EF17C50100130565A2D9B497F4FF1F9F
:1050100083C4C41197F7FF1F83C73711A204DD8C27
:105020008E04B77702006D14BE942286A68517C53C
:1050300001001305E5A097A00100E78020ECB7E789
:105040000400FC47228697F5FF1F9385350E280044
:10505000829793160401C1823000A685094597D036
:10506000FF1FE78000782A8409C917C501001305CE
:10507000E59E97A00100E7804000930770F819466D
:1050800097F5FF1F9385450A4A8517F7FF1F230DE4
:10509000F70897F7FF1FA38B870897F0FFFFE780BC
:1050A000A0D12A84E30E05B497C50100938505BEFF
:1050B00017B501001305854497A00100E78000E4BF
:1050C000A28517C501001305659A95B99947630B29
:1050D000F41297C50100938565BB17B50100130550
:1050E000E54197A00100E78060E117C501001305C5
:1050F0006599F9BA914763E3870297C501009385E3
:10510000E5B817B501001305653F97A00100E780DA
:10511000E0DE17C50100130565985DBA97F4FF1F1F
:1051200083C4C40097F7FF1F83C73700A204DD8C38
:105130008E04B77702006D14BE942286A68517C52B
:1051400001001305E59697A00100E78020DBB7E793
:105150000400FC47228697F5FF1F938535FD280044
:10516000829793160401C1823000A6850D4597D021
:10517000FF1FE78000672A8409C917C501001305CE
:10518000E59497A00100E78040EF930780F8194667
:1051900097F5FF1F938545F94A8517F7FF1F2305EC
:1051A000F7F897F7FF1FA38387F897F0FFFFE780D3
:1051B000A0C02A84E30605A497C50100938505AD28
:1051C00017B501001305853397A00100E78000D3D0
:1051D000A28517C501001305A59095B699476303ED
:1051E000F40297C50100938565AA17B50100130560
:1051F000E53097A00100E78060D017C501001305D6
:10520000A58FF9B0B7E70400FC4F9305000417E53C
:10521000FF1F03452565829797400000E780200126
:10522000994579B18D476303F40297C501009385D1
:10523000E5A517B501001305652C97A00100E780CF
:10524000E0CB17C501001305A58C59B017C50100A7
:105250001305058D97A00100E78020E21305C01219
:1052600097D0FF1FE780E00D014597E0FFFFE78043
:10527000A0E20D4597100000E78000B2294597D0C5
:10528000FF1FE780000C97D0FF1FE78060FC8DBAFE
:1052900099476303F40297C501009385259F17B5CD
:1052A00001001305A52597A00100E78020C517C5BB
:1052B00001001305A58729B817F7FF1F034717E754
:1052C00097F7FF1F83C787E622075D8F9166BA961F
:1052D000C2061166C1821306F6EF8D476365D602DA
:1052E00097E7FF1F9387470D9C4B17F6FF1F034659
:1052F000D6E39386C7002DC203D6070069CA890783
:10530000E39CD7FE89471307A0F8114697F5FF1FC6
:10531000938585E14A8597F6FF1F2387E6E017F717
:10532000FF1FA304F7E097F0FFFFE780E0A82A84BF
:10533000E308058C97C501009385459517B50100D5
:105340001305C51B97A00100E78040BBA28517B5D8
:1053500001001305E57EE5B203D60700630EE60AF9
:105360008907E39BF6FE8D4779BF91476304F402FA
:1053700097C501009385859117B5010013050518A0
:1053800097A00100E78080B717B501001305C57C21
:105390006FF00FF4B7E70400FC4F9305000817E522
:1053A000FF1F0345254C8297C9B897C50100938517
:1053B000E58D17B501001305651497A00100E7807E
:1053C000E0B317B501001305A57A6FF06FF02390D5
:1053D000E70017E5FF1F130525FE97300100E78062
:1053E00060DE97C501009385658A17B50100130536
:1053F000E51097A00100E78060B017B50100130524
:10540000257897A00100E78060AF294597A00100AB
:10541000E780A0B38147C5BD2390070017E5FF1FB4
:10542000130585F997300100E780C0D997C50100C1
:105430009385C58517B501001305450C97A001009C
:10544000E780C0AB17B50100130505755DBFB7E771
:105450000400FC4741112E8606C622C426C24AC05B
:105460002E842A89AA8517F5FF1F1305E5CB82979D
:1054700097C501009385458317B5010013050508FD
:1054800097A00100E78080A797F5FF1F83C5C5C9D6
:1054900017B501001305452997A00100E78000A674
:1054A000294597A00100E78040AA97F4FF1F938445
:1054B000A4C783C7040041479387070693F7F70FF4
:1054C000636FF75A17B701001307C7168A07BA9711
:1054D0009C43BA9782879D476307F40297B5010002
:1054E0009385857C17B501001305450197A0010040
:1054F000E780C0A017B501001305852397A0010020
:10550000E780C09F95A497F7FF1F83C7F7C1DDCB46
:1055100017F7FF1F034777C197F7FF1F83C7E7C040
:1055200022075D8F97F7FF1F83C747C0C2075D8FB4
:1055300097F7FF1F83C797BFE207D98F17F7FF1FA2
:10554000232AF7BC83C7640097B501009385C5750E
:1055500017B50100130585FA17F7FF1F230BF7BADC
:1055600097A00100E780809997F7FF1F938787BA7C
:105570008C4317F6FF1F0346C6B917B50100130584
:10558000E51C97A00100E7806097294597A00100DE
:10559000E780A09B97F7FF1FA38807B82244B2407B
:1055A00092440249930700F817F7FF1F230EF7B63E
:1055B0009D4517F5FF1F130525B74101174300004F
:1055C0006700237197600000E780E04097F7FF1FB6
:1055D000238DA7B49357850017F7FF1FA307F7B4D0
:1055E000935705012A8417F7FF1F2301F7B4935738
:1055F0008501014517F7FF1FA30AF7B29760000066
:10560000E780C04197F7FF1F2383A7B297B501003A
:105610009385856917B50100130545EE97A0010034
:10562000E780C08D17F6FF1F034666B0A28517B549
:10563000010013052513B1B7CD476303F40297B5F5
:1056400001009385656617B50100130525EB97A04A
:105650000100E780A08A17B501001305251279BD66
:1056600097F7FF1F83C767AD17F7FF1F0347D7AC37
:10567000A207D98FC207C18717F7FF1F231AF7A800
:10568000634AF00097F0FFFFE780E0F497F7FF1F11
:105690002390A7A8B7E7040003A387051306000A11
:1056A00089452244B2409244024917E5FF1F034551
:1056B000651B410102838D476303F40297B5010026
:1056C0009385855E17B50100130545E397A001009A
:1056D000E780C08217B501001305051A05B517F458
:1056E000FF1F034484A497F7FF1F83C7F7A397B551
:1056F00001009385655B220417B50100130505E0E1
:105700005D8C97900100E780607FA28517B501004E
:105710001305450897900100E780407E294597A032
:105720000100E78080820D4697F5FF1F9385C59F96
:10573000228597E0FFFFE7802068AA8421C197B502
:1057400001009385655617B50100130525DB979079
:105750000100E780A07AA68517B501001305C504EE
:1057600097900100E78080792244B2409244024938
:1057700029454101179301006700237D97F7FF1F1B
:10578000239A8790B7E70400116603A387051306E1
:1057900006E8914539B78D476303F40297B50100D8
:1057A0009385855017B50100130545D597900100E5
:1057B000E780C07417B501001305C51A81B317F44B
:1057C000FF1F0344849697F7FF1F83C7F79597B58C
:1057D00001009385654D220417B50100130505D21C
:1057E0005D8C97900100E7806071A28517B501007C
:1057F0001305C5FC97900100E780407029459790FC
:105800000100E78080740D4697F5FF1F9385C591D1
:10581000228597E0FFFFE780205AAA841DC197B533
:1058200001009385654817B50100130525CD9790B4
:105830000100E780A06CA68517B50100130545F9A6
:1058400005B797F7FF1F23998782B7E70400116612
:1058500003A38705130606E89305000299B5894757
:1058600063E3870297B501009385054417B50100EE
:105870001305C5C897900100E780406817B501007F
:1058800013050511A5B997F4FF1F83C4048A97F780
:10589000FF1F83C7778997B501009385E540A20470
:1058A00017B50100130585C5DD8C97900100E780D1
:1058B000E064A68517B50100130505F39790010074
:1058C000E780C063294597900100E7800068228641
:1058D00097F5FF1F93854585268597E0FFFFE780B5
:1058E000A04D2A84630E051A97B501009385C53B28
:1058F00017B50100130585C097900100E78000608F
:10590000A28517B50100130565EF99BD854763F9B9
:105910008718834519002244B24092440249B335A6
:10592000B00097E7FF1F2381B77817B50100130573
:1059300025EE4101179301006700435CA2852244D4
:10594000B24092444A8502494101170300006700B2
:10595000E34A99476303F40297B501009385C53480
:1059600017B50100130585B997900100E78000592C
:1059700017B501001305851B51B617E4FF1F03443B
:10598000C47A97E7FF1F83C7377A97B501009385DD
:10599000A531220417B50100130545B65D8C97901B
:1059A0000100E780A055A28517B501001305C5E7E2
:1059B00097900100E7808054294597900100E78087
:1059C000C058194697E5FF1F93850576228597E015
:1059D000FFFFE780603EAA841DC197B50100938553
:1059E000A52C17B50100130565B197900100E7805C
:1059F000E050A68517B50100130505E495B397E7B8
:105A0000FF1F239B8770B7E70400116603A3870578
:105A1000130606E89305000869B1854797B50100AC
:105A20009385852817B50100130545AD630BF40078
:105A300097900100E780804C17B50100130505E140
:105A400075BC97900100E780604B17B50100130506
:105A500065E197900100E780604A29459790010031
:105A6000E780A04E2244B2409244024997E7FF1FCC
:105A70002390076A410117630000670043E697B56A
:105A800001009385652217B50100130525A797909E
:105A90000100E780A04617B501001305650DB9BCEC
:105AA000B24022449244024941018280411106C61B
:105AB00022C426C239C12A8497E00000E780406AE8
:105AC000AA8411EDB7E70400BC4741468145228511
:105AD0008297B240224426859244410182804165EA
:105AE0007D1597E00000E7808068B7E7040001E9D2
:105AF000BC4741468145228582978144D9BF0347EF
:105B0000E501FC479305900819E393050003AA9566
:105B100041462285829785446DBF93170501C18751
:105B20006359F00297E7FF1F2393A75E854717E7A6
:105B3000FF1F230DF75CB7E7040003A38705056685
:105B4000130606C89305002017E5FF1F034585D1FE
:105B500002838280011122CC06CE26CA4AC883471E
:105B600005002A849DC797B501009385E50D17B5FB
:105B700001001305A59897900100E78020384C405C
:105B800017B501001305C53F97900100E780003766
:105B900005A25841B707CF009387777D6319F70CAB
:105BA0000359C500854704450356E50063F82709F6
:105BB00003C7040083C51400F17693178700CD8FC7
:105BC000C207C1879386C6556393D7029707002003
:105BD00083D7A7B56380C7126244F240CA85268581
:105BE0004249D244056117D3FFFF6700635F9547C1
:105BF00063F62705930730056312F70493075004F3
:105C0000639EF50283C62400930710046398F6028E
:105C100083C734006394E70203C744009307B004CA
:105C2000631EF70003C75400930790056318F7003D
:105C3000328597000000E78080EE79BF970700204B
:105C400083D7A7AE638AC700CA85268532C697D098
:105C5000FFFFE780E05832466244F240CA8526855D
:105C60004249D244056117F3FFFF670003DFB7071E
:105C7000CC009387777D6317F70497B50100938570
:105C8000A5FC17B501001305658797900100E78013
:105C9000E0261C448356E4008355C40003C6070075
:105CA00017B501001305452F97900100E7800025E7
:105CB0006244F240D24442492945056117930100EC
:105CC0006700A328B707CE009387777D6304F702A8
:105CD00097B50100938545F717B5010013050582B7
:105CE00097900100E78080214C4017B50100130513
:105CF000251F59BDF2406244D24442490561828069
:105D000097E7FF1F83C78740B9C397E7FF1F238F1C
:105D1000073EB7E70400FC4F411122C406C62A849F
:105D20009305002017E5FF1F0345C5B382978547FC
:105D300011C897E7FF1F9387873D83D7070023107C
:105D4000F4008547B24022443E85410182803E8571
:105D50008280411106C697E0FFFFE780E0050DC194
:105D600097E7FF1F83D76734850717E7FF1F231EB9
:105D7000F73297E7FF1F239BA732B2404101828091
:105D800097E7FF1F83D7A732850717E7FF1F231069
:105D9000F732E5B7411122C491462A8417E6FF1F66
:105DA0001306C6469D652D4506C697D0FF1FE780A2
:105DB00040A3B7F7070003C70701A5476313F70020
:105DC00001A09306001001469D65254597D0FF1F51
:105DD000E78020A197E7FF1F238A87422244B24031
:105DE000914617E6FF1F130666429D65294541014E
:105DF00017D3FF1F6700E39E1171CED7B7E90400E8
:105E000083A7C904CAD917E9FF1F1309E931A2DD25
:105E10002E8686DFA6DB2E84AA854A85829797E7A1
:105E2000FF1F83C767301307700A6385E710636D30
:105E3000F7001307600A6385E704FE506E54DE54D2
:105E40004E59BE59116182801307800A6385E71697
:105E50001307900AE393E7FE8D476306F41C97B59A
:105E600001009385E51E17A501001305256997908C
:105E70000100E780A00817B501001305A51A25A0A9
:105E80008D47630CF40297B501009385651C17A537
:105E900001001305A56697900100E780200617B55D
:105EA00001001305651197900100E7802005294541
:105EB00097900100E780600949B7854717B5010051
:105EC0001305451117E7FF1F2300F71E97900100E8
:105ED000E780A01AB7750200B766020001460545C3
:105EE00097D0FF1FE780E08F930760F817E7FF1F49
:105EF000230CF72297E7FF1FA389072293070026A9
:105F000017E7FF1F2324F722E5779387072117E779
:105F1000FF1F231FF720B14597E7FF1F238B0720A3
:105F200097E7FF1FA387A7204A8597000000E78017
:105F3000E01621B7914763E3870297B50100938587
:105F4000251117A501001305655B97900100E780F7
:105F5000E0FA17B501001305E509B1B797E4FF1F93
:105F600083C4C41C97E7FF1F83C7371CA204DD8CC2
:105F700083A7C9046D14228697E5FF1F9385151B1F
:105F8000280082978E0493160401B7750200C1821F
:105F90003000A695094597D0FF1FE78080849307BE
:105FA00070F817E7FF1F2301F718994597E7FF1FC0
:105FB000A38EA71695BF914763E3870297B50100AB
:105FC0009385050917A50100130545539790010016
:105FD000E780C0F217B5010013054503E9B597E462
:105FE000FF1F83C4A41497E7FF1F83C71714A204DD
:105FF000DD8C83A7C9046D14228697E5FF1F938566
:10600000F512280082978E0493160401B7750200DA
:10601000C1823000A6950D4597C0FF1FE780607CC8
:10602000930780F8BDBF17B501001305E5009790F1
:106030000100E7808004930790F82304F100834770
:1060400019008D452800A304F1008347290023058A
:10605000F10097000000E78060041305C01297C0AC
:10606000FF1FE780002E014597D0FFFFE780C002A9
:106070000D4597000000E78020D2294597C0FF1FFB
:10608000E780202C97C0FF1FE780801C7DB397E737
:10609000FF1F23A5A718828097E7FF1F9387071884
:1060A00003A3070063030300028317430000670094
:1060B00043C241114AC097F6FF1F83D60667328953
:1060C00017D6FF1F0356663122C426C206C62A848D
:1060D000AE8497000000E780406829C921C899472D
:1060E00063F697048347140003470400A207D98F7F
:1060F00013978700A183D98FC2073167C183130724
:10610000C7556395E70297D7FF1F83D7072DA301D4
:10611000F400A1832302F40097F7FF1F83D7E76001
:1061200091C7A302F400A1832303F40097F7FF1F94
:1061300083C7474FA1CB2686A28517D5FF1F0355DE
:10614000C52997000000E78000C1630F090297F797
:10615000FF1F83C7274D8DEB97E7FF1F83C7470CB2
:1061600085C79DC097E7FF1F83C707F491EF22857E
:106170002244B2400249A6859244410117430000DF
:10618000670023B5E31A09FCB24022449244024955
:1061900041018280834755008345450017B50100C2
:1061A0001305C5EDA207DD8D17930100670003D528
:1061B00017B50100130585EB179301006700E3EBAA
:1061C0008D4763F6B708011126CA06CE22CC0344D8
:1061D000350097E4FF1F83C4B40497B5010093858D
:1061E00025EBB337800017E7FF1FA30BF70209C4A5
:1061F00097B50100938585EA17B50100130585EA77
:1062000097900100E78080CF97E7FF1F83C7570172
:106210006386970097000000E780004397400000E6
:10622000E78020DA9967938757EE2316F10068001C
:1062300085479145A30781002307F10097000000DF
:10624000E780C0E5F2406244D244056182808280EA
:10625000894763F7B708011122CC06CE26CA8344CA
:10626000250085472A84639DF404914763F5B704AC
:10627000034545008347340022055D8D97D7FF1FF6
:10628000239DA71497000000E78000569967938725
:1062900067EE2314F1008347340023059100A30522
:1062A000F10083474400954528002306F10097003C
:1062B0000000E780A0DEF2406244D24405618280A3
:1062C000FDF89967938767EE2314F10097D7FF1FB6
:1062D00083D7A710A305F10023050100A183E1B72F
:1062E00082800111996722CCD51717F4FF1F130480
:1062F00064332314F1008347040026CA97F4FF1F78
:106300009384A4422305F10083D704002800954517
:10631000A305F100A18306CE2306F100970000003B
:10632000E780C0D703D604008345040017B50100F9
:10633000130545D897900100E78040BCF2406244C5
:10634000D244056182809D677971D9172316F100C7
:1063500097F7FF1F9387072D83C707001305F100E9
:1063600006D62307F10097F0FFFFE780607409E984
:10637000B7E70400BC47414681451305F100829709
:106380006800CD4597000000E78040D197F5FF1FDA
:1063900083C5452917B501001305C5D497900100A1
:1063A000E780C0B5B250456182806308051641118F
:1063B00026C206C622C44AC097E7FF1F83C757E616
:1063C00097F4FF1F83C4042699C393E424002A840E
:1063D00097100000E78020E319C193E4040137E936
:1063E00004008327890422851306200381458297B0
:1063F000930750FA2300F4009307A005A300F400CC
:106400008D472301F4009147A301F4009307C004D2
:10641000A302F40097F7FF1F83D727312304F4006A
:10642000A183A304F40097D7FF1F83D707FB23039F
:1064300094002305F4009304C400A1832302040004
:10644000A305F400268597F0FFFFE780606619E555
:1064500083278904414681452685829797D7FF1F68
:1064600083D747F5230EF400A183A30EF40093070E
:106470000002230FF400930710FAA30FF4009D47C6
:106480002300F402A3000402B7E70400FC4713054D
:106490002402194697D5FF1F9385053D829797E7FC
:1064A000FF1F83D7C7C02304F402A183A304F4020F
:1064B00097E7FF1F83D767BF2305F402A183A305D6
:1064C000F40297E7FF1F938767BE83970700228533
:1064D000930500032306F402C207C183A183A30628
:1064E000F40297D7FF1F9387A7DD83970700230741
:1064F000F402C207C183A183A307F402970000003E
:10650000E780A0212308A4022181A308A402B240AD
:106510002244924402494101828082805D71E17788
:1065200093C777FF1305E10086C62316F100970095
:106530000000E780C0E76800930540039700000073
:10654000E780C0B5B640616182805DC9411122C457
:1065500026C206C6930750FA2300F5009307A0054C
:10656000A300F50089472301F5009147A301F50039
:106570009307C004A302F50097F7FF1F9387870ACC
:1065800083C707009304C5002A842303F50097E717
:10659000FF1F9387F7C883C7070023020500A303E3
:1065A000F50097F7FF1F83D747182304F500A18351
:1065B000A304F50097D7FF1F83D727E22305F50033
:1065C000A183A305F500268597F0FFFFE780404EE5
:1065D00001E9B7E70400BC4741468145268582971B
:1065E0002285F14597000000E7802013230EA400C8
:1065F0002181A30EA400B240224492444101828032
:1066000082805D710A8586C6A2C497000000E7807B
:1066100000F437E404007C448A85081079468297A8
:106620003C441305E1030946814582971010930508
:106630000002014597D0FFFFE780400CB64026449A
:10664000616182800111B7C7A55A22CC9387C733F5
:1066500017E4FF1F1304D4BC3EC4834704008566BF
:1066600001469965254506CE3EC697C0FF1FE780C7
:1066700040173000A1469965294597C0FF1FE78064
:1066800040168345040017B50100130525B0979007
:106690000100E780A086F24062440561828001111A
:1066A000A146300099652D4522CC06CE97C0FF1F2C
:1066B000E7802013A24737C4A55A1304C433639557
:1066C0008702B24517B50100130505A4B335B00024
:1066D00097E7FF1FA386B7B497900100E780008279
:1066E000F2406244056182809165A1463000938545
:1066F00005F02D4597C0FF1FE780A00EA247E3825B
:1067000087FC97E7FF1FA38D07B0814517B50100F0
:106710001305C5A1D1B7C16769768146FD17050686
:106720001397060141836364B7003E858280330777
:10673000D50003470700B98F214713F81700858359
:1067400063050800B18FC207C1837D171377F70F68
:106750006DF78506F1B741C5A547054763F2B70850
:1067600083471500034705003168A207D98F1397A7
:106770008700A183D98FC207C1831308C855054775
:1067800063900707411106C622C426C203442500B0
:10679000914763F087049307540063ECF502A3016B
:1067A000C50021822302C5009304340091C6A302D0
:1067B000D500A1822303D5002A84A6859700000076
:1067C000E780A0F526942300A4002181A300A40063
:1067D0000147B240224492443A85410182800547F4
:1067E0003A8582800111B7C7A55A22CC9387E73436
:1067F0002A842AC6856601469565254506CE3EC48F
:1068000097C0FF1FE780E0FD3000A1469565294550
:1068100097C0FF1FE780E0FCA28517B501001305B4
:10682000E59897800100E780606D97000000E780A1
:1068300080DDF2406244056182800111A146300092
:1068400095652D4522CC06CE97C0FF1FE78060F9E5
:10685000A24737C4A55A1304E43463958702B245AE
:1068600017B501001305858E97D7FF1F2397B7B67D
:10687000C205C18197800100E7804068F240624410
:10688000056182809165A1463000938505EE2D4516
:1068900097C0FF1FE780E0F4A247E38287FCD1475F
:1068A00017D7FF1F231BF7B2D14517B501001305FA
:1068B000E58BC9B7011122CC2A841305E10026CA51
:1068C00006CEAE8497F0FFFFE780C04309C90355A9
:1068D000E1002686A28597F0FFFFE780C047A685E6
:1068E000228597100000E780A09297E7FF1F83C7DB
:1068F000279399C7A685228597300000E780603DE1
:10690000F2406244D2440561828001114EC606CE37
:1069100022CC26CA4AC893F71500AE899DCBAD6735
:10692000371700409387A7AA1CC3B7E70400BC4FE2
:1069300013060019854517D5FF1F0345E5A9829762
:1069400013C51900F2406244D2444249B24905617C
:10695000828093F725000145F5D717F7FF1F0357EE
:10696000A7DC954763FAE70C014417F6FF1F1306EF
:10697000A6CB9306300513055004130810049308A2
:10698000B00413039005930764006374F7043A841A
:106990007D5997F4FF1F83C424C997F7FF1F83C74E
:1069A000B7C8A204DD8CAD679387B755638CF41428
:1069B00063E4970AA9679387A755638FF414A285A8
:1069C00017F5FF1F130545C697000000E780C0EECE
:1069D000F1A0B307860083C50700639BD50483C578
:1069E00017006397A50483C527006393050583C536
:1069F0003700639FD50283C54700639B150383C798
:106A0000570063976702228915E897F5FF1F83D522
:106A1000A5D1B3852541C205C181F1CD17F5FF1F71
:106A2000130585C04A9597000000E780E0E8E1A0E3
:106A300005044204418081BF3A847D598547E3EAD9
:106A400087F45DC4854517F5FF1F1305E5BD970065
:106A50000000E78060E669A8B1679387C75563893E
:106A6000F404B5679387D755E39BF4F4A28517F533
:106A7000FF1F130565BB97300000E780802589471D
:106A8000630EF4009305E4FFC205C18117F5FF1FF3
:106A90001305A5B997000000E7808077A68517A5A4
:106AA00001001305657297800100E780204589A0E9
:106AB00097200000E780401797000000E780A0744F
:106AC00011C9A28517F5FF1F130505B69700000031
:106AD000E78000740546A28517F5FF1F1305C5B4AE
:106AE00097F0FFFFE780205D97200000E780C0134C
:106AF000FD57E31CF9F097F7FF1F239707C213C553
:106B0000290089B5A28517F5FF1F1305E5B197F098
:106B1000FFFFE780606859B7A28517F5FF1F1305CF
:106B2000A5B097F0FFFFE780E0688DBF411122C458
:106B300037E404005C5C06C6354697A501009385E2
:106B4000252017B501001305E5EF829711E917A578
:106B500001001305A56897800100E780005201A09D
:106B60008327041C82972A84054597C00000E7808C
:106B7000400597700100E780608A97600100E78018
:106B8000605F97B00000E780C0162285B2402244C3
:106B9000410182804111054506C622C426C297C024
:106BA000FFFFE78040391305A00497B0FF1FE7807F
:106BB0000050757585457D1597C0FFFFE780E02281
:106BC0007D7585451305F53697C0FFFFE780402C9E
:106BD000371400408327840A8D451305002093E76E
:106BE00007202324F40A97C0FFFFE7800020B7E4C2
:106BF000040097C0FFFFE7802065C8589780010018
:106C0000E780A04717B501001305C5E39780010091
:106C1000E780A0468327840C8545414593E7070814
:106C20002324F40C97C0FFFFE78080268D451305D1
:106C3000000897C0FFFFE780A02597C0FFFFE7800F
:106C4000805237A507001305051297C0FFFFE780A4
:106C5000204E014597C0FFFFE7804054954505450C
:106C6000894717F7FF1F2303F7AC97C0FFFFE780A3
:106C70008054B7E700E013070006238DE74037078D
:106C8000000423A0E71097D0FFFFE78000D697D03D
:106C9000FFFFE78000E897000000E78060E99700C9
:106CA0000000E78000A097000000E78040B997E06F
:106CB000FFFFE780C0D597000000E780A05697004F
:106CC0000000E780801083A7040817050000130563
:106CD00005C4829797C7FF1F2380A770BC4C13067B
:106CE00000648545829797B0FF1FE780607001457B
:106CF0008280AD67371700409387A7AA1CC3B7E708
:106D000000E03707400023A0E71801000100B7F7B3
:106D1000070003C70701A5476316F70093974501CE
:106D200091C301A04111AE860146AA85254506C63C
:106D300097C0FF1FE780E0AAB240B7E700E037073F
:106D4000400023A0E710410182804111B2862E86C7
:106D5000AA852D4506C697C0FF1FE78080A8B240D0
:106D60000145410182809307000463ECC7041D7153
:106D7000A2CC2A840808A6CACAC886CE32C6978082
:106D80000100E780400CAD67371700409387A7AA42
:106D90001CC3B7E400E03709400023A02419010018
:106DA0000100B2461008A285294597C0FF1FE78061
:106DB00040A3F640664423A02411D64446492561E9
:106DC00082803955828041110D658D4506C697C078
:106DD000FFFFE7808001B71700408D6623A6D70A22
:106DE00017F5FF1F1305C5941387C70A9387870AF2
:106DF0001CC15CC5856689675CC958C114C518C9C2
:106E0000B7E70400B24003A3871E41010283814516
:106E1000B307B5008387070089E7172300006700E1
:106E200043E78505C205C181E5B7011106CE2307F9
:106E3000010001ED17A501001305455C9700000056
:106E4000E78020FDF240056182805800A947BA859D
:106E500029462548B376C502FD1793F7F70F9386A9
:106E60000603A304D700B356C5026375A8007D17B7
:106E70003685EDF33385F500D1B797A701009387E9
:106E800027581357C5003E9703470700011106CE48
:106E90002304E100135785003D8B3E97034707000D
:106EA00023060100A304E100135745003D8B3D89F3
:106EB0003E97AA970347070083C7070028002305CA
:106EC000E100A305F10097000000E78080F4F240A4
:106ED00005618280797117A501001305654B06D6FF
:106EE00022D426D24AD04ECE97000000E78060F22E
:106EF00017F5FF1F0355658397000000E78020F812
:106F000097E7FF1F83C7077217A501001305C54543
:106F100089C717A501001305A54497000000E78065
:106F200040EF17A501001305E54697000000E78034
:106F300040EE17A501001305654697000000E780A5
:106F400040ED114597000000E78060EE17B50100A5
:106F5000130545A397000000E780A0EB01459700CB
:106F60000000E780C0EC17B501001305A5A197004C
:106F70000000E78000EA1305C00497000000E780E6
:106F800000EB97D7FF1F83C7B72917A5010013058B
:106F9000253E89E717A501001305053E970000006F
:106FA000E78020E717A501001305C53F9700000003
:106FB000E78020E637A507001305051297000000BB
:106FC000E780E0E617A501001305453E97000000A5
:106FD000E78020E497E7FF1F83C7077717A5010025
:106FE0001305053A89E717A501001305E539970050
:106FF0000000E78000E217A501001305E53B9700BC
:107000000000E78000E117A501001305653B97002C
:107010000000E78000E017A501001305E53A97009E
:107020000000E78000DF17C5FF1F0355A538970054
:107030000000E780C0E417A501001305253997007B
:107040000000E78000DD17C5FF1F035505399700D5
:107050000000E780C0E217A501001305A5379700DF
:107060000000E78000DB17D5FF1F0355450497009C
:107070000000E780C0E017A5010013052536970042
:107080000000E78000D917D5FF1F035505029700C0
:107090000000E780C0DE17A501001305A5349700A6
:1070A0000000E78000D717D5FF1F03552500970084
:1070B0000000E780C0DC17A501001305E53297004A
:1070C0000000E78000D517C5FF1F0355651F970017
:1070D0000000E780C0DA17A50100130565319700AD
:1070E0000000E78000D3014497C9FF1F9389C97747
:1070F00097A401009384C4301949B307340183C7AE
:1071000007000A85050413D74700BD8B2697A6976D
:107110000347070083C70700230101002300E100A4
:10712000A300F10097000000E780A0CEE31724FD44
:1071300017A501001305452C97000000E78060CDDE
:107140000A8597F0FFFFE780A0960A84040883472A
:107150000400034514000904A2075D8D9700000098
:10716000E780E0D1E39584FEB25022549254025954
:10717000F24945618280411126C2E97797E4FF1FF9
:107180009384846B22C49387A7552E842381B400F3
:107190002E86AA8517E5FF1F1305456A06C62390AC
:1071A000F400A381040097800100E780C0C9930523
:1071B0002400C205C18117E5FF1F1305056897F07C
:1071C000FFFFE7808055B38784002382A7002181D9
:1071D000A382A700930564002244B240268592440E
:1071E000C205C181410117230000670083AA09C9B4
:1071F0009307000463E6B700170300006700E3F796
:10720000828017E5FF1F03452554828097E7FF1F03
:1072100083C7476289E717230000670083A782803E
:1072200097E7FF1F83C7A76599EF411106C697200F
:107230000000E780E09DB240854717E7FF1F23006D
:10724000F7644101828082806307053E6385053EC5
:107250001D71CAC8CEC686CEA2CCA6CAD2C4D6C21A
:10726000DAC05EDE62DC66DA6AD86ED6B947AA8911
:107270002E8963F9B706394697A501009385C5FCA9
:1072800097800100E780C0B931ED83C7E90013079B
:1072900010036394E702854717E7FF1F230CF75895
:1072A00017A50100130545FB97E7FF1F2393075818
:1072B00097000000E780E0B5E5A01307000317A5DD
:1072C0000100130565FCE395E7FE97E7FF1F2383A5
:1072D000075697E7FF1F239E075417A501001305C4
:1072E00025F9F9B797E7FF1F83C7C754639F07289E
:1072F000B706400001475946A5061314070141800F
:1073000063742433B384E90083C70400D91793F767
:10731000F70F6367F600B3D7F600858B0507F1FF1B
:107320003304894042044180BD4763FE87264146BD
:1073300097A50100938585F7268597800100E78052
:1073400020AE6314052617A50100130565F7970005
:107350000000E78000AC97000000E780E0B71795D9
:10736000010013056576A9B7B387490183C60700F5
:1073700097E7FF1F83D7E74BB9E39307A005639B0C
:10738000F600854717E7FF1F2315F74A97E7FF1F0A
:10739000238ED73A050A93170A01C183E3E627FD36
:1073A000F6406644D6444649B649264A964A064BB4
:1073B000F25B625CD25C425DB25D25618280854D8C
:1073C000639BB7039307500A639EF600894717E74C
:1073D000FF1F2310F746930750FA17E7FF1FA30775
:1073E000F7364DBF9307A005E386F6FA97E7FF1F30
:1073F0002391074445B7138717004207DA97418363
:107400002380D70017E6FF1F2315E6428D47E3F3DD
:10741000E7F817E4FF1F0344943397E7FF1F83C780
:10742000073322045D8C9307F4FFC207C1839306E0
:10743000F00DE3EDF6FA93076400C207C183E31B86
:10744000F7F493052400C205C18117E5FF1F13055A
:10745000053097F0FFFFE780402C33078B00834710
:10746000570003474700A207D98F17E7FF1F2312D2
:10747000073C6311F5108144630CB40197E4FF1FCE
:1074800083C4042DA20497E7FF1F83C7772CDD8CEC
:10749000170500001305E5D597F0FFFFE78060BFF3
:1074A0006385740963EF9B026388A4059307EC6509
:1074B0006383F40697E7FF1F83C787290547638027
:1074C000E70881CB1387A7051377F70F8D4663F97C
:1074D000E6081307F0072300E100A300F100894547
:1074E00095A8638994059387FA77E395F4FC97F060
:1074F000FFFFE780E00211A8A28517E5FF1F130533
:10750000252597F0FFFFE780E0CB014597F0FFFFCF
:10751000E78020B841B5A28517E5FF1F1305452375
:1075200097F0FFFFE78000D3CDB797F0FFFFE7802C
:1075300080DBE1BF97F0FFFFE78020E1F9B7930719
:1075400010F8130511002300F10097F0FFFFE7800A
:107550000000FD450A8597000000E78000C275B76E
:10756000A28517E5FF1F1305A51E97F0FFFFE78013
:10757000E08861BF9307F00789450A852310F10071
:1075800097000000E78060BF31B5BD6A396C014AE1
:1075900017EBFF1F130B8B1B938BFA55938CFA661B
:1075A000130DEC55CDBB6311F4083D4697A50100C2
:1075B000938545D2268597800100E780608611E596
:1075C00017A50100130505D259B3C14763FE87040F
:1075D000414697A50100938525D226859780010015
:1075E000E780008431E183C7040113071003639C23
:1075F000E700854717E7FF1F2308F71417A50100C9
:107600001305C5D075B11307000317A501001305B5
:10761000E5D2E39FE7C897E7FF1F2387071217A567
:107620000100130525D069B1CA854E8597C0FFFFBB
:10763000E78000BBB5B38280411126C2AE848D4580
:1076400022C406C62A8497C0FFFFE7806084B7176C
:10765000004099C803A5C70C418D23A6A70CB240D2
:10766000224492444101828003A5870C418D23A4CA
:10767000A70CF5B78347050003471500A207D98F6C
:10768000C2076177C18713072720639AE700834504
:1076900025003705040017030000670023FA8280E5
:1076A00017E6FF1F1306061E8147B2861303F00F6D
:1076B000A9483308F6000348080013F7F70F6307DB
:1076C000A80C630668008507E39517FF2947B38771
:1076D000E6002380A70097E7FF1F9387671B5DA83D
:1076E000411113D765001347170006C693F63500FE
:1076F000058B954791CA054699476387C600094699
:107700009D476383C600A14713F645003336C0008A
:1077100093F68503050685C2A145638BB604E14552
:10772000638AB604930580026388B60493058003D8
:107730006393B600914697E5FF1F2380F53C97E5DC
:10774000FF1F238BC53A97E5FF1FA387D53ABE8558
:1077500017A501001305C5CE97700100E780007AD8
:10776000B240854717E7FF1FA309F7384101828020
:107770008546D1B78946C1B78D4675BF17A50100AB
:10778000130585CE177301006700437717E7FF1FC6
:1077900013070710BA972380B700E147E302F5F417
:1077A00093077002E30CF5FC82802A872380050092
:1077B000814717E5FF1F1305E50C1308F00F294655
:1077C000B306F50083C606006396E60297E6FF1F40
:1077D0009386060CB69783C7070005452380F500FE
:1077E0009947636EF7029D4763FDE700E147630D2C
:1077F000F7008280638506018507E393C7FC014596
:10780000C5B7238005008280B737004003C7370023
:1078100083C7050093F70704D98F2380F500828082
:107820005D7152DC56DA5ED6716A97EBFF1F938B5F
:10783000EB3D8D6AA6C24EDE62D486C6A2C4CAC023
:107840005AD866D26AD06ECEC1495E8C97E4FF1FCB
:107850009384C404130A0A20938A7ADC17E9FF1F71
:107860000349C93DB3872B0183C7070093F7F70F7F
:10787000C9EFB787004003C76700058BE310077C9B
:1078800003C76700118BE30D077E83C75700918BF9
:1078900099E36F10200317E7FF1F0347473A854717
:1078A0006304F7006F10400197E7FF1FA387E724E9
:1078B00097E7FF1F2384070A97E7FF1F2382071616
:1078C00097E7FF1F2380072297E7FF1F238D0720DD
:1078D00097E7FF1FA384070897E7FF1FA3820714FA
:1078E00097E7FF1FA380072097E7FF1FA38D071EC1
:1078F00097E7FF1FA384072097E7FF1FA3810734A3
:10790000B787004011476F0070779307190093F70E
:10791000F70F3D476364F70617E7FF1F2300F732B1
:1079200097E7FF1F93878730CA9783C7070013071E
:10793000100293F7F703638EE71E6366F7040544AE
:107940006385871CE38C07620947638EE710130782
:107950000002E384E74EB7E700E03707400023A0CA
:10796000E71801000100629923000900FD1923A016
:10797000E71093F9F90FE39309EEE5BD97E7FF1FD1
:10798000238E072A71BF130730026388E70C63E870
:10799000E71613074002638CE70A13070003E39C12
:1079A000E7FA97E7FF1F93876727CA9703C7070080
:1079B000A1471377F70FE31BF71483C7640097E61B
:1079C000FF1F2383F61297E7FF1F83C797ED91C729
:1079D000FD5797E6FF1F2389F61097E5FF1F83C524
:1079E000F5EB97E7FF1FA381B71097E7FF1F83C74A
:1079F000E7EA13FB07089306000493F70706639F63
:107A0000D74C9307A009638DF51663EAB712930765
:107A1000F0056386F54A930750096384F52A01440B
:107A200097E7FF1F83C7570C1547E392E736B7E781
:107A300000E03707400023A0E71801000100B786E7
:107A4000004023808602130680FC6F00500EFD5715
:107A500017E7FF1F2309F708FDBDFD5717E7FF1FB5
:107A60002302F708CDBD17A50100130565B1977076
:107A70000100E780806097E7FF1F9387271ACA9766
:107A800003C40700014B97ECFF1F938CACF91374F0
:107A9000F40F17AD0100130D2DAF63478B0429457B
:107AA00097700100E780604A854717E7FF1FA30929
:107AB000F7F617E7FF1F230687F617E7FF1F230FC9
:107AC000F70237E700E0B70640002320D71801008F
:107AD0000100378600408347A60293F7370F23053E
:107AE000F6022320D71085BDB3876C0183C507003C
:107AF0006A85050B97700100E780404079BF854794
:107B000017E7FF1F230EF7F0B9B517E7FF1F13079D
:107B1000E7104A970347070097E6FF1FA380F6E4A4
:107B200097E6FF1F238DE6E217E7FF1F2308F7FC08
:107B30001DB5854717E7FF1F2302F7E229BD93070D
:107B4000400A6389F5349307200B6384F536930765
:107B5000100AE396F5EC838724000144E3D207EC96
:107B600097E7FF1F83C7B7D393F63700638A061AD8
:107B70000546638AC62209466395C61A1D4755A263
:107B800017E5FF1F0345A5D1C94797ECFF1F83CC1D
:107B90001CD197E5FF1F83C5A5D017E4FF1F034441
:107BA00034D06315F510CD476392FC10930770082D
:107BB000639CF5021307300FB7170E006308E4004B
:107BC0001307900DB7B704006314E40817E7FF1F0D
:107BD0002322F7F2BE8517A501001305659B977058
:107BE0000100E780A03125BD93078008639DF50063
:107BF000B307804013F4F70FB7774600938787CD1C
:107C0000B3D78702E1B793079008639AF500B307EB
:107C1000804013F4F70F91679387C766D5B7930732
:107C2000A008639BF500B307804013F4F70FB71764
:107C30003D0093870790E9B79307B008639AF50072
:107C4000B307804013F4F70F9167938797D04DBF28
:107C500093F5F5078D47639BF500B307804013F458
:107C6000F70FB7975B00938707D859BF8947639B86
:107C7000F500B307804013F4F70FB7770B00938735
:107C8000071BBDBF8547639AF500B307804013F417
:107C9000F70FDD67938767E3A5B7D28785F9B30749
:107CA000804093F7F70FB3D7FA020DB797000000A3
:107CB000E780409FA285668597000000E780809E50
:107CC000B9BB9305610017E5FF1F034545BD17E4E8
:107CD000FF1F0344D4BC97000000E78040AD93052C
:107CE0007100228597000000E78060AC3C0017E738
:107CF000FF1F232BF7F0834761002304F100834724
:107D00007100A304F100894717E7FF1F230EF7DC7A
:107D10008357810017E7FF1F2312F7B8094409B3FF
:107D2000154793F64700B336D00093F787038506CF
:107D300085C32146638BC7066146638AC70613065F
:107D400080026388C706130680036393C7009147C8
:107D500017E6FF1F2302D6DA97E6FF1FA38EF6D899
:107D600097E7FF1F238BE7D817E7FF1F034747B3AA
:107D70009376070497E7FF1F83C797B28DEE1377BB
:107D8000770C93067008630CD7021377F7078D46BC
:107D90006312D70CB307F040B7955B0093F7F70F6A
:107DA000938505D849A81947ADBF854755B7894779
:107DB00045B78D4771BF930670086311D70213074B
:107DC000300FB7150E006389E7021307900DB7B5A2
:107DD00004006383E7021307700845BF9306800C15
:107DE0006311D702B307F040B775460013F7F70FDA
:107DF000938785CDB3D5E70297E7FF1F23ACB7CEB6
:107E0000D9BB9306900C631CD700B307F04093F5E1
:107E1000F70F91679387C766B3D5B702F1BF930693
:107E2000A00C631DD700B307F040B7153D0093F7D2
:107E3000F70F93850590B3D5F5027DBF9306B00C7F
:107E4000E315D7F4B307F04093F5F70F91679387E5
:107E500097D0D9B78946631BD700B307F040B775F1
:107E60000B0093F7F70F9385051BF1B78546631A4F
:107E7000D700B307F040DD6593F7F70F938565E30F
:107E80005DBFD28535FBB305F04093F5F50FB3D553
:107E9000BA029DB783C72400C18B99C7854717E7EE
:107EA000FF1F2306F7C4A5BE97E7FF1F238107C462
:107EB000BDB6854717E7FF1FA301F7C48DB63C0089
:107EC00017E7FF1F2322F7D4094793070003231462
:107ED000F10097E6FF1F2389E6C02DBD6394075686
:107EE000A94763E5B742179701001307A7528A0510
:107EF000BA959C41BA97828717E4FF1F0344349ACE
:107F0000894C6306940D63E68C0685476303F40889
:107F10009307F00F17E7FF1F034707BD63F6E7005E
:107F200017E7FF1F2302F7BC97ECFF1F83CCCCBBE6
:107F30009307000413F4FC0F63F497011304000487
:107F400097E7FF1F938747CC03AD0700228626855E
:107F5000EA85B38C8C40229D97700100E780A0EEEB
:107F600097E7FF1F238297B997E7FF1F23AEA7C9A3
:107F700045BC8D47630CF40A9947E31BF4F89797C7
:107F800001009387A74F17E7FF1F232FF7C6A947C5
:107F900051B717E7FF1F034787CA97E7FF1F93876C
:107FA000A7B6494697950100938545566306870015
:107FB00097950100938585513E8597700100E78074
:107FC00080E817E7FF1F2321A7C4C947A1B797E699
:107FD000FF1F83C6C6C6054797E7FF1F9387C7B233
:107FE0006394E6023E85130670029795010093851F
:107FF000654F97700100E78000E517E7FF1F232515
:10800000A7C09307700239B73E85130630049795D1
:1080100001009385654797700100E780C0E217E78C
:10802000FF1F2323A7BE93073004EDB597E5FF1F7D
:1080300083C5E586179501001305C55697700100A5
:10804000E780C0EB054D97EDFF1F83CD4DBF97E552
:10805000FF1F83C5C584179501001305A5546398B8
:10806000AD0B97700100E78060E997E7FF1F83C7BA
:108070000783B5CBE36EF4E8179401001304444D75
:10808000638CB701179401001304044D63869701B4
:10809000179401001304C44D228597700100E780F6
:1080A00000FF1375F50F93071500860717E7FF1FED
:1080B000230CF7A48D4717E7FF1FA307F7A497E743
:1080C000FF1F938767A40147BE861376F70F8907C2
:1080D0006365A60297E7FF1F23A8D7B297E7FF1FA4
:1080E00083C787A205BD979701009387673F17E76E
:1080F000FF1F232BF7B0914731BD3306E400034641
:108100000600A380070005072380C7007DBF977086
:108110000100E780A0DE97D7FF1F83C74778E1D72C
:10812000E368F4DE179401001304843F638CA70115
:10813000179401001304443F6386970117940100CC
:1081400013040440228597700100E78040F4137502
:10815000F50F93071500860717E7FF1F2306F79A09
:108160008D4717E7FF1FA301F79A97E7FF1F938734
:10817000A7990147BE861376F70F8907E37CA6F41B
:108180003306E40003460600A380070005072380AA
:10819000C700D5B797D5FF1F83C565701795010038
:1081A0001305054197700100E78040D597E7FF1F51
:1081B00083C7579593E7470017E7FF1FA304F7947A
:1081C00083C7240017E7FF1FA30CF79289B8179500
:1081D00001001305253F97700100E78000EA97E74B
:1081E000FF1F9387E79183C7070017D7FF1F230758
:1081F000F76A17E4FF1F0344248F333480000DB067
:10820000179501001305453D97700100E780E0E6F2
:1082100097E7FF1F83C7178F93E7070117E7FF1F34
:10822000A302F78E83C7240017E7FF1F230AF78CEA
:108230006FF0EFFE179501001305453B97700100A5
:10824000E780A0E303C704007D8B51EFB7870040B0
:1082500003C767021377C70B136727002383E7025F
:1082600003C7A7021377C70B136727002385E7020D
:1082700003C7E7021377C70B136727002387E702BB
:1082800003C727031377C70B136727002389E70268
:10829000854717D7FF1F2303F76C17D7FF1F23014D
:1082A000F77817E7FF1F230FF78217E7FF1F230C4D
:1082B000F78297D7FF1FA383076A97D7FF1FA38172
:1082C000077697E7FF1FA38F078097E7FF1FA38C11
:1082D000078097E7FF1FA383078297E7FF1FA3800D
:1082E00007966FF0CFF389476312F70297D7FF1F06
:1082F00083C7075B9146638CD70863E0F604638EFF
:10830000E70C6369F70A05476380E70EFD5717D747
:10831000FF1FA30BF77C37074000B7E700E023A05F
:10832000E71801000100B78600401306F0FC238126
:10833000C60223A0E7106FF00FE213072008638244
:10834000E7086362F70213071008E391E7FC378739
:1083500000408347670293F7C70B93E72700230387
:10836000F7026FF0CFEB130730086389E7021307BA
:108370004008E39DE7F8378700408347270393F7DA
:10838000C70B93E727002309F7026FF04FE9378700
:1083900000408347270393F73707F5B73787004037
:1083A0008347E70293F7C70B93E727002307F702FA
:1083B0006FF0EFE6378700408347E70293F7370710
:1083C000F5B7378700408347A70293F7C70B93E7BA
:1083D00027002305F7026FF08FE4378700408347BB
:1083E000A70293F73707F5B737870040834767023F
:1083F00093F73707ADB71795010013052520977040
:108400000100E78080C797D7FF1F23890748D5B3AE
:10841000179501001305851F97700100E780E0C5DF
:1084200097D7FF1F239C074697D7FF1F9387C76BDC
:1084300003C40700894763F3870009441374F40FEA
:108440006FF00FDE13070002E392E7EC631B0B0AE9
:10845000638FF500930720026383F50817950100E9
:108460001305451E97700100E78040A945B5179593
:1084700001001305651A97700100E78000C00144F0
:10848000179D0100130D8D1AA14CB387840083C57D
:1084900007006A85050497700100E78020A6E316AF
:1084A00094FF178501001305256897700100E78088
:1084B000C0BC17D4FF1F0344A43E01E897D7FF1F99
:1084C0002380073C014B6FF0AFD58947E310F4E4FC
:1084D000854717D7FF1F2305F73A6FF04FD417D6FC
:1084E000FF1F0346D63B97D5FF1F83C5453B179516
:1084F00001001305251497700100E78020A06FF09C
:108500000FD26380F50693071002E399F5F497D52F
:10851000FF1F83C5E538179501001305A513977054
:108520000100E780A09D97D7FF1F23AF976C97D7D7
:10853000FF1F9387275C944383D7470017D7FF1FFC
:108540000347A75B17D6FF1F232AD6341D4497D6AF
:10855000FF1F2397F63497D7FF1F2384E7346FF06C
:108560002FCC97D5FF1F83C5A533179501001305A1
:10857000E50F97700100E780609897D7FF1F238170
:10858000073097D7FF1F239B07306FF02FF9254740
:10859000638FE7C89946378700406394D70223006A
:1085A0008702B7E700E0B706400023A0D718010014
:1085B0000100130600FC2301C70223A0D7106FF0AF
:1085C0008FB99306100A639FD70023008702B7E78D
:1085D00000E0B706400023A0D718010001001306F1
:1085E00080FCD1BF9306A009E381D7FE9306400A21
:1085F000E38DD7FC93062002639DD700B7E700E028
:10860000B706400023A0D71801000100230087020D
:10861000F9B78546E384D7FE93070008E300FBFE25
:10862000B7E700E0B706400023A0D718010001001B
:10863000130620FC23008702BDBF17D7FF1F034787
:10864000B74A6302F71E63E7E70295476300F71036
:108650009947630AF704B786004023800602B7E70C
:1086600000E03707400023A0E718010001001306CF
:10867000A0FC75B99307F005630AF700930750094A
:108680006306F70093071002E317F7FCB7E700E073
:108690003707400023A0E71801000100B78600401B
:1086A000130620FC69B117DBFF1F034BEB43930755
:1086B00000045A8D63F46701130D000497D7FF1F60
:1086C0009387875483AC07001374FD0F2286E685D9
:1086D000268597600100E7800077B3078B4066949A
:1086E00017D7FF1F2302F74097D7FF1F23AE8750EE
:1086F000B7870040630C0B022380A703B7E600E0B6
:108700003706400023A0C6180100010003C7270256
:10871000134707042381E70203C727021377C70F14
:108720002381E70223A0C6106FF0EFA22380070287
:1087300037E700E0B70640002320D718010001000A
:10874000130620FC2381C7026FF0AFB937870040C2
:108750008347370097D6FF1F83C6963A93F70708DB
:10876000D58FA301F700B7064000B7E700E023A0CC
:10877000D718010001001306A0FC35BD97D7FF1FD5
:108780009387C749CA9783C7070093F7F70FC1CFED
:1087900097D7FF1F83C7A74AD9E717D7FF1F0347FC
:1087A000B734930700026310F70883AD040017DDA8
:1087B000FF1F034DED0E97DCFF1F83CC7C0E17DBF4
:1087C000FF1F034B0B0EE6876A87DA866E8697D506
:1087D000FF1F83C5E50A179501001305A5EA9760F9
:1087E0000100E780A07197D7FF1F23A5B73197D766
:1087F000FF1F2383A73197D7FF1FA38F972F97D7EB
:10880000FF1F238C672F97D7FF1FA38A8706B7E721
:1088100000E03707400023A0E71801000100B786F9
:1088200000406FF04FA2B7E700E03707400023A0F9
:10883000E71801000100B786004015BD97D6FF1F5D
:1088400083C6E63F0547639CE60429472381E70288
:1088500009472383E7022385E70297D7FF1FA38FEA
:10886000072897D7FF1FA38C073CB7870040A38139
:10887000070017D7FF1FA305072805472383E70035
:10888000B640264496440649F259625AD25A425B8F
:10889000B25B225C925C025DF24D6161828029478D
:1088A0002381E70209472383E7022385E702238721
:1088B000E7022389E70255B717D7FF1FA301F7FC8B
:1088C0006FE01FFF854717D7FF1F2309F70817D74A
:1088D000FF1F2307F71417D7FF1F2305F72017D70C
:1088E000FF1F2302F7206FE0BFFE854717D7FF1F4A
:1088F0002306F70617D7FF1F2304F71217D7FF1F0A
:108900002302F71E17D7FF1F230FF71C17D7FF1FD0
:10891000A306070417D7FF1FA304071017D7FF1FCD
:10892000A302071C97D7FF1FA38F071A828041114C
:1089300006C697000000E78080FBB78700402380D1
:108940000700130740FC2386E7001307C004A38633
:10895000E70017D7FF1F130767F42398E70017D71F
:10896000FF1F1307A7F7239AE70017D7FF1F130767
:108970002703239CE70017D7FF1F1307A70E239E8B
:10898000E70029472381E70209472383E70223857C
:10899000E7022387E7022389E702A3810700930602
:1089A00000F8A380D700930690022380D700FD56DD
:1089B0002383D7002381E7009306000537E700E013
:1089C000230BD740B70640002320D71003C717005A
:1089D00013671700A380E700B24097D7FF1F2391CA
:1089E000071241018280411106C697000000E7800E
:1089F00000F0B787004023800700130700FC2386A0
:108A0000E7003147A386E70017D7FF1F130707E9E1
:108A10002398E70017D7FF1F130747EC239AE700B7
:108A200017D7FF1F1307C7F7239CE70029472381A8
:108A3000E70209472383E7022385E702A3810700B2
:108A4000930600F8A380D700930690022380D700F6
:108A5000FD562383D7002381E7009306000537E7FF
:108A600000E0230BD740B70640002320D71003C7F0
:108A7000170013671700A380E700B24097D7FF1FC6
:108A80002390070841018280F1679387072017D759
:108A9000FF1F2321F706854717D7FF1F231EF70463
:108AA000A14717D7FF1F230AF70497D7FF1FA386F5
:108AB000070497D7FF1F2383070497D7FF1F23813E
:108AC00007DC97D7FF1FA38C07DA814717D5FF1F55
:108AD000130545DBFD5517D6FF1F130666DB294737
:108AE000B306F5002380B600B306F6002380060027
:108AF0008507E397E7FE97D7FF1FA38807FE97D761
:108B0000FF1FA38607FE97D7FF1F238107FE97D776
:108B1000FF1F238C07FC97D7FF1F238B07FC97D7DA
:108B2000FF1FA38507FC97D7FF1F238207FC814700
:108B300017D6FF1F1306860D4147B306F6002380A4
:108B400006008507E39BE7FE828017D7FF1F0347D8
:108B5000070F85476316F700170300006700E3E877
:108B6000170300006700E3DC411122C406C617D7D3
:108B7000FF1F0347C70C85472E8613F4F50FAA8500
:108B80006317F70417D5FF1F130585E597600100EC
:108B9000E780602B97D7FF1F238407E8B787004043
:108BA00023848702B7E600E03706400023A0C618FA
:108BB0000100010003C7A7021377C70F2385E7024F
:108BC000B240224423A0C61001454101828017D53E
:108BD000FF1F1305A5D497600100E780C02697D733
:108BE000FF1F238D07D6B787004023828702B7E691
:108BF00000E03706400023A0C6180100010003C7AB
:108C000067021377C70F2383E7025DBF411106C6D2
:108C100097000000E78080E7B240410117030000A1
:108C20006700E3F2411106C697F0FFFFE78080BFBF
:108C300097D7FF1F83C797D2A1CB97D5FF1F83C5B7
:108C400005D289C917D5FF1F130585D197E0FFFF0E
:108C5000E780C05F97D7FF1FA38207D097D7FF1F7A
:108C6000238E07E837E700E0B70640002320D71837
:108C700001000100378600408347660293F7370FF3
:108C80002303F6022320D710B2404101828041C95C
:108C9000D9C597D7FF1F83C7A7E6D1C3011122CC3F
:108CA0004AC84EC656C25AC006CE26CA52C42E89DB
:108CB000AA890144930A0004371B03006377240345
:108CC000B3078940C207C183BE8463F4FA009304EA
:108CD0000004C204C180130A1BD497D7FF1F83C7A7
:108CE000E7C79DE37D1A631C0A00F2406244D24448
:108CF0004249B249224A924A024B0561828097F06A
:108D0000FFFFE78020B2D1BF338589002694A68576
:108D1000420497000000E78060E5418045B782800B
:108D200097D7FF1F9387070418429C4383D64500BB
:108D30000345070083C5C700035646006396A50098
:108D400083D5E700638DD502011106CE2386A700E7
:108D50002397D700B705CF00DC4B9385757D0507BA
:108D60007D162EC2230001003AC42316C10023172A
:108D7000D10099C30A858297F24005618280828082
:108D8000411122C417A4FF1F130484675C4C06C65C
:108D900091CBC84B01C9B7E70400BC5782975C4C24
:108DA00023AA0700B240224441018280DC4DDC4B03
:108DB00081CFB7E70400904503A38705914517D5F8
:108DC000FF1F034565FA02838280B7E7040003A30F
:108DD0000705A14517D5FF1F034505F902836D71EE
:108DE0003C083EC6B707E500232291103EC8AA847E
:108DF0003C083285232611103ECA232481102320EB
:108E000021112E8997300000E780605A2A849795B7
:108E100001009385A58A177501001305256E9760DB
:108E20000100E780A00DA285179501001305C595E7
:108E300097600100E780800C294597600100E7807A
:108E4000C010B705CB009385757D680097100000B2
:108E5000E780E05FA285680097300000E7808047E8
:108E6000014781467000CA85268597200000E7806B
:108E7000608305CD2A849795010093852584177515
:108E800001001305A56797600100E7802007A28510
:108E9000179501001305059097600100E780000613
:108EA000294597600100E780400A8320C110032410
:108EB000811083244110032901105161828097D7CA
:108EC000FF1F938727EA18429C43797122D406D664
:108ED0000348070083C807012A8483D64500035549
:108EE00046006396080183D82701638DD802238842
:108EF000070105072399D7003708CC00DC4B13087E
:108F0000787D3ACC1307F5FF42CA23080100231EDF
:108F1000E100231FD10099C7080832C62EC48297EA
:108F20003246A245228597000000E78080EBB250D0
:108F3000225445618280797131469775010093858D
:108F4000A54C280006D697600100E780C0EF97A7E0
:108F5000FF1F83D7E74A231B0100231C0100231DA9
:108F60000100231E0100231F010099E3C167FD17C3
:108F7000231AF10097A7FF1F83D7A74891EB97D734
:108F8000FF1F938727DE9C439C43DC4783D7070062
:108F900097A6FF1F9386C646231BF100D84E83D7A2
:108FA0004600231CF1005C4B91CB97A7FF1F83C7A2
:108FB000974581EB97000000E780C0DCB250456127
:108FC0008280FD1717A6FF1FA30FF6420356070165
:108FD00083C706014C472800230FF100973000009B
:108FE000E780602C97D7FF1F9387C7D79C43014723
:108FF0009786010093860676884330004C089710C8
:109000000000E780206A5DD975B799C9B7E7040009
:1090100003A30705A14517D5FF1F0345E5D4028328
:1090200082805C4EDC4BB9CFB1CD411122C41775A3
:1090300001001305A54C2E84978501009385456D8D
:1090400006C697600100E78060EBA28517850100E6
:109050001305456E97600100E78040EA2945976057
:109060000100E78080EEB7E704002244B24003A38A
:10907000870517D5FF1F034525CF130640069145E9
:10908000410102838280411122C417A4FF1F1304EF
:10909000E4341C4C06C689C7DC4399C34C4882970C
:1090A000584CB7E70400BC57484B82975C4CB24021
:1090B000224423AA07004101828017A7FF1F13073C
:1090C000E733834707009306F00B850793F7F70F05
:1090D00063E9F60097A6FF1F2382F63203450700D7
:1090E0008280930700F8FDB78357450099E37D55CB
:1090F0008280011122CC17A4FF1F130464305C4C42
:109100004AC84EC6DC4B52C406CE26CA56C2B289E5
:109110002E8A2A898DC7B7E70400FC5F829797D70C
:10912000FF1F938727C29C431307301FB307F540E7
:1091300071556375F70697000000E780A0C4930798
:10914000D00D7D5563EC3705B7E4040093878900A3
:10915000B858832AC401139507014181029723AAB5
:10916000AA00484C584921E7978501009385455846
:10917000177501001305853897600100E78000D856
:10918000178501001305C56397600100E78000D7CC
:10919000294597600100E78040DB5D55F24062445D
:1091A000D2444249B249224A924A056182801387D9
:1091B0004900B705CF002319E5009385757D31057A
:1091C00097100000E780A028484C834569003105CE
:1091D00097300000E7800010484C4E86D28531055C
:1091E00097300000E780200C7146CA8517A5FF1F45
:1091F0001305052197600100E780E0C4FC5C8297BD
:109200000326C90097D7FF1F23AEA7B211CABC4CD3
:10921000854517D5FF1F034525B582970145BDBF7D
:1092200097000000E78060D1D5BF411106C622C477
:1092300026C217D4FF1F130424B397000000E78051
:1092400060B4B7E40400FC4C0345040085458297F4
:1092500003450400224403A3C405B2409244A1453F
:1092600041010283411126C297D4FF1F938484AF2A
:109270009C4006C622C44AC0D5C3DC43C5C35CC1FA
:109280002300B5002A84978501009385A5411775B1
:1092900001001305A52697600100E78020C6294537
:1092A00097600100E78060CA9C4023A4070023A2C6
:1092B000070097A7FF1F93876712DC4FDC4B91C70E
:1092C000295597000000E78040DC97A7FF1F938790
:1092D0002713DC4FDC4B89C797000000E78020F59F
:1092E00037E904008327C905894517D5FF1F0345C2
:1092F000A5A782978327C905914517D5FF1F034569
:10930000A5A682979C4003A3470163090300228519
:109310002244B2409244024941010283B2402244B5
:1093200092440249410182800111328506CE22CC4D
:1093300026CA2E8497300000E7806007AA849785AC
:10934000010093856539177501001305251B97608A
:109350000100E780A0BA0307840003566400835528
:109360004400A686178501001305453F976001005C
:10937000E780C0B8294597600100E78000BD97A746
:10938000FF1F83C70706639D9700014597000000F4
:10939000E780A0CF81450A8597000000E780C0ECF8
:1093A000F2406244D244056182806D7123248110B1
:1093B000232611102322911093F745002E846387F2
:1093C00007143C083EC0B707E5003EC23C083EC457
:1093D000231701002318010023190100231A01009B
:1093E000231B010097A7FF1F83D747FF99E3C1679E
:1093F000FD172316F10097A7FF1F83D747FE91EBB8
:1094000097D7FF1F938707969C439C43DC4783D7DE
:10941000070017A7FF1F130767FC2317F100544F1E
:10942000835747002318F100DC4AA1E79785010024
:109430009385C52E177501001305450C9760010033
:10944000E780C0AB178501001305053E976001005A
:10945000E780C0AA294597600100E78000AF134567
:1094600044008320C11003248110832441105161E2
:10947000828097A7FF1F83C7D7F62555D9C3FD174D
:1094800017A6FF1FA30FF6F403D6060183470701B3
:10949000CC460A85230BF10097300000E780A0E05E
:1094A00097D7FF1F9387078C9C4317A7FF1F1307AE
:1094B000E7F2978601009386662788430A866C0048
:1094C00097100000E780001EAA8451D997850100FB
:1094D0009385C524177501001305450297600100A7
:1094E000E780C0A1A685178501001305A534976004
:1094F0000100E780A0A0294597600100E780E0A473
:10950000268597000000E78040B891BF93F72500BB
:109510009DC7B7E70400BC474146814528088297AC
:10952000255597000000E78040B628089305F00F06
:1095300097000000E78040D3134524001DB793F740
:10954000150081CB97000000E780209F1345140091
:1095500009BF93F78500014589D717A7FF1F034768
:1095600097EA97A7FF1F9387A7E90DC3D84F584BDA
:1095700011CF37E70400384F9047854517C5FF1FC7
:109580000345857E029713458400E1BD97F0FFFFF8
:10959000E780407FCDBF5C4D411106C688C317C729
:1095A000FF1F2321F77CB7E7040083A707081705EF
:1095B00000001305C5DF8297B24097C7FF1F2385C0
:1095C000A77A01454101828001113335A000A3072C
:1095D000A100B7E7040083A7471706CE1306F100E2
:1095E0008545130550308297F24005618280828064
:1095F000411122C406C697B7FF1F83C777C205442F
:1096000089EF97C7FF1F83C7E701014499E717B4A4
:10961000FF1F0344E4C01344140022859700000098
:10962000E780C0FA178501001305852709E417852F
:1096300001001305E5272244B240410117630100F0
:109640006700C38B797122D4A30F010037E40400B3
:109650008327841726D24AD006D6AA842E891305DA
:1096600050309305F10132C6829732468347F101AB
:1096700093150601C18185CB01452EC697000000D8
:10968000E780C0F483274417B2454A86268582972F
:10969000054597000000E78060F3B25022549254D1
:1096A000025945618280832744174A86268582971E
:1096B000EDB741119397050122C406C626C2C187A2
:1096C0002E8463D40702B7E40400FC5417A5FF1FDF
:1096D000034505D6829719C1BC5482972165218D17
:1096E000B240224492444101828093F715008DC715
:1096F000B7E7040083A7471A17A6FF1F130646D231
:1097000097C5FF1F9385056717A5FF1F034545D222
:10971000829713451400E9B793F725000145E9D373
:1097200097C7FF1F83C7876685E7B7E7040003A8CD
:10973000871A1307401F97A7FF1F83C767CF81466C
:1097400013064006994517C5FF1F0355A5630298E8
:109750001345240071B797C7FF1F83D7A76263988B
:10976000A70217C7FF1F2310B76217C7FF1F231DCC
:10977000C76017C7FF1F231AD7602E861785010001
:1097800013058519BE8517530100670023771785D8
:1097900001001305E519176301006700038E0357E5
:1097A000450097C7FF1F83D7E75D6318F702C167BE
:1097B000F91717C7FF1F2327F75C97C7FF1F23A5BC
:1097C000075C97C7FF1F238D075A97C7FF1F238F7B
:1097D000075A170300006700E3E11785010013052E
:1097E000251517630100670043897D15954763E2DE
:1097F000A71C17870100130727090A053A951C4182
:10980000011122CC06CEBA972E84828717850100DB
:109810001305851297600100E7802086A1A203C787
:10982000250099476311F7022E8597000000E78015
:1098300040F783456400178501001305E510975034
:109840000100E780A06B97B7FF1F238B079C17854C
:109850000100130525117DBF03C725009547631936
:10986000F702C16717C7FF1F0357C751F91703D581
:10987000A5006309F702B7E7040083A7C71782971B
:10988000178501001305050F97500100E780E07E62
:10989000854717B7FF1F2305F798178501001305A4
:1098A000E50F8DBF97C7FF1F239EA74C83D7E50009
:1098B00097C6FF1F2399F64C83D7050197C6FF1F54
:1098C0002394F64C83D7250197C6FF1F239FF64AA2
:1098D00097C7FF1F2386074A631BE502B7E704000B
:1098E000BC4F096613060690894517A5FF1F03455F
:1098F00025B482970356E4008355A4001785010020
:109900001305850897500100E780405F51B7930722
:10991000700F2316F100B7E7040083A7870D17A681
:10992000FF1F0346E6B06C0082974DF9854717C7C5
:10993000FF1F2307F7445DB7178501001305C50610
:10994000D1BD83C5250091476392F50217850100BB
:109950001305050797500100E7802072970000006B
:10996000E78040C9F2406244056182809947639272
:10997000F502228597000000E780A0E2834564009D
:1099800017850100130545FC97500100E78000573B
:10999000D1BF9547639AF50083471400E1F317851B
:1099A000010013052504BDB5178501001305050445
:1099B000E1BF82803757315F97A7FF1F938787A842
:1099C000130777D598C39356C5001787010013076F
:1099D00067F1BA9683C5060093568500BD8ABA968C
:1099E00003C6060093564500BD8A3D89BA962A975C
:1099F00083C6060003470700238407002383D7009C
:109A0000A383E7002382B700A382C70097A7FF1FA5
:109A1000938747A42383B700A383C7002384D70079
:109A2000A384E7008280411106C697000000E7800A
:109A3000A0F8B7E7040083A7871417A6FF1F130633
:109A400066A0D54501458297B2404D4697A5FF1FB8
:109A5000938545A01305703041011703000067008E
:109A6000A3BE61712324811A37E40400832704080C
:109A70002326111A2322911A2320211B232E311968
:109A800017050000130525C3829717A9FF1F1309A7
:109A9000299A994785442300A900231CF100978542
:109AA0000100938525E39307400617750100130510
:109AB000E5A4231CF1082308910097C9FF1F93898F
:109AC000C9C697500100E780604383D50900178518
:109AD0000100130525DF97500100E780204229454A
:109AE00097500100E780604603D509009700000009
:109AF000E78080EC83274417100885451305503014
:109B000082978327441717A6FF1F1306A694CD45F7
:109B10001305703082978327441717A6FF1F13067B
:109B20006691B54513056030829783274417300846
:109B300089451305103182978327441730098945D9
:109B4000130520318297832744159305000A0D459C
:109B50008297832744159305000A11458297A30530
:109B600091002306910002CD23080100230C01007F
:109B70008327841630099145130570408297832707
:109B800084161306B100854513050040829783278C
:109B9000841670008545130510408297832784162C
:109BA00030088545130520408297832784161008C6
:109BB0008545130550408297832704157D5582976C
:109BC000832744137D5582977D5597A0FFFFE7803B
:109BD000C0AB8327440C829797A0FFFFE7802087C4
:109BE0008327841417A6FF1F1306C685D545014594
:109BF000829789471306700F814528092306F100D3
:109C00009780FFFFE780A0508D471306000881452D
:109C10002808230CF1089780FFFFE780404F914709
:109C2000230CF100976701009387C77E984383C791
:109C300047003AC8230AF10097D0FFFFE780A09CB5
:109C400070008545054597A0FFFFE78020AB3009F0
:109C50009305700F094597A0FFFFE78020AA300801
:109C6000930500080D4597A0FFFFE78020A9100885
:109C70009545114597A0FFFFE78040A8C16717C72A
:109C8000FF1F13072710F9171CC32322070017957E
:109C9000FF1F1305A57997A0FFFFE78000A5832785
:109CA000C41D17C5FF1F1305650C82973C4803456B
:109CB0000900854582978320C11A0324811A8324D1
:109CC000411A0329011A8329C1195D618280C16784
:109CD00017C8FF1F0358080BF9176301F8083DCD9B
:109CE000B5CD011126CAB7E4040083A7841222CCA3
:109CF0002E862315B10006CE2A8401478146ED4504
:109D0000428582972AC611ED178501001305C5BE4D
:109D100097500100E7806036F2406244D24405610A
:109D20008280FC440356A100A28582972C0017C5AF
:109D3000FF1F0355250597A0FFFFE780C0A769DD3A
:109D400017850100130585BC97500100E780E032BC
:109D500083A7C412ED45280082977DBF82800DC580
:109D600085471797FF1FA30CF76C9797FF1F238951
:109D7000076C35469795FF1F9385C56B13056030BB
:109D8000170300006700438C9797FF1FA389076A9A
:109D9000E9BF97C7FF1F83C767FFA9EFC16717C751
:109DA000FF1F035727FEF9176306F7044111854784
:109DB00022C417C7FF1F230BF7FC37E404007C4CB9
:109DC00006C689451795FF1F0345856682970323BD
:109DD000841A2244B2409797FF1F83C7676517C54F
:109DE000FF1F035525FA1307401F81463146994549
:109DF0004101028382806D7123248110232611107A
:109E000023229110328401CD8947630AF502832011
:109E1000C110032481108324411051618280178571
:109E20000100130565BDAE8497500100E780E02472
:109E3000A285268597B0FFFFE780A061C9BFB7E77D
:109E40000400FC472800829717850100130585BB95
:109E500097500100E78060228347810039C41307CF
:109E6000000B6380E7021387A7051377F70F8D4672
:109E700063EDE602A285280097C0FFFFE78000F8A7
:109E800079B78547E3F587F8834591001775010099
:109E900013050598B335B00097A7FF1F2386B72099
:109EA00097500100E78080059DB703479100A20706
:109EB000B966D98F1387E6556384E70C636DF704A1
:109EC0002D671307B755638FE708636AF7002967A3
:109ED0001307A755638FE708A2852800A1BF316744
:109EE0001307C7556388E70635671307D755E3950A
:109EF000E7FE8947E3FD87F097000000E780A0E9CF
:109F00009305E4FFC205C1811305A1009790FFFFEF
:109F1000E780002DEDBD3D671306F7556389C70641
:109F2000636DF6009386E665E398D7FAA28528006C
:109F300097C0FFFFE7800032D9BD9306F766638DB7
:109F4000D7041307F777E399E7F897C0FFFFE78097
:109F5000205D75BD0146A285280097C0FFFFE78000
:109F6000801575B5A285280097C0FFFFE780C02245
:109F700079BDA285280097C0FFFFE780A02341BDDF
:109F8000A285280097C0FFFFE780C02349B597C08E
:109F9000FFFFE7804035A5BD97C0FFFFE780E03AAF
:109FA000BDB5C16717C5FF1F0355C5DDF9176307A9
:109FB000F500B7E7040003A3C7170283828017F3F5
:109FC000FFFF670023631783FFFFE702A30F2A84C5
:109FD00008452E89B28919C900C1971500009385DB
:109FE000A586610597300100E780600481447D5AB1
:109FF00097100000E780E03963C7A40481449710FC
:10A000000000E780003A63C8A40497C7FF1F938746
:10A0100027D89C43DC47B307F94091872302F4001B
:10A02000638309048327C900B307F4409587A3021B
:10A03000F4001C4C89C79C4799C3228582971783DB
:10A04000FFFF6700630B5C44139714008504BA9705
:10A050002390470171BF1C48139714008504BA97D9
:10A060002390070069BF832789000547B307F440A1
:10A070009587A302F40083570400638EE7028DC323
:10A0800009476384E7040D47E395E7FA97870100E2
:10A09000938707EA1CCC97870100938767EA11A88A
:10A0A00097870100938747B01CCC9787010093875F
:10A0B000A7B05CC8BDBF978701009387E79B1CCC06
:10A0C000978701009387479CEDB797870100938797
:10A0D000E7EA1CCC97870100938747EBD9BF95E54A
:10A0E0001783FFFFE702A3FF00461844834794004D
:10A0F00075839D8B6317F70097100000E78060B4AD
:10A1000048C41783FFFF6700C3FF82801783FFFFE8
:10A11000E70243FB13893500C16442094111AA8952
:10A120000144F11413590901054A2EC69710000085
:10A13000E7802026B2456348A4000145410117830A
:10A14000FFFF670063FB83A7090013171400BA978A
:10A1500083D707006388B7006394970063742A016C
:10A160000504E1B70545D9BF1783FFFFE702A3F454
:10A17000AA892E89328BB6843A8ABE8A97A00000BB
:10A18000E78000FE71C9268597200000E780C00C9B
:10A190008D4763E7A7007D551783FFFF670023F511
:10A1A00083DB440097100000E780A0242A849710E6
:10A1B0000000E78040259307740031443305850291
:10A1C00063CDA70297100000E780A022971000003F
:10A1D000E78020222A8497100000E780C02293079E
:10A1E000740031443305850263C3A704971000004F
:10A1F000E78020209307450029A897100000E780FA
:10A200008020330585021307F0179307C017E35F1B
:10A21000A7FA2D55E3C277F963040B02D68652865E
:10A22000A6854A8597200100E78000BDB5B7971045
:10A230000000E780401D330585029307C5FFD1BFAD
:10A24000832749001385C90083D5270097000000A4
:10A25000E78000EC61F581B769553DBF97C7FF1FE7
:10A26000239AA7B297C7FF1F938787B2904381476E
:10A270000C463307F500420741836393B7008280A1
:10A280005446139847008507C2962390E600D5B739
:10A2900097C7FF1F9387C7AF9C4303C58700828082
:10A2A00017C5FF1F035505AF82801783FFFFE70225
:10A2B00003E3C1671387D7FF630BE502636AA70057
:10A2C000F1176300F50201451783FFFF670063E3A1
:10A2D0001387E7FF6302E502FD171D8D1335150097
:10A2E000E5B797500000E780A0297D15C5BF9750BE
:10A2F0000000E78020FED5BF97500000E78040FCBB
:10A30000EDB71783FFFFE70283DD4111AA84014403
:10A310002EC697100000E780C008B2456348A4002D
:10A32000014541011783FFFF6700A3DD9C4813151A
:10A3300014003E9583570500E385B7FE0504C9BFA9
:10A3400003485500814693F7F60F63E507018147FF
:10A350003E858280584593975600BA9703D72700C9
:10A360006316B70003D70700E304C7FE8506E1BF05
:10A370008346450001479377F70F63E4D700814791
:10A3800011A81C45131657000507B29703D60700FE
:10A39000E313B6FE3E8582801783FFFFE70283D278
:10A3A00093170501C18797CAFF1F938A6A9E635B53
:10A3B000F00883A70A00C0479C4703570400198D83
:10A3C000420541816368F500014422851783FFFF40
:10A3D000670083D212052A94CDBFDC47139449004D
:10A3E000014A3E94834744006341FA02014A83478D
:10A3F00054006349FA028509C20993D9090183A768
:10A400000A009847E3EBE9FCC1B71C4413195A0052
:10A41000A6853E994A8597000000E780C0EE05E1D9
:10A42000050AC9B75C4413195A00A6853E994A85A6
:10A4300097000000E78020ED19E1050A4DBFE30C0D
:10A4400009FA61B7AA8481495DBF1783FFFFE7025C
:10A4500003C91C452A8481E79307C5001CC51C4419
:10A46000231204001CC09307F00F63EDB70093F5AF
:10A47000F50F228597200000E780C0E51783FFFFD6
:10A48000670023C893940501C167C18063F9F50093
:10A49000A685228597200000E780E0E8C5B7C18146
:10A4A00093F5F50F228597200000E780A0E2A685AE
:10A4B000228597200000E780E0E3C9B797C7FF1F18
:10A4C0009387078D884382801C4599C797C7FF1FD4
:10A4D00023A0A78C014582807D55828097C7FF1FEE
:10A4E0009387078B984383474500484792073E95DB
:10A4F00082801783FFFFE70283BE617100451C184D
:10A500003EC6B70780013EC81C183ECA83574400A8
:10A5100002CE02D002CC231EF100834784002A8998
:10A5200002D22301F1023C083ED402D6970000007B
:10A53000E78000FB835705002316F10297500000C7
:10A54000E78040C72307A1025C4003556400F18304
:10A5500013F717008347F10252055181F99BD98FF8
:10A56000A307F10297100100E780607839CDAA8433
:10A570000355050097A00000E78060BF83D7040063
:10A580002AD26800231CF10083D72400231DF10088
:10A590001C4803D647008C4397200000E780A0D0DA
:10A5A0008347B400CA8617760100130666468117F2
:10A5B000A305F4006C00481097200100E780C083D9
:10A5C0005D611783FFFF6700C3B32155D5BF1C45ED
:10A5D000B1CF03C5A700894613576500630BD702A7
:10A5E0008D46630ED70285466300D70213074006E7
:10A5F0003305E50203C7B700418B15CB83C7B7000E
:10A60000BD8B3355F54082801375F5031307803EEB
:10A61000C5B709671375F50313070771D1BF37274E
:10A6200009001375F5031307077CD9B7014582802C
:10A630001783FFFFE702A3AA03A98500630C09049F
:10A640008347B900AE8493F7070E85C3034599008D
:10A65000930520030D810505B305B5028844610506
:10A6600097300100E780C0AC35A02E859700000030
:10A67000E78020F62A8419CD97000000E780605C0F
:10A680008325C900B307B54063FA87002E94B3054C
:10A69000A440E9F51783FFFF6700A3A685457DBFAA
:10A6A0001783FFFFE702A3A32A8403D50500011146
:10A6B00032C636C43AC22EC002CA02CC02CE97A01D
:10A6C0000000E780C0AA82452ACA22852ECC9700C6
:10A6D0000000E780E0E003570500231EE1009750EB
:10A6E0000000E78020ADA24632469247230FA1002A
:10A6F00036874C08B2862285014697000000E78025
:10A70000E0A605611783FFFF6700A39F1783FFFF84
:10A71000E702E39C61711C183EC6B70780013EC882
:10A720001C183ECA3C0800453ED4AA8402CC02CE86
:10A7300002D002D202D697000000E78060DA835789
:10A74000050035592316F10297500000E78080A6D6
:10A750002307A10209C48357440081EB21594A858C
:10A760005D611783FFFF6700C399035564005205BD
:10A77000518197100100E78080572A8965D183476E
:10A78000B40093F7070E99C71305840197300100B1
:10A79000E780409C83574400231EF10083478400D8
:10A7A0002301F1025C4003550900D98313F7070820
:10A7B00083471102231CA10093F7F707D98FA30049
:10A7C000F10283572900231DF1005C40F18313F748
:10A7D00017008347F102F99BD98FA307F10297A0D5
:10A7E0000000E780C0982AD235D9834794006800DA
:10A7F000139757008347B400FD8BD98FA305F4004E
:10A800001C4803D647008C4397200000E780A0A98E
:10A81000A687177701001307A71F740005464C1081
:10A82000268597000000E78060942A890DD9834728
:10A83000B400A685FD8BA305F40097000000E78017
:10A8400060DF31BF1783FFFFE7026389832485FE42
:10A850002A844111268597000000E78080D783472E
:10A8600034FF93F7070E8DCB2AC62685970000008C
:10A87000E78060C809CD834734FFB245FD8BA3094B
:10A88000F4FE91C5228597300100E780608A41017E
:10A890001783FFFF6700E3867DD98327C4FF2685E2
:10A8A000829775F5834734FF93F7070E91C722858A
:10A8B00097300100E780008A032584FE970000009E
:10A8C000E78000E5E9B71773FFFFE702437E9C418D
:10A8D00041112A8903C7070089472E8493566700D0
:10A8E0006380F6040D466388C6049307F00763048B
:10A8F000F7022E8597200000E78060ABAA8481498B
:10A90000C16B130C490097B7FF1F938767489C439F
:10A91000984763E4E90441011773FFFF6700E37C94
:10A9200003D745008547E3F8E7FE2E859720000012
:10A93000E78040ADE1B703D74500E3FEE7FC2E8595
:10A9400097200000E780A0A6AA8422859720000017
:10A95000E78000A8C204C98C5DB7DC470355A90095
:10A96000139A49003E9A93170501C187635DF00071
:10A9700083570A006397A70263E774038327CA001B
:10A98000034D5A002DA0A1672167A98F1307F7EF88
:10A99000E374F7FE6397090097000000E7802091B9
:10A9A00061FD85098DB783278A00034D4A00835DC9
:10A9B000A90003576900216A138BC7003AC6814A70
:10A9C00033CA4D01631E5D0197B7FF1F9387C73CD4
:10A9D0009C43E1DBA2866286814526858297D1B7BA
:10A9E000A1679387F7EF930C4BFF63F24703B245E0
:10A9F0005A8597F0FFFFE780A0710DC103278B00F8
:10AA0000104709CE10436382C4023107D5BFEE85DB
:10AA1000668597000000E780008F71F993861A0021
:10AA200093FAF60F130B0B0271BF835644005C437D
:10AA3000E3E9F6F622853AC697200000E7802081F8
:10AA4000A1679387D7042A8A035D4400324763E8ED
:10AA500097008347D90093E707F8A306F9001C473E
:10AA600066852286E2858297C1670844FD17337A9E
:10AA7000FA00529508C02312A40125B797B7FF1F0B
:10AA8000938707319843814715C31447814763FF74
:10AA9000D500939745004C47BE9519C903C755008B
:10AAA00081476375E600DC451606B2973E858280D5
:10AAB00003C745008147E37BE6FE16069C45F5B7D4
:10AAC0001773FFFFE7020360AA892E8A814497BAB1
:10AAD000FF1F938AEA2B83A70A00984763E6E400E6
:10AAE0001773FFFF67004361DC471394440001497B
:10AAF0003E9413BB140083474400634BF9000149A3
:10AB000013BB140083475400634FF9008504E1B779
:10AB10000844931759005287DA860146A2853E956C
:10AB200082990509C9BF4844931759005287DA86AC
:10AB30000546A2853E9582990509E9B71773FFFF7F
:10AB4000E702E359814517F5FFFF1305054897B75D
:10AB5000FF1F2391072497000000E780A0F61773DA
:10AB6000FFFF6700035A97B7FF1F938767229C4335
:10AB700095C31773FFFFE7028356814517F5FFFF63
:10AB80001305A54497000000E780C0F31773FFFF8B
:10AB90006700235782801773FFFFE702A35237E451
:10ABA00004008327841241112315E100AE89328904
:10ABB000368A3A8681460147ED45AA8482972AC69D
:10ABC00021C90356A100D28597400100E780A02744
:10ABD0008327C413CE8526858297058905C98327D7
:10ABE000440D2314210101462C00268582972A84D6
:10ABF00001C9B7E7040083A7C712ED452800829773
:10AC0000228541011773FFFF6700034F4944D5B701
:10AC10006554FDB75C41FD175CC182801773FFFF6F
:10AC2000E702E34BB7E70400FC5F829795473305E3
:10AC3000F50281450D811773FFFF6700834C177381
:10AC4000FFFFE702C349B7E70400FC5F829795471F
:10AC50003305F5020D811773FFFF6700834A1773F1
:10AC6000FFFFE702C347B7E7040083A7870B03553D
:10AC7000050082971773FFFF6700A3481773FFFF54
:10AC8000E702E345035505003287AE861796FF1F9E
:10AC90000356668297B5FF1F938545109700000005
:10ACA000E780A0EF1773FFFF6700A3451773FFFF4F
:10ACB000E702E342B7E7040083A7C7178297177339
:10ACC000FFFF670003441773FFFFE7024341B7E745
:10ACD000040083A7871397B5FF1F9385250C8297E0
:10ACE00001451773FFFF6700C3411773FFFFE702BA
:10ACF000033FB7E7040083A7C71F81451785FF1FE0
:10AD00000355657782971773FFFF6700833F1773BB
:10AD1000FFFFE702C33CB7E7040083A7871397B59B
:10AD2000FF1F9385A508829701451773FFFF6700F2
:10AD3000433D1773FFFFE702833AB7E7040083A799
:10AD4000C71F81451785FF1F0355E5788297177345
:10AD5000FFFF6700033B1773FFFFE70243382E85B1
:10AD600097800000E780C0B297800000E780C0EFC6
:10AD70001773FFFF6700E3381773FFFFE7022336FF
:10AD800097800000E780C0F91773FFFF6700633703
:10AD90005C49E1175CC95CC583572501A1072319EC
:10ADA000F50083570501A1072318F5008280F147BC
:10ADB0003305F50297B7FF1F938747019C433E95E4
:10ADC00082808D476315F60803D74600854763F0F8
:10ADD000E7081773FFFFE7028330368536842E8934
:10ADE00097100000E780A05C29C9835744009314A2
:10ADF0000501C18063E39704228597100000E78076
:10AE0000005BFD14231294009307A0026300F50277
:10AE10009307B0026307F50293079002631FF500E2
:10AE2000228597000100E780A08801A80146CA8515
:10AE3000228597A00000E78040B31773FFFF6700EB
:10AE4000432C228597100000E7806007FDB78280C1
:10AE500097B6FF1F9386C6F79C42014599CF98434A
:10AE6000D44217B6FF1F2325E6F66396D70097B6A0
:10AE7000FF1F23A1E6F61385C7FE82801773FFFF2D
:10AE8000E702E32597000000E780A04B71443305FB
:10AE90008502914597900000E78000EC11E565552B
:10AEA0001773FFFF6700E32597B7FF1F23AEA7F0D7
:10AEB00097000000E780E0483305850291459790B0
:10AEC0000000E78060E961DD97B7FF1F23A0A7F0CE
:10AED00097000000E780E04697B7FF1F2390A7EE9A
:10AEE00097000000E780E04597B7FF1F2399A7EC84
:10AEF00097770100938707B717B7FF1F2324F7EC55
:10AF000097070000938707E917B7FF1F232AF7EA7F
:10AF1000014579B71773FFFFE702631CAA8517B5D0
:10AF2000FF1F1305A5E997100000E780605F177306
:10AF3000FFFF6700031D1773FFFFE702431A970027
:10AF40000000E78060FD97100000E780E05E97B7A3
:10AF5000FF1F9387E7E79C4391CF1387C7FE19CB69
:10AF600083D5C7FF17B5FF1F130505E7972001001D
:10AF7000E780001C1773FFFF6700A3181773FFFF1C
:10AF8000E702E31597000000E780C0EC09CD834796
:10AF900085002A8493F7070499EB0355E500970091
:10AFA0000000E78080F91773FFFF67008315834770
:10AFB000C5009304450117B9FF1F130969E185E333
:10AFC000832709005CC997B7FF1F23A397E0832756
:10AFD0004900F1FB97B7FF1F23AE97DEE9B7FD17D6
:10AFE0002306F500610597800000E780A0D983075C
:10AFF000840063CB07048347840093E707F82304A6
:10B00000F400B7E704009C5F82974205A94741819D
:10B010003375F5028347840093F707FCC98F230437
:10B02000F4008347D4003E951C402318A40089CF28
:10B03000984319CB8347C4005040814585073305A9
:10B04000F502420541810297832709005CC897B742
:10B05000FF1F23AF97D68327490089E797B7FF1FC4
:10B0600023AA97D68347C4009DDF8355040117B5F3
:10B07000FF1F130565D697200100E780600B25B7F9
:10B080001773FFFFE702A30597B7FF1F938707FA20
:10B090009C4701448583858B85E3AE84B2853A86DF
:10B0A00097100000E780204F2A8419C597100000F0
:10B0B000E7806045829408CC22851773FFFF670004
:10B0C00043041773FFFFE702E3FF41112E8932C6E5
:10B0D000AA8997000000E780C031324713060502B5
:10B0E000CA86970500009385C5CC17B5FF1F1305C9
:10B0F000E5CC97000000E780E0F82A8425C9930496
:10B10000C50097000000E780E0411946AA85268522
:10B1100097100000E78020198545268597100000CC
:10B12000E780001517750100130585914E9583453D
:10B130000500268597100000E780C0195C4831465D
:10B140008145A1075CC85CC483572401E11723191A
:10B15000F40083570401E1172318F4001C4C3E85CA
:10B160009770FFFFE780A0FAA30425012285410123
:10B170001773FFFF670043F81773FFFFE70223F61B
:10B180004111AA842EC632C497100000E780003A0D
:10B19000004DB2452246834784000CC050C093F74F
:10B1A000F70393E707042304F4002318040026851B
:10B1B00097100000E780203583479400A9462317A5
:10B1C000A40013D7370005073307D7029D8B8507E7
:10B1D0002306F400A306E40083C70401D8488507CA
:10B1E000230FF7FE17B7FF1F130787BE5843232A05
:10B1F00004009307440129E317B7FF1F232CF7BC72
:10B2000017B7FF1F2326F7BC17B4FF1F1304C4BCD6
:10B21000228597200100E780E0E31C44858B5D8D4B
:10B2200019E58145228597200100E78060F0410102
:10B230001773FFFF6700E3EC1CC317B7FF1F232B37
:10B24000F7B8D9B71773FFFFE70263E99705000066
:10B25000938565B7014597000000E78000B0014580
:10B260001773FFFF6700E3E91773FFFFE70223E7A8
:10B2700097000000E78080B01773FFFF670063E866
:10B280008347C500A5E31773FFFFE70243E52A8460
:10B290000355E50097000000E78000C821C18347FF
:10B2A000840093F7F7FB2304F4001C4091C7DC43B0
:10B2B00081C74C400145829797000000E78080B924
:10B2C00017B5FF1F130545B197200100E78080E8FF
:10B2D0000355E40097000000E78020C61773FFFFC6
:10B2E000670023E282801773FFFFE70243DF97B70F
:10B2F000FF1F9387E7AD97050000938565C817B5D5
:10B30000FF1F130565AD23A0070023A207009720A8
:10B310000100E780C0D11773FFFF670083DE1C4D7B
:10B3200091CFDC4381CF1773FFFFE70243DB8345F7
:10B33000070082971773FFFF6700A3DC828097B72F
:10B34000FF1F9387A7AB9C4303C50700828097B775
:10B35000FF1F9387A7AA9C4303C51700828097B756
:10B36000FF1F9387A7A99C4303C52700828097B737
:10B37000FF1F9387A7A89C4303C54700828097B708
:10B38000FF1F9387A7A79C4303C53700828097B709
:10B39000FF1F9387A7A69C4303C55700828097B7DA
:10B3A000FF1F9387A7A59C4303C56700828097B7BB
:10B3B000FF1F9387A7A49C4303C57700828097B79C
:10B3C000FF1F9387A7A39C4303C58700828097B77D
:10B3D000FF1F9387A7A29C4303C59700828097B75E
:10B3E000FF1F9387A7A19C4303C5A700828097B73F
:10B3F000FF1F9387A7A09C4303C5B70011E11D451C
:10B40000828097B7FF1F9387679F9C4303C5C70040
:10B41000828097B7FF1F9387679E9C4303C5D70021
:10B42000828097B7FF1F9387679D9C4303C5E70002
:10B43000828097B7FF1F9387679C9C4303D50701C2
:10B44000828097B7FF1F9387679B9C4303C52701A3
:10B45000828097B7FF1F9387679A9C4303D5470164
:10B46000828097B7FF1F938767999C4303D5670135
:10B47000828097B7FF1F938767989C4303D5870106
:10B48000828097B7FF1F938767979C4303C5A701E7
:10B49000828097B7FF1F938767969C4303C5B701C8
:10B4A000828097B7FF1F938767959C4303C5C701A9
:10B4B000828097B7FF1F938767949C4303C5D7018A
:10B4C000828097B7FF1F938767939C43885782803A
:10B4D00097B7FF1F938787929C4303D5C70282804B
:10B4E00097B7FF1F938787919C4303D5E70219E124
:10B4F0001305800C828097B7FF1F938727909C438A
:10B5000003C50703828097B7FF1F9387278F9C434C
:10B51000C85B828097B7FF1F9387C78D884382805F
:10B5200097B7FF1F9387478D8843828019E17D5528
:10B530008280F5DE984265DFFDD917B7FF1F13073C
:10B54000E7AE1847AA877155058B631D072403C50D
:10B5500007001547E37DA7FC03C737001305F00577
:10B560007D171377F70FE364E5FC03C35700E3008F
:10B5700003FC83C86700E38C08FA03C777004945DA
:10B5800079171377F70FE364E5FA03C7A7001148AB
:10B590001305F7FF1375F50FE36BA8F803CE9700BB
:10B5A0000D481305FEFF1375F50FE362A8F803C8F5
:10B5B000B7006309080065181378F80F1305600DCC
:10B5C000E36705F703C5C700794879151375F50FCB
:10B5D000E36FA8F403C8D7000D457D181378F80F62
:10B5E000E36705F503D80701930E40175118420889
:10B5F00013580801E3ED0EF303C8E7007D18137834
:10B60000F80FE36605F303C827017D181378F80FD8
:10B61000E36F05F103C88700C54E75181378F80F5E
:10B62000E3E70EF103D86701856E938EBEE06D18D7
:10B63000420813580801E3EC0EEF03D847016D18D8
:10B64000420813580801E3E40EEF03D88701791884
:10B65000420813580801E36C05ED03C8A7017D18E3
:10B660001378F80FE36505ED03C5B7011D487D1597
:10B670001375F50FE36DA8EA03C5D7017148791575
:10B680001375F50FE365A8EA03D5E7011308E00F8A
:10B690007D1542054181E36CA8E803C507024948CE
:10B6A00079151375F50FE364A8E8C85301C937C8C5
:10B6B00034005915130858BFE36BA8E603A88702A6
:10B6C00037C53400130555BF5918E36205E717A5C0
:10B6D000FF1F2323C57203C6050117A5FF1F232FD4
:10B6E000F5700545E375C5E403D82501D0493376E7
:10B6F0000603E31E06E203C61501E30A06E217A6E7
:10B70000FF1F2329B66E83C5270001466387A50066
:10B7100003C61700F1453306B60283C70703930536
:10B72000C00272971A071307C70516031A979608DF
:10B730004697B387B70241553E97329742074183F8
:10B740006362E8061773FFFFE70263993685978007
:10B750000000E780806B97000100E780004B2A849F
:10B7600097A00000E780605D2A9497F00000E780D2
:10B7700040292A9497900000E78080842A9497F0CB
:10B78000FFFFE780E06F2A9497400000E780009772
:10B790002A9497700000E780809F22951773FFFF1F
:10B7A0006700239682801773FFFFE70243934111DE
:10B7B000A307A10097A00000E78080C89305F100CF
:10B7C000170500001305E5B597F0FFFFE780802F10
:10B7D000014541011773FFFF6700A3921773FFFF35
:10B7E000E702638D17B4FF1F130444840328840009
:10B7F00079599368180097B4FF1F23AD1483137809
:10B80000180063100802BA84BE89368B328A2E89EA
:10B81000AA8A97F0FFFFE780E0A77D15269519E536
:10B8200031594A851773FFFF6700638C97F0FFFF5C
:10B83000E78040A67D152695A167E353F5FE97B7EF
:10B84000FF1F9387A7B598433E8C814B01CB0145E1
:10B8500097F00000E7800047933B15004A85DA86A1
:10B860005686D28597900000E780A0502A8911CD96
:10B870001C44F99B17A7FF1F232EF77A83270C0080
:10B88000CDD3E3800BFA829769BF268597A7FF1F68
:10B8900023A0077A97F0FFFFE780809C4146CE8582
:10B8A00017B5FF1F1305058297300100E780A059E7
:10B8B00097D00000E780209C0325040B97D0000060
:10B8C000E780E09F054597D00000E780E0A60545AA
:10B8D00097000000E78060EDA9B797A7FF1F938747
:10B8E000E7749C47858BEDC71763FFFFE702237F53
:10B8F00017A5FF1F1305457B97A7FF1F23A80772F6
:10B9000097A7FF1F23A6077297A7FF1F23A40772FD
:10B9100097200100E780008497500000E780C0F87E
:10B9200097100100E780804F97100100E780805555
:10B9300097A7FF1F9387076E9C4391C70545978084
:10B940000000E780202397A7FF1F938767569C433B
:10B9500099C741657D1597700000E78020A597F095
:10B960000000E780C04097D00000E780609297B762
:10B97000FF1F9387A7809C43139717016356070007
:10B9800097F00000E780E0AF97A7FF1F23AC077296
:10B9900097A7FF1F23AA077297A7FF1F23A8077265
:10B9A00097A7FF1F23A6077297000000E780008C6F
:10B9B00097000000E780A07597F0FFFFE780401830
:10B9C00097F00000E78020D91763FFFF67006373DB
:10B9D000828097A7FF1F938767658843828097A718
:10B9E000FF1F9387A764C8438280B7E7B00093879F
:10B9F000075063E1A70297A7FF1F93872763D843E8
:10BA0000FD576367E50097A7FF1F23A3A762814740
:10BA10003E858280B957EDBF1763FFFFE702236CB5
:10BA200097800000E780A07497800000E78000778F
:10BA30001763FFFF6700E36C1763FFFFE70283688C
:10BA40002A849304140201112E85B289A685214609
:10BA500036C63A8997300100E780803C0DE9B2464E
:10BA600038082686CE851305940497500000E78099
:10BA7000A04021462C084A8597300100E780403AD3
:10BA80001335150005611763FFFF6700E366014585
:10BA9000D5BF1763FFFFE70283649305450617A52B
:10BAA000FF1F1305E53597100100E78060681763F5
:10BAB000FFFF670003651763FFFFE7024362411161
:10BAC0002EC697F0FFFFE780C017B24588C141013D
:10BAD0001763FFFF6700E3621763FFFFE702835E00
:10BAE000AA842E8497800000E780406BAA89854550
:10BAF000228597000000E780E07D83C7E401138979
:10BB0000940899E313890403CE85228597000000E9
:10BB1000E780407C214693051902228597000000AA
:10BB2000E780607897A7FF1F938747508C43228553
:10BB300097100000E780C082214693858402228509
:10BB400097000000E78020761763FFFF6700C35A65
:10BB50001763FFFFE7022356397197F00000E78073
:10BB600020B49305400661E997800000E780405FBC
:10BB70006302051497A7FF1F83C7472A13B717004F
:10BB800097A6FF1F238CE628014499CFC16417A90B
:10BB9000FF1F1309A9499309400EFD1497000000E7
:10BBA000E78020836342A40A97F0FFFFE7806009E3
:10BBB0004169B7290900096AFD7A2A8B81447D19F8
:10BBC0009389F97B130A0A71938A8AC79700000048
:10BBD000E780208063D7A4041304400EB387840257
:10BBE00017A7FF1F130787440324070B3E948357AF
:10BBF000C4016382270B18403307EB4063EAE90076
:10BC0000834744008507B3874703D6976365F708E2
:10BC100001468145094597F0FFFFE780C04AAA8B9E
:10BC200029E597400000E780C08285476317F50645
:10BC300089659385057117A5FF1F1305651C97106E
:10BC40000100E780E04E95A0B30734030327090BFA
:10BC5000BA9703D7C7016308970003C75700A382A9
:10BC600007002382E700050415BF9305C500228560
:10BC700097000000E78080E65E85228697650100D8
:10BC8000938545DD97F0FFFFE780404F5E85971075
:10BC90000000E780608A850415BF97A7FF1F938780
:10BCA000E7389C478D83858BC1F721611763FFFFC0
:10BCB0006700E34301468545094502D002D202D41C
:10BCC00002D697F0FFFFE7800040AA8479DD97F065
:10BCD0000000E780209C1389C4002A8481454A859E
:10BCE00097000000E780005F0C4041464A859700BE
:10BCF0000000E780405B832944006385090C4E8582
:10BD000002D802DA02DC02DE97300100E780203838
:10BD10002ACE141005462C0808184ECC9750000067
:10BD2000E780200A1375F50F51ED8355840093E5E4
:10BD300025004A8597000000E780E05E11460C1060
:10BD40004A8597000000E78000560146976501008C
:10BD50009385C5D0268597F0FFFFE7802042268592
:10BD600097000000E780407D5C40A1D301468545F7
:10BD70000D4597F0FFFFE7800035AA841DD54840A8
:10BD80001389C40097300100E78060302AC64A85D5
:10BD900097000000E780404C3246636FC5004C407E
:10BDA0004A8597000000E7800050014681452685BE
:10BDB00097F0FFFFE780803C268597000000E78032
:10BDC000A077E5B583558400ADB71763FFFFE702A1
:10BDD000033197A7FF1F938767259C471DC193E7F2
:10BDE000870017A5FF1F1305A50117A7FF1F232312
:10BDF000F72497100100E78080311763FFFF670089
:10BE00004330DD9B17A7FF1F2326F7229730000042
:10BE1000E78020647DF117A5FF1F130565FE9710CD
:10BE20000100E7802033D1BF1763FFFFE702A3289B
:10BE30004169AA892E8AB28A368BBA8B814417ACA3
:10BE4000FF1F130CAC1E930C400E7D1997F0FFFFE3
:10BE5000E780205863C4A40001443DA033849403C8
:10BE600083270C0B3E948357C401638627055A87AA
:10BE7000D6865286CE851305040397000000E7801E
:10BE8000E0BB01C923800B0022851763FFFF670019
:10BE900003268347F40185C35A87D6865286CE850A
:10BEA0001305940897000000E78040B909C585474D
:10BEB0002380FB00D1BF850451BF835745006380B9
:10BEC000071E1763FFFFE702E31F01112A84970093
:10BED0000000E780C04D09C985476309F506056183
:10BEE0001763FFFF6700432197E00000E780407B76
:10BEF0007DF5835744004947ED9BE392E7FEC1453A
:10BF0000228597000000E7804033AA8422859700AD
:10BF10000000E780204F0357440002CE91472A8952
:10BF2000631AF700228597000000E780A0513C08C3
:10BF30002ACC3ECE97E00000E780C0755C55C5D3A3
:10BF400074084A86A6850545829751BF0357440069
:10BF5000D147E3F6E7F8032A0400C169014997AA2B
:10BF6000FF1F938AAA0C130B400EFD1997F0FFFFD9
:10BF7000E7802046634FA90E2285032A040097001C
:10BF80000000E780C042A1452A8922859700000071
:10BF9000E780A02AAA84228597000000E780804AD3
:10BFA00014402A86AA8978082685CA859700000049
:10BFB000E780C0E7AA8405D503C7F4018947631564
:10BFC000F7008347C10181DF5546D28513856400A0
:10BFD00097300100E78020E7014597800000E78067
:10BFE000001901C583D7C401A5E797A7FF1F938751
:10BFF000E7039C4793551900858913D73700058BB4
:10C0000001CF8983858B6399B70001452EC69700C0
:10C010000000E780C0DBB2454E8597800000E780D6
:10C02000A01E0346C1012A849375190026859790A6
:10C030000000E780203935C1268597800000E78021
:10C040002018268511C0014597800000E780404BED
:10C0500097300000E780E03F8547E312F5E883C7AB
:10C0600054001307F00FE38CE7E68507A382F40082
:10C07000BDB5B304690383A70A0BBE9483D7C4017B
:10C08000638B37015546D2851385640097300100D4
:10C09000E78000D955DD0509D1BD5DD86DB7828037
:10C0A0001763FFFFE702030297800000E780400B61
:10C0B00005C1C164014417A9FF1F130929F793099A
:10C0C000400EFD1497F0FFFFE780A030634EA40000
:10C0D00017A5FF1F1305C5D297100100E7802003A5
:10C0E0001763FFFF67004301330534038327090B00
:10C0F0003E958357C50163889700231205009780FA
:10C100000000E780E00B050475BF97A7FF1F93872A
:10C11000E7F19C478D83858B8DE31763FFFFE70273
:10C1200003FC17A5FF1F1305A5CD97100100E7809D
:10C1300060021763FFFF6700C3FC82801763FFFF85
:10C14000E702E3F9970500009385C5A017A5FF1F37
:10C15000130505CB97100100E78060ED1763FFFF23
:10C16000670023FA1763FFFFE70263F78841B7E729
:10C170000400BC5B050542054181829709C58547DE
:10C180002300F50005051763FFFF670083F783C7EA
:10C19000F5FF2E858507A38FF5FE828083C7F5FF07
:10C1A000FD1793F7F70FA38FF5FE99EF1763FFFFC6
:10C1B000E702E3F2B7E70400BC571385F5FF829767
:10C1C0001763FFFF6700E3F382801C4103574500BC
:10C1D0008D8FBA951CC12312B5003E85828093D7FE
:10C1E0008500A2051441DD8D835745001387E6FFC6
:10C1F00018C189072312F50013D685004111238F3A
:10C20000B6FEA38FC6FE4101828018419307F7FF57
:10C210001CC18357450085072312F500A30FB7FE05
:10C220008280835745008D8F2312F5001C41BE95F7
:10C230000CC12E858280AA8703D7470008410D8F45
:10C24000AA952392E7008CC38280184108453305E4
:10C25000A740828083574500035765001D8F1C410E
:10C2600008453385A7403305A74082801763FFFF49
:10C27000E702E3E641112EC62A8497000000E7801A
:10C28000A0FDB2456373B50001A083574400084088
:10C29000BE952312B4003E9541011763FFFF67006E
:10C2A00043E61763FFFFE70283E341112E84B28563
:10C2B00032C697000000E780A0FB3246A285973087
:10C2C0000100E78040B841011763FFFF670063E3A7
:10C2D0001763FFFFE702A3E02E8485459700000067
:10C2E000E78000F9230085001763FFFF670063E123
:10C2F0001763FFFFE702A3DE41112317B100894551
:10C3000097000000E780C0F68347E1002300F500B6
:10C310008347F100A300F50041011763FFFF6700A9
:10C3200043DE1763FFFFE70283DB93D78500A20597
:10C330004111DD8D2317B100894597000000E7808A
:10C3400020F38347E1002300F5008347F100A300B9
:10C35000F50041011763FFFF6700A3DA1763FFFFD2
:10C36000E702E3D71397850193D78501C1669386CA
:10C3700006F0D98F13D78500758FD98FA20537079F
:10C38000FF00F98D4111DD8D2EC69145970000000B
:10C39000E78000EE6C00114697300100E780A0AA0C
:10C3A00041011763FFFF6700C3D51763FFFFE70273
:10C3B00003D31C41854503C4070097000000E780B4
:10C3C00080E622851763FFFF6700A3D31763FFFF93
:10C3D000E702E3D01C414111894503C7070083C729
:10C3E00017002307E100A307F10097000000E78092
:10C3F00080E30355E10041011763FFFF670063D04D
:10C400001763FFFFE702A3CD1C414111894503C714
:10C41000070083C717002307E100A307F100970077
:10C420000000E78040E08357E100410113D5870019
:10C43000A2075D8D420541811763FFFF670063CC52
:10C440001763FFFFE702A3C90C4141112A8411467B
:10C45000680097300100E780009F91452285970092
:10C460000000E78040DCB247C166938606F0139770
:10C47000870113D58701598D13D78700758F598D83
:10C48000A2073707FF00F98F5D8D41011763FFFF9A
:10C49000670023C71C45BE950CC18280AE879443BC
:10C4A00091E6584101EF0CC15CC1828003C757007F
:10C4B00013671700A382E700B687D5B70CC3EDB7A3
:10C4C000AA87084119CD1841D44398C36313D500F6
:10C4D000D8C32A87034657009376160081E62320A7
:10C4E00007008280944381CA8C4203A847008CC312
:10C4F00063930601CCC3799A14C3A302C70036879D
:10C50000D1BF1C45DC471D8DB777DBB6938777DB42
:10C5100009853305F502420541818280F147B385E3
:10C52000F50248452E958280834745008507230202
:10C53000F50082801763FFFFE70263BA2A8409E4EB
:10C540001763FFFF6700E3BB83474400F5DBFD177C
:10C5500093F7F70F2302F400E5F71C4403D72700F5
:10C5600005072391E700DC4399C3228582974C4855
:10C5700089CD83475400898B99E71C4422859C47C9
:10C580009C439C478297232A0400004023200400F8
:10C590007DB71763FFFFE70283B48357250041117E
:10C5A0002EC681EB0144228541011763FFFF67001E
:10C5B00043B5035705008147F146E305F7FEB38510
:10C5C000D702404585072E948345440008C4F5F5FD
:10C5D000B247AA8481E7232A040009A81C456C00FD
:10C5E00022859C439C43829748C84DDD8547231292
:10C5F000F400B24723200400231804002319F40098
:10C600005C485CC483D72400FD172391F40061BF0C
:10C610001763FFFFE702A3AC97A7FF1F938747802D
:10C6200088432326050023240500410597100100B7
:10C63000E78040B21763FFFF6700A3AC1763FFFFFB
:10C64000E702E3A91794FF1F1304847D1C404111E6
:10C6500099CF9C472300B5002AC65CC19700000013
:10C66000E78040FB1C40DC4399C33245829741017F
:10C670001763FFFF6700E3A80347450029E3584D10
:10C68000AA877D551DCF1763FFFFE70243A51CC393
:10C69000DC479796FF1F23A5E678F156130507019F
:10C6A0002390D7009705000093850502971001009D
:10C6B000E780E09701451763FFFF670083A47D557E
:10C6C000828082801763FFFFE70263A10111614648
:10C6D000814528009760FFFFE78060A39797FF1FC1
:10C6E000938707749C4328009305F00FDC473EC6F0
:10C6F00097000000E780C0F405611763FFFF670043
:10C7000043A09797FF1F9387A7719C43D847A167C2
:10C710009387C702631EF70A397106DE22DC26DA28
:10C7200080004AD84ED652D456D23285B284970071
:10C730000000E780C0C7AA89268597000000E7802F
:10C7400020C92318A4FC268597000000E78040C874
:10C750002319A4FC268597000000E78060C783D7D3
:10C7600044000A8A231AA4FC858393F7F70F230E4B
:10C77000F4FC8607BD0793F7073F3301F1408A8A2F
:10C7800001498347C4FD6367F902CE85130584FC24
:10C79000232C54FD97000000E78080EA52811301AA
:10C7A00004FCF2506254D2544259B259225A925A5D
:10C7B00021618280268597000000E78060C1931781
:10C7C0001900D69705092390A7001379F90F55BFD3
:10C7D00082809797FF1F9387A7649C43D847A167E0
:10C7E0009387A702631AF70A397106DE22DC26DA7C
:10C7F00080004AD84ED652D456D23285B2849700A1
:10C800000000E780C0BAAA89268597000000E7806B
:10C8100020BCFD572318A4FC26852319F4FC97009F
:10C820000000E780E0BA83D744000A8A231AA4FCF8
:10C83000858393F7F70F230EF4FC8607BD0793F764
:10C84000073F3301F1408A8A01498347C4FD63678A
:10C85000F902CE85130584FC232C54FD97000000BB
:10C86000E78000DE5281130104FCF2506254D2547E
:10C870004259B259225A925A2161828026859700E4
:10C880000000E780E0B493171900D69705092390BC
:10C89000A7001379F90F55BF82809797FF1F9387E1
:10C8A00027589C43D847A16789076310F70A397155
:10C8B00006DE22DC26DA80004AD84ED652D456D282
:10C8C0003285328997000000E78060AEAA894A85E8
:10C8D00097000000E780C0AF835749000A8A2318F9
:10C8E000A4FC858393F7F70F230CF4FC8607BD07A0
:10C8F00093F7073F3301F1408A8A8144834784FDDF
:10C9000063E7F402CE85130584FC232A54FD9700C7
:10C910000000E780E0D25281130104FCF25062541F
:10C92000D2544259B259225A925A216182804A8580
:10C9300097000000E780C0A993971400D69785045C
:10C940002390A70093F4F40F55BF82809797FF1FA1
:10C950009387074D9C43D847A1679387E704631EDD
:10C96000F70A397106DE22DC26DA80004AD84ED674
:10C9700052D456D23285B28497000000E78020A3BB
:10C98000AA89268597000000E78080A42318A4FCCC
:10C99000268597000000E780A0A3231AA4FC268523
:10C9A00097000000E780C0A283D744000A8A2319B9
:10C9B000A4FC858393F7F70F230EF4FC8607BD07CD
:10C9C00093F7073F3301F1408A8A01498347C4FD49
:10C9D0006367F902CE85130584FC232C54FD970070
:10C9E0000000E780E0C55281130104FCF25062545C
:10C9F000D2544259B259225A925A216182802685D4
:10CA000097000000E780C09C93171900D69705098E
:10CA10002390A7001379F90F55BF82809797FF1FC6
:10CA2000938707409C43D847A1679387C704631A3D
:10CA3000F70A397106DE22DC26DA80004AD84ED6A3
:10CA400052D456D23285B28497000000E7802096F7
:10CA5000AA89268597000000E7808097FD57231854
:10CA6000A4FC2685231AF4FC97000000E78040967A
:10CA700083D744000A8A2319A4FC858393F7F70F10
:10CA8000230EF4FC8607BD0793F7073F3301F140FF
:10CA90008A8A01498347C4FD6367F902CE8513057D
:10CAA00084FC232C54FD97000000E78060B952817C
:10CAB000130104FCF2506254D2544259B259225A22
:10CAC000925A21618280268597000000E78040907D
:10CAD00093171900D69705092390A7001379F90F2A
:10CAE00055BF82809797FF1F938787339C43D84712
:10CAF000A167DD076317F7041753FFFFE702235E03
:10CB000079713285328497000000E780408A2AC616
:10CB1000228597000000E780A08B2311A1022285C7
:10CB200097000000E780A088B2452300A1022808F2
:10CB300097000000E780C0B045611753FFFF670012
:10CB4000435C82809797FF1F9387872D9C43D8472C
:10CB5000A167938787046317F7041753FFFFE70262
:10CB6000035879713285328497000000E780208471
:10CB70002AC6228597000000E78080852311A10244
:10CB8000228597000000E7808082B2452300A10241
:10CB9000280897000000E780A0AA45611753FFFF0F
:10CBA0006700235682809797FF1F938767279C43D0
:10CBB000D847A1679387A7046312F7021753FFFFB3
:10CBC000E702E35101112800814597000000E7804A
:10CBD00020A705611753FFFF6700A3528280979734
:10CBE000FF1F9387E7239C43D847A167938757028A
:10CBF0006319F7021753FFFFE702634E01113285F5
:10CC000097F0FFFFE780A07A2308A1008145280064
:10CC100097000000E780C0A205611753FFFF67007F
:10CC2000434E82809797FF1F9387871F9C43D84767
:10CC3000A1679387E702631BF7041753FFFFE7021F
:10CC4000034A01113285328497F0FFFFE780407874
:10CC5000AA84228597F0FFFFE7808077854709E95E
:10CC6000228597F0FFFFE78080744205B337A0006C
:10CC700028008145231891003ECA97000000E780F4
:10CC8000209C05611753FFFF6700A3478280979799
:10CC9000FF1F9387E7189C43D84799476313F7080A
:10CCA0001753FFFFE702A34379713285328497F06F
:10CCB000FFFFE780C06F2AC6228597F0FFFFE7805D
:10CCC00020712310A102228597F0FFFFE780206EDC
:10CCD0002301A102228597F0FFFFE780406DA301A9
:10CCE000A102228597F0FFFFE780606C2302A1027A
:10CCF000228597F0FFFFE780806B2313A102228536
:10CD000097F0FFFFE780A06AB2452314A10228082C
:10CD100097000000E780C09245611753FFFF67004E
:10CD2000433E82809797FF1F9387870F9C43D84786
:10CD3000A1679387C7036313F7081753FFFFE70241
:10CD4000033A79713285328497F0FFFFE7802066DD
:10CD50002AC6228597F0FFFFE78080672310A10293
:10CD6000228597F0FFFFE780A0662311A1022285AC
:10CD700097F0FFFFE780A0632302A102228597F0CE
:10CD8000FFFFE780C062A302A102228597F0FFFFA8
:10CD9000E780E0612303A102228597F0FFFFE7808F
:10CDA0000061B245A303A102280897000000E780B4
:10CDB000208945611753FFFF6700A3348280175312
:10CDC000FFFFE702C33101112A8497F0FFFFE780DC
:10CDD000005EAA84228597F0FFFFE780605F2285CE
:10CDE00097F0FFFFE780C05E035744008D4763F76D
:10CDF000E700228597F0FFFFE780805D228597F0AE
:10CE0000FFFFE780E05C2800A68597000000E78030
:10CE1000208305611753FFFF6700A32E9797FF1F1D
:10CE2000938707009C43D847A167FD07631FF7005E
:10CE30001753FFFFE702A32A328597000000E7801F
:10CE400040F81753FFFF6700C32B82809797FF1F9F
:10CE5000938707FD9C43D847A167E5076315F7084B
:10CE60001753FFFFE702A32779713285328497F0C9
:10CE7000FFFFE780C0532AC6228597F0FFFFE780B7
:10CE80002055228597F0FFFFE78080542310A102F0
:10CE9000228597F0FFFFE780A053520551812311AF
:10CEA000A10222852302010297F0FFFFE7802050B4
:10CEB000A302A102228597F0FFFFE780404F2303E2
:10CEC000A102228597F0FFFFE780604EB245A303E1
:10CED000A102280897F0FFFFE7808076456117538D
:10CEE000FFFF6700032282809797FF1F938747F316
:10CEF0009C43D847A1679387E703631FF700175345
:10CF0000FFFFE702C31D328597000000E78060EB5A
:10CF10001753FFFF6700E31E82809797FF1F9387D9
:10CF200027F09C43D847A16793874704631EF70205
:10CF30001753FFFFE702A31A79713285328497F005
:10CF4000FFFFE780C0462AC6228597F0FFFFE780F3
:10CF50002048B245280897F0FFFFE780606E4561E2
:10CF60001753FFFF6700E31982809797FF1F93878E
:10CF700027EB9C43D847A167938787026310F70488
:10CF80001753FFFFE702A31579713285328497F0BA
:10CF9000FFFFE780C0412AC6228597F0FFFFE780A8
:10CFA0000041B2452300A102280897F0FFFFE78067
:10CFB000206945611753FFFF6700A3148280175350
:10CFC000FFFFE702C311011197F0FFFFE780203E4A
:10CFD000AA85280097F0FFFFE78080660561175358
:10CFE000FFFF670003129797FF1F938767E39C4338
:10CFF000D847A167D107631FF7001753FFFFE70268
:10D00000030E328597000000E780A0FB1753FFFF57
:10D010006700230F82809797FF1F938767E09C43E9
:10D02000D847A167C507631FF7001753FFFFE70243
:10D03000030B328597000000E780A0F81753FFFF2D
:10D040006700230C82809797FF1F938767DD9C43BF
:10D05000D847A167B907631FF7001753FFFFE7021F
:10D060000308328597000000E780A0F51753FFFF03
:10D070006700230982809797FF1F938767DA9C4395
:10D08000D847A167AD07631FF7001753FFFFE702FB
:10D090000305328597000000E780A0F21753FFFFD9
:10D0A0006700230682809797FF1F938767D79C436B
:10D0B000D84789476318F7021753FFFFE702230297
:10D0C0000111328532C897F0FFFFE780402EAA8514
:10D0D000280097F0FFFFE780A05605611753FFFF78
:10D0E0006700230282809797FF1F938767D39C4333
:10D0F000D847A1678D076311F7041753FFFFE702B5
:10D1000003FE01113285328497F0FFFFE780202A69
:10D1100013066100AA844C00228597300000E78046
:10D1200000232800A68597F0FFFFE7806051056186
:10D130001753FFFF6700E3FC82809797FF1F9387D9
:10D1400067CE9C4381CFDC4391CB1753FFFFE702AF
:10D1500003F982971753FFFF6700A3FA82801753E2
:10D16000FFFFE702C3F779713C08AE843ED2A165A8
:10D17000B7070A002A843ED448103C08DD053ED695
:10D1800036C432C63AC297D0FFFFE780402C124720
:10D190004810BA8597F0FFFFE780C0133246481069
:10D1A000B28597F0FFFFE780E014A2464810B685ED
:10D1B00097F0FFFFE7800012501001478146A685D7
:10D1C000228597D0FFFFE780E04D45611753FFFFB1
:10D1D000670023F31753FFFFE70263F001117C00A0
:10D1E0000329C501AE843ECAA165B70707002A849A
:10D1F0003ECC48087C00C5053ECE97D0FFFFE780B7
:10D2000000258345D900480897F0FFFFE780800C90
:10D21000500801478146A685228597D0FFFFE78009
:10D22000604805611753FFFF6700A3ED1753FFFF29
:10D23000E702E3EA83C7950093F7F707A384F500B5
:10D2400097000000E78040F91753FFFF670063EB8A
:10D250001753FFFFE702A3E879713C08AE843ED282
:10D26000A165B70709002A843ED448103C0893857D
:10D2700045043ED632C636C497D0FFFFE780201D56
:10D28000A2464810B68597F0FFFFE780A00432461B
:10D290004810B28597F0FFFFE780C00550100147A6
:10D2A0008146A685228597D0FFFFE780A03F456194
:10D2B0001753FFFF6700E3E41753FFFFE70223E282
:10D2C00083C7950041112A8493F7F707A384F500DB
:10D2D00032852EC697F0FFFFE780800F85672AC44E
:10D2E0006370F50297700000E78060E82246B2455F
:10D2F00009ED11478146228597000000E78060E62E
:10D3000041011753FFFF6700C3DF01478346F50163
:10D31000DDB71753FFFFE702E3DA01113C003ECA15
:10D32000B7070A003ECC3C003ECE83C79500AA89D1
:10D33000328593F7F707A384F5002E8497F0FFFF5B
:10D34000E78000098567637DF504A165AA8493855C
:10D350008504480897D0FFFFE780600F2685977007
:10D360000000E780C0E02A8929E19145480897F04C
:10D37000FFFFE78020F6A685480897F0FFFFE780CB
:10D3800060F7CA85480897F0FFFFE780A0F40147DF
:10D3900081465008A2854E8597D0FFFFE7808030F8
:10D3A00005611753FFFF670023D58145480897F0B3
:10D3B000FFFFE78020F20349090275BF1753FFFF03
:10D3C000E70243D079711C103ECAB7070F003ECC6C
:10D3D000404D1C10AA84AE894808994532C636894A
:10D3E0003ECE97D0FFFFE780800632464808B285E0
:10D3F00097F0FFFFE78000EE630C0902A54548089F
:10D4000097F0FFFFE780C0E62546CA859720010018
:10D41000E78060A3500801478146CE85268597D0D6
:10D42000FFFFE780202845611753FFFF6700C3CC4B
:10D430008355C402480897F0FFFFE780A0EB03552F
:10D44000E402814505C5854785456301F502C1674D
:10D45000FD179305F00F630BF5007D159770000025
:10D46000E780608D9305150093F5F50F480897F058
:10D47000FFFFE78020E683450403480897F0FFFF9D
:10D48000E78040E583451403480897F0FFFFE780F5
:10D4900060E483552403480897F0FFFFE78080E5A8
:10D4A00083554403480897F0FFFFE780A0E49DB749
:10D4B0001753FFFFE702A3C283C7950081460146C9
:10D4C00093F7F707A384F50097000000E78040EF8B
:10D4D0001753FFFF6700E3C21753FFFFE70223C0A4
:10D4E00079713E841C103ECA2E89B7070F00A165D2
:10D4F0003ECCFD051C10AA84480842C03AC23ECE6C
:10D5000036C432C697D0FFFFE78060F43246480841
:10D51000B28597F0FFFFE780E0DBA2464808B685BA
:10D5200097F0FFFFE78000DD12474808BA8597F0C3
:10D53000FFFFE78020DC0248630C080291454808A1
:10D5400097F0FFFFE780C0D21146A2859720010027
:10D55000E780608F500801478146CA85268597D0AD
:10D56000FFFFE780201445611753FFFF670063B991
:10D570008945480897F0FFFFE78080CF8347040084
:10D580002300F50083471400A300F500E1B717530B
:10D59000FFFFE70223B383C7950001112A8A93F79F
:10D5A000F707A384F5003285AE8432C697F0FFFFFB
:10D5B000E78000E232462A89328597F0FFFFE78054
:10D5C00000DF85676373F902AA894A8597700000B6
:10D5D000E780E0B92A8419ED114781464A86A6857D
:10D5E000528597000000E780C0B705611753FFFF21
:10D5F000670083B09387E9FF93F7F70F0547E3666A
:10D60000F7FE8347F50195EB8947E380F9FE8346F2
:10D61000F401528501474A86A68597000000E780FD
:10D6200040B4A167D90748083ECC230A010002CEC6
:10D6300097000000E780A0B04DBF639EE7008947D8
:10D64000639EF90093071020231FF50097700000D8
:10D65000E78000B76DBF0947E39BE7FA8D47E39882
:10D66000F9FA228597700000E780C0DE9797FF1FC8
:10D670009387479A9C4399E79797FF1F9387478320
:10D680009C4399C703D5040097800000E780E0CD54
:10D69000231F040022855DBF1753FFFFE70223A469
:10D6A00001113C003ECAB7070B003ECC3C003ECE09
:10D6B00083C795002A89328593F7F707A384F5007D
:10D6C000AE8497F0FFFFE780A0D093170501C187D4
:10D6D000635AF006A1652A849385E502480897D02D
:10D6E000FFFFE780C0D6A285480897F0FFFFE780DC
:10D6F00060C09787FF1F9387A77B9C43A9EB0144DA
:10D700009375F40F480897F0FFFFE780A0BC93558E
:10D71000844093F5F50F480897F0FFFFE78080BB42
:10D720009355044193F5F50F480897F0FFFFE78004
:10D7300060BA014781465008A6854A8597D0FFFF09
:10D74000E78040F605611753FFFF6700839B416543
:10D7500085460546A2857D1597500000E780A0BC50
:10D7600059DD510597000100E780C08E1304400683
:10D770003344850271B71753FFFFE7024396011147
:10D78000B70706003EC683C7950021642A8993F730
:10D79000F707A384F500AE8428009305A4040AC407
:10D7A0000AC897D0FFFFE78080CA30000147814652
:10D7B000A6854A8597D0FFFFE780C0EE97E0FFFF80
:10D7C000E780E01113049404480822CC230A0100E6
:10D7D00002CE97000000E780809605611753FFFF97
:10D7E000670023921753FFFFE702C38DC1642A89A4
:10D7F00001449799FF1F93896983130A8002FD14DE
:10D8000097E0FFFFE780E0BD6347A40001451753A1
:10D81000FFFF6700638EB307440303A7C90ABA97E3
:10D8200003D707006306970083D727006384270187
:10D830000504F9B70545E1BF1753FFFFE7028388E9
:10D840002A8A2E8999C123A0050081498144978A9B
:10D85000FF1F938A6A5D614B97E0FFFFE780A0BEE0
:10D8600063C7A4004E851753FFFF6700E388338426
:10D87000640383A70A003E948357040099E7630476
:10D880000900232089008504C1BF4146D2851305C4
:10D89000440097100100E780A05875F5A289E5B70C
:10D8A0001753FFFFE702038239717C083ED4B707A4
:10D8B0000A003ED67C083ED883C795002A8A328566
:10D8C00093F7F707A384F5002E8932C697F0FFFF80
:10D8D000E78000B085676373F5083246AA84328515
:10D8E00097F0FFFFE780A0AC8547AA8963E8A70609
:10D8F000A16593858504281097D0FFFFE78020B5A8
:10D90000268597700000E78080862A8429ED91455E
:10D91000281097F0FFFFE780E09BA685281097F07E
:10D92000FFFFE780209DCE85281097F0FFFFE7805E
:10D93000609A014781463010CA85528597D0FFFF13
:10D94000E78040D6A1679387770448183EDC230A16
:10D95000010202DE97F0FFFFE780607E216117433E
:10D96000FFFF670063798145281097F0FFFFE7808C
:10D970006096A685281097F0FFFFE780A0979797FD
:10D98000FF1F938767A19C4381CB22856389090090
:10D9900097D00000E78080238345040271B797D0B9
:10D9A0000000E7800022CDBF1743FFFFE70283712D
:10D9B00083C795004111AA8993F7F707A384F5005F
:10D9C0003285AE84328A97F0FFFFE78060A08567DA
:10D9D000637FF5022A8997600000E78040792A84F6
:10D9E000914631C58347F50105476387E70291C733
:10D9F0000D476366F704AD461DA89305050303258F
:10DA00000A00414697100100E78080410DE941017D
:10DA10001743FFFF6700436E9305950803250A002F
:10DA2000414697100100E780A03F814669F54A868C
:10DA3000A6854E8597000000E780C081C9BF832579
:10DA40000A001305940897700000E780E02819C1C8
:10DA5000C146F1BF9787FF1F9387C75B9C4399E738
:10DA60009787FF1F9387C7449C4399C72285978058
:10DA70000000E780608969FD8547A30FF4002285D7
:10DA800097B00000E780A083228597600000E780C0
:10DA900020734E8581464A86A68597F0FFFFE78072
:10DAA000607BA1679387570448003EC423020100AE
:10DAB00002C697F0FFFFE780806891BF1743FFFF22
:10DAC000E702635F83C795004111AA8993F7F707BF
:10DAD000A384F50032852E89B28A97F0FFFFE78094
:10DAE000208F85676374F50EAA8497600000E78035
:10DAF00000682A840DED416B014A978BFF1F938BC1
:10DB0000EB52130C400E7D1B19A833048A0383A724
:10DB10000B0B3E948357C40163836705050A97E0A6
:10DB2000FFFFE780008BE342AAFE95460DA08357D6
:10DB3000C501639697029305050303A50A004146B4
:10DB400097100100E780C02D994611E18146268695
:10DB5000CA854E8597F0FFFFE780C06F85A883A533
:10DB60000A001305040397700000E780E016C14621
:10DB700079FD2285231E940097A00000E780207481
:10DB8000228597600000E780A0639797FF1F938727
:10DB9000A7809C43A9C323000402228597D00000DC
:10DBA000E78080EF4E8581462686CA8597F0FFFF85
:10DBB000E780406AA1679387070448003EC42302B8
:10DBC000010002C697F0FFFFE7806057410117434D
:10DBD000FFFF6700C35189472300F402E1B73971A1
:10DBE00006DE22DC4AD8800052D456D25AD026DA39
:10DBF0004ED65ECE2E8A32892A8B97D0FFFFE780E1
:10DC0000407A0605710541998A8A3301A140232291
:10DC100024FC231404FC97D0FFFFE780807883471F
:10DC20009A000605350593F7F7072315A4FCA3040E
:10DC3000FA004A85232624FC97E0FFFFE78040791D
:10DC400093170501C1876340F0025681130104FC5C
:10DC5000F2506254D2544259B259225A925A025B3B
:10DC6000F24B21618280AA844A8597E0FFFFE7801A
:10DC70002076AA894A8597E0FFFFE7806075A16555
:10DC80009385C5022A89130544FC97C0FFFFE780EE
:10DC9000007C268597C0FFFFE7804070854511C94D
:10DCA0004A86CE8597C0FFFFE780C069AA8B21E92D
:10DCB0008945130544FC97E0FFFFE780A061A68536
:10DCC000130544FC97E0FFFFE780C062CE85130593
:10DCD00044FC97E0FFFFE780E061CA85130544FC40
:10DCE00097E0FFFFE780006101478146130644FC8F
:10DCF000D2855A8597D0FFFFE780C09AB9B7814592
:10DD0000130544FC97E0FFFFE780C05CA685130580
:10DD100044FC97E0FFFFE780E05DCE85130544FCFF
:10DD200097E0FFFFE780005DCA85130544FC97E09C
:10DD3000FFFFE780205C814497D0FFFFE7806066AB
:10DD4000E3D4A4FA83A70B0113971400BA9783D5E1
:10DD5000070099C5130544FC97E0FFFFE780805951
:10DD60008504D9BF797106D622D44AD000184ECE88
:10DD700052CC56CA26D25AC8AE893289AA8A97D0BE
:10DD8000FFFFE78000620605690541990A8A3301B1
:10DD9000A140232A24FC231C04FC97D0FFFFE7802A
:10DDA000406083C7990006052D0593F7F707231DEB
:10DDB000A4FCA384F9004A85232E24FC97E0FFFFEE
:10DDC000E780006193170501C187634FF00052811E
:10DDD000130104FDB250225492540259F249624A8E
:10DDE000D24A424B45618280AA844A8597E0FFFF70
:10DDF000E780005EA1659385A5022A89130544FD8D
:10DE000097C0FFFFE780A064268597C0FFFFE780EB
:10DE1000E058854509C9CA8597C0FFFFE78080554E
:10DE20002A8B29E18945130544FD97E0FFFFE78030
:10DE3000604AA685130544FD97E0FFFFE780804B0D
:10DE4000CA85130544FD97E0FFFFE780A04A01471C
:10DE50008146130644FDCE85568597D0FFFFE780A7
:10DE60006084B5B78145130544FD97E0FFFFE78067
:10DE70006046A685130544FD97E0FFFFE7808047D5
:10DE8000CA85130544FD97E0FFFFE780A046814463
:10DE900097D0FFFFE780E050E3DBA4FA83270B0174
:10DEA00013971400BA9783D5070099C5130544FD4D
:10DEB00097E0FFFFE78000448504D9BF1743FFFFC9
:10DEC000E702E32183474500404DD5EFFD575DC490
:10DED0008346940009476363D70A0346B400854626
:10DEE00063EEC6088306E40063CA06085C45F9567B
:10DEF0002390D7009787FF1F83C747F399E3A304B5
:10DF0000E4009787FF1F9387A7FA9C4381E789471F
:10DF1000A306F4009787FF1F938707489C4381E778
:10DF200089472306F4009705000093854506AA84D7
:10DF30001305040197F00000E780600FFD57231AD6
:10DF4000F40281471CDC01489787FF1F23AC87EC54
:10DF50009787FF1F938747ED232E040304C0804358
:10DF600097D0FFFFE780204E61463306C50281450A
:10DF700022859740FFFFE780801981473E85174340
:10DF8000FFFF67000318FD57D5BF1743FFFFE702E8
:10DF900003152A840355450297600000E780201D81
:10DFA00019E5231E04001743FFFF670083158357FD
:10DFB000E401F5DB930504FF174501001305C5E3F4
:10DFC00097E00000E7802014F9BF1743FFFFE70246
:10DFD00003112E89A16541119385E5032A8436C476
:10DFE00032C6BE843AC297C0FFFFE7804046124760
:10DFF0002285BA8597E0FFFFE780C02D3246228553
:10E00000B28597E0FFFFE780E02EA2462285B68525
:10E0100097E0FFFFE780002E630309029145228508
:10E0200097E0FFFFE780C0241146A6859710010006
:10E03000E78060E141011743FFFF6700830C8945DA
:10E04000228597E0FFFFE780A02283C7040023001A
:10E05000F50083C71400A300F500E9BF1743FFFFD5
:10E06000E702E30783C79500444D054793F7F70799
:10E07000A384F5001C42411183C707006367F706BC
:10E080002E842A89B1C003C7D400630FF702178713
:10E09000FF1F1307E7E1184305C3A386F40097A009
:10E0A0000000E780804983C7D40099E741657D156A
:10E0B00097400000E780802F83D72403918B89C786
:10E0C00097E00000E78000134A85A28597F0FFFFE4
:10E0D000E7808010A167C10748003EC42302010009
:10E0E00002C697F0FFFFE780800541011743FFFF5D
:10E0F000670023011743FFFFE70263FE03D74500D4
:10E100008D47AA8441112E8432892E8563E3E7026C
:10E1100097E0FFFFE780C02BAA8523000900268532
:10E1200097C0FFFFE780002541011743FFFF67000D
:10E1300043FD97E0FFFFE780A0292AC6228597E0EC
:10E14000FFFFE780E028B24585472A862300F900D3
:10E15000268597C0FFFFE780E01EF9B7397106DE1C
:10E1600022DC26DA80004ED652D456D24AD85AD073
:10E170005ECEAE89B284AA8A97D0FFFFE780602185
:10E1800006051305250241990A8A3301A14023227D
:10E1900024FC231404FC97D0FFFFE780801F83C773
:10E1A000990006054D0593F7F7072315A4FCA384F2
:10E1B000F9002685232624FC97E0FFFFE780402115
:10E1C00093170501C1876340F0025281130104FCDB
:10E1D000F2506254D2544259B259225A925A025BB6
:10E1E000F24B21618280AA8B03AB040097C0FFFF32
:10E1F000E780C01A51E583D7440001498544F117EF
:10E2000093B71700A301F4FC834734FCA165C9C789
:10E210009385E504130544FC97C0FFFFE7802023A6
:10E22000A685130544FC97E0FFFFE780A00ADE8582
:10E23000130544FC97E0FFFFE780C00B834734FCE5
:10E24000114691E30946DA85130544FC97E0FFFF88
:10E25000E78060058144630A0900416B7D1B97D00C
:10E26000FFFFE780001363CCA40201478146130639
:10E2700044FCCE85568597C0FFFFE780A042B1B72A
:10E28000A685130634FC97000000E780E0E693348F
:10E2900015002A8986048DBF9385C504A5BF8327F1
:10E2A000C90013971400BA9783D5070063886501E6
:10E2B000130544FC97E0FFFFE780C003850445B7E2
:10E2C0001743FFFFE70223DF79711C103EC4B70735
:10E2D0000F003EC61C103EC883C79500AA8A32852F
:10E2E00093F7F707A384F500AE89328497E0FFFF28
:10E2F000E780000E93170501C187635AF0062A8A4A
:10E30000228597E0FFFFE780A00C2A895285032B26
:10E31000040097C0FFFFE780600839ED8357440091
:10E3200081440544F11793B71700A303F100834517
:10E330007100DA872287CA8652862800970000007B
:10E34000E780E0C8014781463000CE85568597C0FA
:10E35000FFFFE7802035A1679387D70348083ECCAD
:10E36000230A810026CE97F0FFFFE78040DD45615C
:10E370001743FFFF6700A3D7A2851306710097001C
:10E380000000E78060D7AA84094455D13544E300F2
:10E3900055FB4A8597F0FFFFE78000450D4441D9C2
:10E3A000014497D0FFFFE780C0FE634DA400C16B1E
:10E3B0000144FD1B97D0FFFFE780A0FD634EA40042
:10E3C0001544B5B7DC4413171400BA9783D7070078
:10E3D000638327030504F1B7D84493171400BA9751
:10E3E00003D70700631B770123902701268597A099
:10E3F0000000E780C0DA01441DBF050465BF174374
:10E40000FFFFE70223CC83C7950041112A8A93F7C7
:10E41000F707A384F50032852E89328497E0FFFF49
:10E42000E78000FB93170501C1876353F006AA89B3
:10E43000228597E0FFFFE780A0F92311A1004E8518
:10E44000832A040097C0FFFFE78040F539E5835732
:10E45000440085440144F11793B71700A300F1006D
:10E460000348110003572100D6875285CE862686A1
:10E47000CA8597F0FFFFE7806006A167F1074800B3
:10E480003EC42302910022C697F0FFFFE78020CB15
:10E4900041011743FFFF670023C6A2851306110041
:10E4A00097000000E78040C52A84894455D98357E6
:10E4B000210011678544BA97C2071167C18313070A
:10E4C000F7EFE36FF7F89787FF1F9387A7B49C4395
:10E4D00081CB85451305210097500000E7806074CB
:10E4E000835521002285814497C0FFFFE780A0E18A
:10E4F00025D923100500228597A00000E78080CC55
:10E5000085B71743FFFFE70203BB83C7950041119F
:10E510002A8B93F7F707A384F50032852E8A32847D
:10E5200097E0FFFFE780C0EA93170501C1876351B9
:10E53000F006AA8A228597E0FFFFE78060E92A8932
:10E540005685832B040097C0FFFFE78020E531E567
:10E550008357440081440544F11793B71700A30182
:10E56000F10003483100DE875A854A87D686228625
:10E57000D28597F0FFFFE78060F6A167ED074800BE
:10E580003EC42302810026C697F0FFFFE78020BB30
:10E5900041011743FFFF670083B5A28513063100D1
:10E5A00097000000E78040B5AA8409445DD99167CF
:10E5B000CA97C2071167C1831307F7EF0544E362E7
:10E5C000F7FACA8597C0FFFFE780E0D3014451F90D
:10E5D000814997D0FFFFE780C0DC63DBA900984842
:10E5E00093971900BA9703D7070005EF23902701E7
:10E5F00097D0FFFFE780E0DA1544E384A9F626858B
:10E6000097A00000E78000BC9787FF1F938787A033
:10E610009C430144B9D74A8597500000E7800058D1
:10E6200089B785097DB71743FFFFE702A3A9797171
:10E630003E847C083EC82E8AB7071400A1653ECAF6
:10E64000E5057C08AA89080836C4428932C6BA8A18
:10E65000C6843ECC97C0FFFFE78060DFCA8508080C
:10E6600097E0FFFFE78000C732460808B28597E0D1
:10E67000FFFFE78020C8A246630A09049D450808F9
:10E6800097E0FFFFE780C0BE1D4681459740FFFF32
:10E69000E780E0A763890A089145080897E0FFFF33
:10E6A000E78000BD1146A68597000100E780A079AC
:10E6B000100801478146D2854E8597C0FFFFE7804D
:10E6C00060FE45611743FFFF670003A3B685080896
:10E6D00097E0FFFFE78000C21C400808D84393552D
:10E6E000C701858912075183B205D98D97E0FFFFD5
:10E6F000E78040C01C40080883C5870097E0FFFF03
:10E70000E78040BD1C40080883C5A70097E0FFFFD5
:10E71000E78040BC1C40080883C5970097E0FFFFD6
:10E72000E78040BB85BF8945080897E0FFFFE78089
:10E7300020B483C704002300F50083C71400A3009E
:10E74000F500BDB71743FFFFE702C39783C79500E6
:10E750004111AA8993F7F707A384F5003285AE84A7
:10E76000328497E0FFFFE780A0C693170501C187B9
:10E77000635DF0042A89032A040097C0FFFFE78045
:10E78000E0C119E9835744000548F11793B7170012
:10E79000A307F100814631A81306F100A285970076
:10E7A0000000E78060951DC51C459DC783D64700C6
:10E7B00001480347F10093078500D2884A86A68561
:10E7C0004E8597000000E78040E641011743FFFFB8
:10E7D0006700839209487DBF1D486DBF1743FFFF47
:10E7E000E702438E65715C083EC4B7077B013EC6F5
:10E7F0005C083EC883C795002A8A328593F7F707DD
:10E80000A384F500AE8997E0FFFFE78040BA835705
:10E81000E100E1C78945280097C0FFFFE78020C3DA
:10E820008145280097E0FFFFE780C0AA97C0FFFF5F
:10E83000E78000C99787FF1F938707B69C4317742B
:10E84000FF1F0344A45EAA843334800099C3136479
:10E8500024009777FF1F9387A7659C4399C3136490
:10E8600044009777FF1F9387E77A9C4399C313640B
:10E87000840083D504002800014997E0FFFFE7806A
:10E8800060A783D52400280097E0FFFFE78080A6DB
:10E8900083D54400280097E0FFFFE780A0A597D02C
:10E8A000FFFFE78000AB93150501C181280097E0C9
:10E8B000FFFFE78020A4A285280097E0FFFFE78004
:10E8C00060A39C446360F902014781463000CE8515
:10E8D000528597C0FFFFE780E0DC59611743FFFFD7
:10E8E00067008381DC441314490028003E9497E0BC
:10E8F000FFFFE78060968347440003475400890781
:10E900000607BA978607E36AF5FC835524002800BA
:10E91000814A97E0FFFFE780E09D8345440028009F
:10E9200097E0FFFFE780009B83455400280097E0B5
:10E93000FFFFE780209A8347440063C9FA00814AB9
:10E940008347540063C1FA020509A5BF1C4413970D
:10E950005A002800BA9783D50700850A97E0FFFF81
:10E96000E7804099C9BF032BC40093975A00280041
:10E970003E9B83552B00850A97E0FFFFE780809739
:10E9800083550B00280097E0FFFFE780A0964DBF5E
:10E990001733FFFFE702A3745C4993E717005CC9D4
:10E9A00097A00000E78060B51733FFFF670063752D
:10E9B0001733FFFFE702A3722E84814597F0FFFF14
:10E9C000E780C0E705C583570500FD172310F50054
:10E9D00009C4835725002310F40097000000E78046
:10E9E00060FB01451733FFFF6700A37131457DD8F8
:10E9F00023100400C5BF1733FFFFE702A36C83C7D2
:10EA0000950041112A8A93F7F707A384F500328510
:10EA10002E89328497E0FFFFE780809B93170501E2
:10EA2000C1876356F006AA89C145228597E0FFFF9A
:10EA3000E780A0802A8B4E85832A040097C0FFFFC1
:10EA4000E780C09531E98357440023110100054454
:10EA5000F11793B71700A300F10081440348110098
:10EA600003572100D6875285CE862286CA8597F025
:10EA7000FFFFE780A0A6A1679387170248003EC466
:10EA80002302810026C697E0FFFFE780406B41012B
:10EA90001733FFFF6700436613061100A28597F046
:10EAA000FFFFE7806065AA8409E52311010009449E
:10EAB00075B7930521005A8597000000E78080EF25
:10EAC000835721002A84D9DB9777FF1F93878754C8
:10EAD0009C4381CB85451305210097500000E780BA
:10EAE0004014835521002685314497C0FFFFE780FD
:10EAF00080812DD523100500268597900000E780A2
:10EB0000606C0144A1BF1733FFFFE702435D411171
:10EB10002E896C00AA8402C697F0FFFFE78000D21E
:10EB20000DC10357050005072310E50097000000FD
:10EB3000E78040E681473E8541011733FFFF6700CC
:10EB4000435C3247954765DBCA85268597300000D0
:10EB5000E780800CC147E34005FE324485474146CB
:10EB60002310F40083570900A685130544002311E0
:10EB7000F40097000100E780002D228545BF173380
:10EB8000FFFFE702235483C795004111AA8A93F738
:10EB9000F707A384F5003285AE89328497E0FFFF42
:10EBA000E780008393170501C1876356F0062A8A20
:10EBB000C145228597D0FFFFE7802068AA8452854F
:10EBC000032B040097B0FFFFE780407D31E98357B6
:10EBD0004400231101008544F11793B71700A300E7
:10EBE000F10001440348110003572100DA875685DC
:10EBF000D2862686CE8597F0FFFFE780208EA1671C
:10EC00009387070248003EC42302910022C697E082
:10EC1000FFFFE780C05241011733FFFF6700C34D7C
:10EC2000A2851306110097F0FFFFE780E04C2A84CD
:10EC300009E523110100894475B726859305210054
:10EC400097000000E78060ECAA8449FD835521000D
:10EC5000228597B0FFFFE780006B49F5014997C017
:10EC6000FFFFE7800074635DA9001848931719003F
:10EC7000BA9703D707000DEF035721002390E70051
:10EC800097C0FFFFE780E071630625039777FF1FBA
:10EC9000938747389C4399C703552100975000003C
:10ECA000E780C0EF228597900000E780A0511DBF4C
:10ECB000050975B795443DB705C19307F00F630F7C
:10ECC000F500C547630CF5009307F5FF05453315BF
:10ECD000F5004205418182800145828041657D15B4
:10ECE0008280B9E91733FFFFE702633F034506035C
:10ECF000328497000000E78060FC9305803EB305F6
:10ED0000B502C205C18181CD0357E402854763F88E
:10ED1000E7001305040197E00000E7806041835796
:10ED2000E40241677D176385E700FD172317F402AE
:10ED30001733FFFF6700E33C82801733FFFFE702D2
:10ED40008337004283C79500444D0349140093F76D
:10ED5000F707A384F500834704002209116733698C
:10ED6000F900A167B347F90041112A8BAE8A63EC21
:10ED7000E70E834724001307C00EB91793F7F70F68
:10ED80006373F71003473400C14763EEE70E834710
:10ED900044001307E00793C707086371F70C834922
:10EDA000840083477400A209B3E9F900856763F71B
:10EDB000F90A034A6400834754004E85220A336AE5
:10EDC000FA0097500000E780803A61C1239624033F
:10EDD000834B3400137AFA00239A34032388740394
:10EDE0002399440393890401631C090023A60402A8
:10EDF000239804024E8597E00000E780A0353DA0EF
:10EE0000034924004A8597000000E78020EB239700
:10EE1000A402834744004E85A388F402E38D0BFCD3
:10EE2000E30B09FC97E00000E780602E979000005C
:10EE3000E780407281460146D6855A8597E0FFFFFC
:10EE4000E7800058A167938797033EC4230201001F
:10EE5000480002C697E0FFFFE780602E41011733AC
:10EE6000FFFF6700C3288544A2862686D6855A857B
:10EE700097E0FFFFE780C054A167938797033EC4E4
:10EE800023029100F1B7BD44C5B79144F1BF1733D8
:10EE9000FFFFE702232301111C08404D3EC2B707C4
:10EEA0000F003EC41C083EC62A89AE8997C0FFFFEA
:10EEB000E78000D7585C1C5C6346B70E6394E5009E
:10EEC00063E2A70E3385A740B3B7A700B305B740E9
:10EED0001306803E81469D8D97000100E780C0B6F5
:10EEE00093140501C180A1659385C503480097B0BF
:10EEF000FFFFE780C0558145480097D0FFFFE780BE
:10EF0000603D83550404480097D0FFFFE780803EB2
:10EF100083552404480097D0FFFFE780A03D81453A
:10EF200089CCC167FD179305F00F6388F40026852F
:10EF300097500000E78020E0AA85480097D0FFFFA7
:10EF4000E780403903554404814501CDC167FD1771
:10EF50009305F00F6307F50097500000E780A0DDF0
:10EF6000AA85480097D0FFFFE780C0368345640438
:10EF7000480097D0FFFFE780E035834574044800E0
:10EF800097D0FFFFE7800035500001478146CE85CE
:10EF90004A8597B0FFFFE780E07005611733FFFFF8
:10EFA00067008315814481B71733FFFFE7022313FE
:10EFB00083C7950093F7F707A384F5009700000037
:10EFC000E78020ED1733FFFF6700A3131733FFFF20
:10EFD000E702430F83C795004111404D93F7F707B0
:10EFE000A384F5002A8A3285B284AE8997D0FFFFC8
:10EFF000E780003E2A8B268597D0FFFFE780403DC3
:10F000002A89268597D0FFFFE780603A93170B0186
:10F0100063CA0702E177CA97C207C183116763E336
:10F02000E70293070910C207C1831307B00F637B80
:10F03000F70093170901C187AA8A634AF000C54700
:10F0400063FE570141011733FFFF6700E30A97B0E2
:10F05000FFFFE7802025E31725FFD5B763080B02E4
:10F0600063060902814463890A02B7077F002310FF
:10F070006405231124057CC0568597000000E780B5
:10F08000E0C39304803EB304950239A0B7077F0024
:10F09000232004047CC081440355240497E000002D
:10F0A000E780E0A2A1C497C0FFFFE78060B7269584
:10F0B00093D7F44133379500AE97BA9708DC5CDC00
:10F0C000CE85528597000000E780A0DC99E02322DE
:10F0D0000404A1679387B70348003EC423020100DC
:10F0E00002C697E0FFFFE7808005A9BF814701487E
:10F0F0001CDC232E0403E9B71733FFFFE70223FECE
:10F1000097C0FFFFE7802034E1473305F5029145C2
:10F1100097500000E78040C4E55711C59777FF1F5F
:10F1200023A4A7D081473E851733FFFF670063FD07
:10F130001733FFFFE702A3FA9777FF1F938787CE66
:10F1400080433DC0835704046390A706835724047B
:10F15000639CB7043689B28497C0FFFFE78040AC58
:10F160005C5C63C3B7046395B7001C5C63EEA702E5
:10F170008347640463F3F400A6872303F4048347FE
:10F18000740463F39700A687A303F404835744042D
:10F1900041677D176385E70085072312F4043C442B
:10F1A00081C7CA85268582971733FFFF670063F5FD
:10F1B0009777FF1F938707C79C43014599C303C5F2
:10F1C000870082801733FFFFE70263F10111B70761
:10F1D00007003EC683C79500584D0AC493F7F7074A
:10F1E0000AC8A384F5002A89AE8411CB1C4283C7C8
:10F1F00007002304F70097900000E78000342164A3
:10F2000093055402280097B0FFFFE7804024970041
:10F210000000E78020FAAA85280097D0FFFFE7804A
:10F22000600B300001478146A6854A8597B0FFFFF5
:10F23000E780404713044402480822CC230A010017
:10F2400002CE97E0FFFFE78080EF05611733FFFFF5
:10F25000670023EB1733FFFFE70263E801117C002F
:10F260003ECAB70707003ECC7C003ECE83C7950060
:10F270002E84AA8493F7F707A384F500A1659385EC
:10F280005502480897B0FFFFE780601C9700000018
:10F29000E78040F2AA85480897D0FFFFE780800307
:10F2A000500801478146A285268597B0FFFFE78079
:10F2B000603F05611733FFFF6700A3E49777FF1FE7
:10F2C000938747B69C43094599C303C5970082803D
:10F2D0009777FF1F938707B59C43094599C303C5DB
:10F2E000D70082809777FF1F9387C7B39C43014560
:10F2F00099C303C5A70082801733FFFFE70283DCB1
:10F300000111B70708003EC683C79500404D0AC4E7
:10F3100093F7F7070AC8A384F5002A89AE8429C4A5
:10F320001442854703C7060063E0E70A8347940059
:10F33000094681496380C702B307F740A304E4008C
:10F34000B339F00083C716002305F400979000003E
:10F35000E780A01E03572403058B19C763860900A5
:10F3600097D00000E78000E921649305840228001B
:10F3700097B0FFFFE780A00D97000000E78040F402
:10F38000AA85280097D0FFFFE780C0F4970000000F
:10F39000E78080F5AA85280097D0FFFFE78080F3FB
:10F3A000014781463000A6854A8597B0FFFFE78078
:10F3B000602F13047402480822CC230A010002CEF5
:10F3C00097E0FFFFE780A0D705611733FFFF6700D5
:10F3D000A3D21733FFFFE70283D001117C003ECA9E
:10F3E000B70708003ECC7C003ECE83C795002E8434
:10F3F000AA8493F7F707A384F500A1659385850296
:10F40000480897B0FFFFE780800497000000E7807E
:10F4100020EBAA85480897D0FFFFE780A0EB970074
:10F420000000E78060ECAA85480897D0FFFFE780DE
:10F4300060EA500801478146A285268597B0FFFF04
:10F44000E780402605611733FFFF670083CB97777E
:10F45000FF1F9387279D9C43014599C303C5B700B0
:10F4600082801733FFFFE70283C70111B707070048
:10F470003EC683C79500404D0AC493F7F7070AC8F4
:10F48000A384F5002A89AE8405C81C42054783C7BA
:10F4900007006368F7060347B400630FF700A3058E
:10F4A000F40097900000E78040098347B400B9CF8B
:10F4B00097D0FFFFE78000BF21649305B4002800C8
:10F4C00097B0FFFFE780A0F897000000E78060F8A2
:10F4D000AA85280097D0FFFFE780C0DF014781465B
:10F4E0003000A6854A8597B0FFFFE780A01B29045E
:10F4F000480822CC230A010002CE97E0FFFFE780F4
:10F5000000C405611733FFFF6700A3BF97D0FFFF5B
:10F51000E780E0BF55B71733FFFFE70243BC011197
:10F520007C003ECAB70707003ECC7C003ECE83C7B6
:10F5300095002E84AA8493F7F707A384F500A165AC
:10F54000AD05480897B0FFFFE78060F09700000026
:10F55000E78020F0AA85480897D0FFFFE78080D792
:10F56000500801478146A285268597B0FFFFE780B6
:10F57000601305611733FFFF6700A3B89777FF1F7C
:10F580009387478A9C43094599C303C5C700828076
:10F590001733FFFFE702A3B401117C00AE843ECA1B
:10F5A000A165B70707002A843ECCD1057C00480836
:10F5B0003ECE97B0FFFFE78080E997000000E7802C
:10F5C00020FCAA85480897D0FFFFE780A0D050080C
:10F5D00001478146A685228597B0FFFFE780800C12
:10F5E00005611733FFFF6700C3B11733FFFFE70261
:10F5F00003AF83C7950093F7F707A384F50097003F
:10F600000000E78020F91733FFFF670083AF17334F
:10F61000FFFFE70223AB83C795000329C501411112
:10F6200093F7F707A384F5001C4283C907008547B9
:10F6300063E637079777FF1F938707D69C432E848F
:10F64000AA8485CF97000000E78080F3894763068E
:10F65000F502630409028347C90063803703230668
:10F66000390197900000E78040ED83572903898B8B
:10F6700089C797D00000E780E0B72685A28597006C
:10F680000000E78020F1A167CD0748003EC42302B7
:10F69000010002C697E0FFFFE78060AA410117332F
:10F6A000FFFF670063A59767FF1F9387A7779C43BA
:10F6B0001D4599C303C5E70082801733FFFFE702AA
:10F6C00003A20111B70707003EC683C79500584D36
:10F6D0000AC493F7F7070AC8A384F5002A89AE8401
:10F6E00015C71C4283C7070093968701E18663C450
:10F6F000060685466381D7068346E7006388F600E1
:10F700002307F70097900000E78020E3216493052A
:10F71000E400280097B0FFFFE78060D39700000067
:10F72000E780A0F8AA85280097D0FFFFE78080BA7D
:10F73000014781463000A6854A8597B0FFFFE780E4
:10F7400060F63504480822CC230A010002CE97E077
:10F75000FFFFE780C09E05611733FFFF6700639AD4
:10F760001733FFFFE702A39701117C003ECAB707DA
:10F7700007003ECC7C003ECE83C795002E84AA8431
:10F7800093F7F707A384F500A165B905480897B07A
:10F79000FFFFE780C0CB97000000E78000F1AA855B
:10F7A000480897D0FFFFE780E0B250080147814644
:10F7B000A285268597B0FFFFE780C0EE056117336D
:10F7C000FFFF670003941733FFFFE702A38FAA84AC
:10F7D00001441769FF1F13092965E14997C0FFFF1D
:10F7E000E78060C66344A400014519A833053403CB
:10F7F000832709003E9583572500639797001105DD
:10F800001733FFFF6700438F0504C9BF032E850030
:10F81000630A0E121763FF1F1303C37F0323030042
:10F820006315030029436390061203234E016315F9
:10F8300003001D43639907101733FFFFE702A387F7
:10F84000C689428A3E89BA8AB684328BAE8B2A84B4
:10F85000B5E103554E0019E501431A851733FFFF43
:10F860006700E388A167A98F116763FBE700970032
:10F870000000E78080F5814597F0FFFFE780801367
:10F880000844B70700E05841F98F18455CC1B70735
:10F89000001FF98F1CC55C4991C7610597E0000006
:10F8A000E780408BE38A09FA228597900000E78081
:10F8B00060C65DB7328597C00000E78040430D43C6
:10F8C00049DD1C44116703D54700A167A98F63FB7D
:10F8D000E70097000000E78040EF814597F0FFFFC9
:10F8E000E780400D0323840093164B01D1828347A8
:10F8F000B300035663008588FD8BA305F300FD77F5
:10F900007D8E558EFD76FD16B204F18E8327430160
:10F91000C58E231273012313D3002304530123053F
:10F920002301A3044301BDDF228597B0FFFFE780D9
:10F9300040CAAA850844B5D1610597D00000E78088
:10F94000207F8DB71D431A8582801723FFFFE702B2
:10F9500063770569AA84AE89328A0144FD5A7D190C
:10F9600097C0FFFFE780E0A26347A400014517238B
:10F97000FFFF67006378D84493171400BA9703D742
:10F980000700631F37032390570163070A0026858A
:10F9900097900000E780A0809C449DC383D76700B8
:10F9A000B3F72701639E3701D28801488147014799
:10F9B000814601468145268597000000E78040E5A5
:10F9C000050479BF1723FFFFE702C36F79711C108D
:10F9D0003EC4B7070F003EC61C103EC883C7950043
:10F9E000AA8A328593F7F707A384F5002E8932841B
:10F9F00097D0FFFFE780C09D93170501C187635A29
:10FA0000F006AA89228597D0FFFFE780609C2A8AAA
:10FA10004E85032B040097B0FFFFE780209839ED57
:10FA20008357440081440544F11793B71700A3039B
:10FA3000F10083457100DA872287D2864E8628003E
:10FA400097E0FFFFE780A058014781463000CA8554
:10FA5000568597B0FFFFE780E0C4A1679387F7035F
:10FA600048083ECC230A810026CE97D0FFFFE780CE
:10FA7000006D45611723FFFF67000368A285130629
:10FA8000710097E0FFFFE7802067AA84094455D101
:10FA9000528597E0FFFFE78020D50D4459D90546F0
:10FAA000D285268597000000E78060EA2A8451B756
:10FAB0001723FFFFE702A3628355070003462700D1
:10FAC00041112A842E8532C62EC497E0FFFFE780BD
:10FAD000A0D101C93246A245228597000000E780E7
:10FAE00000E741011723FFFF6700A3611723FFFF12
:10FAF000E702635C83C795004111AA8A93F7F70771
:10FB0000A384F5003285AE89328497D0FFFFE78069
:10FB1000208C93170501C1876357F00AC1452A8AD3
:10FB2000228597C0FFFFE78040712A8D228597D0FC
:10FB3000FFFFE780E0892A89228597D0FFFFE780D1
:10FB40000087930705F893F7F70F1307E007AA8BD1
:10FB5000637BF706228597D0FFFFE78040852A8CDC
:10FB6000228597D0FFFFE7808084AA8C5285032BE3
:10FB7000040097B0FFFFE780608239E983574400B3
:10FB8000231101008144F11793B71700A300F1007E
:10FB9000054403471100835621009387840056854E
:10FBA000DA8822885286CE8597F0FFFFE780E0A7AB
:10FBB000A167E90748003EC42302810026C697D00A
:10FBC000FFFFE780C05741011723FFFF6700235263
:10FBD00013061100A28597E0FFFFE780E051AA8499
:10FBE00009E52311010009446DB7930521006A85D9
:10FBF00097F0FFFFE78060F12A8441FD83552100E3
:10FC00009356C9001316490185486688E2875E87C6
:10FC1000858A5182268597000000E78060BF2A848C
:10FC20008DBF1723FFFFE702034983C795004111EA
:10FC30002A8B93F7F707A384F5003285AE893284C7
:10FC400097C0FFFFE780C07893170501C187635213
:10FC5000F00A2A8A228597C0FFFFE7806077AA8A88
:10FC6000228597C0FFFFE780A0762A89228597C06A
:10FC7000FFFFE780C073930705F893F7F70F1307AB
:10FC8000E0072A8C6377F706228597C0FFFFE7809D
:10FC90000072AA8C228597C0FFFFE78040712A8DF1
:10FCA0005285832B040097A0FFFFE780206F39E582
:10FCB0008357440085440144F11793B71700A3010B
:10FCC000F10003473100930784005A85DE882688B7
:10FCD000D6865286CE8597F0FFFFE78000958D4748
:10FCE00048003EC42302910022C697D0FFFFE78060
:10FCF000004541011723FFFF6700633FA2851306FC
:10FD0000310097E0FFFFE780203F2A84894455D9DE
:10FD10009356C9001316490185486A88E6876287A9
:10FD2000858A5182D68597000000E78060AEAA845C
:10FD300049BF1723FFFFE702E3382A8981440144C2
:10FD4000617A916A176BFF1F130BCB2C97B0FFFFE3
:10FD5000E780206563C7A40022851723FFFF6700A3
:10FD6000A3398327090093991400CE9703D5070080
:10FD700033074501420741836364570305C10327E5
:10FD80000B0019C785453E8597400000E78060E974
:10FD9000832709000504CE972390070085047DB7CB
:10FDA00097000000E78060A2832709000504CE9732
:10FDB0002390070065D5814597F0FFFFE78080BF5E
:10FDC000F1BF1723FFFFE702E32F83C7950041111F
:10FDD0002A8A93F7F707A384F50032852E893284A7
:10FDE00097C0FFFFE780C05E93170501C187635A84
:10FDF000F004AA89832A040097A0FFFFE780005A35
:10FE000031E58357440085440144F11793B7170047
:10FE1000A301F10003483100D68752850147CE8601
:10FE20002686CA8597D0FFFFE780406BA167F5075C
:10FE300048003EC42302910022C697D0FFFFE7800E
:10FE4000003041011723FFFF6700032BA285130633
:10FE5000310097E0FFFFE780202A2A8489445DD99A
:10FE60009767FF1F9387071B9C4381CF044997B077
:10FE7000FFFFE7800053AA85268597400000E780B2
:10FE800040DA1305040197000000E780C0EA2285EC
:10FE900097800000E78000338144ADBF1723FFFF48
:10FEA000E702632183C795004111AA8A93F7F707F8
:10FEB000A384F5003285AE8932842311010097C0F6
:10FEC000FFFFE780E05093170501C1876354F006F8
:10FED0002A8AC145228597C0FFFFE7800036AA8B9A
:10FEE0005285032B040097A0FFFFE780204B21E9F8
:10FEF0008357440085440144F11793B71700A300CA
:10FF0000F1000348110003572100DA875685D28695
:10FF10002686CE8597D0FFFFE780405CA167938758
:10FF2000270248003EC42302910022C697D0FFFF5B
:10FF3000E780E02041011723FFFF6700431BA285F4
:10FF40001306110097E0FFFFE780001B2A84894415
:10FF50004DD99767FF1F9387E70B98433E8901CFE1
:10FF6000044997B0FFFFE780C043AA8526859740E4
:10FF70000000E78000CB1305040197000000E78034
:10FF800080DB97B0FFFFE780C04195443DD99305E2
:10FF900021005E8597F0FFFFE78020B7AA8435F146
:10FFA0001C480357210022852390E700978000001A
:10FFB000E780402183270900A9D7035521009740F6
:10FFC0000000E780A0BD35BF1723FFFFE702A30EA7
:10FFD00083C795004111AA8A93F7F707A384F50018
:10FFE0003285AE89328497C0FFFFE780603E931769
:10FFF0000501C1876351F0062A8A228597C0FFFF59
:020000040001F9
:10000000E780003D2A895285032B040097A0FFFF5B
:10001000E780C03831E58357440085440144F11737
:1000200093B71700A301F10003483100DA87568522
:100030004A87D2862686CE8597D0FFFFE780004A82
:10004000A167F90748003EC42302910022C697D059
:10005000FFFFE780C00E41011723FFFF6700230960
:10006000A2851306310097E0FFFFE780E0082A84AD
:1000700089445DD99167CA97C2071167C183130785
:10008000F7EF8544E362F7FA9767FF1F938787F8D6
:100090009843BE8B01CF044997B0FFFFE7806030E3
:1000A000AA85268597400000E780A0B713050401C4
:1000B00097000000E78020C897B0FFFFE780602E20
:1000C00095443DD11C482285814423902701978087
:1000D0000000E780200F83A70B00B9D74A8597401F
:1000E0000000E780A0AB89B71723FFFFE70223FFDB
:1000F0002A844105B28497000000E780C0C311C57F
:10010000228597800000E780E00B81460146A685A6
:10011000228597800000E780C04E1C4C89C7DC47D1
:1001200099C3228582971723FFFF670083FD976796
:10013000FF1F938727CF9C43014599C31385070170
:1001400082809767FF1F9387E7CD884382801723BC
:10015000FFFFE702C3F89317C600DD8DC20541110A
:10016000C1812A8432C697C0FFFFE780A0183246BB
:10017000228511829375F60F97C0FFFFE7808015E7
:1001800041011723FFFF6700C3F71723FFFFE702B3
:1001900063F379713C083ED2B7070C003ED43C08AB
:1001A0003ED683C79500AE842A8993F7F707A384C8
:1001B000F500A16593853504481097A0FFFFE780FF
:1001C0000029C165FD150144176AFF1F130A0AE6DD
:1001D000930A400EAE892E8B2EC697B0FFFFE780A4
:1001E000401F4205931704014181C183B24563E971
:1001F000A702C167FD176387F500481097C0FFFF8E
:10020000E780400F501001478146A6854A8597A098
:10021000FFFFE780204945611723FFFF6700C3ED1B
:100220003307540383270A0BBA9703D6C701630A1F
:100230003601638A3501481097000000E78060F1BD
:10024000DA85050451BFB285EDBF1723FFFFE70232
:1002500083E679717C083EC8B70711003ECA7C0866
:100260003ECC83C79500AA89328593F7F707A3840C
:10027000F5002E8997C0FFFFE780801585676378BA
:10028000F504A165AA848905080897A0FFFFE78007
:10029000001C268597400000E78060ED13341500B0
:1002A0000A04A285080897C0FFFFE780A002A68580
:1002B000080897C0FFFFE780E00325CC014781468F
:1002C0001008CA854E8597A0FFFFE780A03D4561D5
:1002D0001723FFFF6700A3E1B30754030327CA0AEC
:1002E000BA9703D70700631C970003D627006380E3
:1002F0006505080897000000E780A0E5DE85050495
:100300002EC697B0FFFFE780C00D4205931704018A
:100310004181C183B245E3E1A7FCC167FD17E38FCB
:10032000F5F8080897C0FFFFE780C0FC41BFB28521
:10033000F9B7C165FD150144176AFF1F130A0ACFFB
:10034000930A80022E8BAE8B65BF1723FFFFE70257
:1003500003D918418347170083460700A207D58FAA
:10036000D207D1832390F500834727000347170066
:100370008D45A207D98F91832310F60097C0FFFF08
:10038000E78060EA1723FFFF6700A3D71723FFFF6B
:10039000E70243D3C16401441769FF1F130909C968
:1003A00093098002FD1497B0FFFFE7808003634745
:1003B000A40001451723FFFF670003D4330534036E
:1003C0008327C90A3E9583570500E38597FE0504F8
:1003D000D9BF1723FFFFE702E3CE2A8AAE89B28492
:1003E000B68A97400000E78080D819E591473E859E
:1003F0001723FFFF670043D02A894E8597C000006E
:10040000E780E08E2A84638E0A048D476DD10357FE
:100410000500C547E31D47FD0347F9018546AD4784
:10042000E317D7FC8347450081CF4146A6855D058C
:1004300097F00000E780C09E814755D9AD4745BF82
:10044000130965012302E500CA852685971000007F
:10045000E780606231C1A547E38B0AF823020400FC
:1004600079B705C183570500E39247F94146A68550
:10047000190597F00000E780A09A81472DD9994788
:10048000BDB74E8597000000E78080F02A8495472D
:1004900039DD130955004DBF4146A685231044019F
:1004A000231134011305190097F00000E780A0998B
:1004B000228597800000E780A0EA81470DBF1723BF
:1004C000FFFFE702C3C179717C003ECCB7070A0089
:1004D0003ECE7C003ED083C79500B2842E8493F735
:1004E000F707A384F5001306A1002A892C002685AE
:1004F00097000000E780A0E5A16528088D0597A07A
:10050000FFFFE780C0F490408355A10003558100B0
:10051000854697000000E78000ECAA84AA85280899
:1005200097C0FFFFE78000DB0356A10083558100E1
:10053000280897000000E780C0C1300801478146C5
:10054000A2854A8597A0FFFFE780C0158547481020
:100550003ED42302910202D697D0FFFFE78020BE4F
:1005600045611723FFFF6700C3B91723FFFFE702A9
:1005700003B779717C003ECCB7070A003ECE7C0001
:100580003ED083C79500B2842E8493F7F707A384E7
:10059000F5001306A1002A892C002685970000008B
:1005A000E780E0DAA16528088D0597A0FFFFE780C6
:1005B00000EA90408355A1000355810081469700D1
:1005C0000000E78040E1AA84AA85280897C0FFFFC1
:1005D000E78040D00356A10083558100280897008A
:1005E0000000E78000B7300801478146A2854A85B0
:1005F00097A0FFFFE780000B48102302910202D46E
:1006000002D697D0FFFFE78080B345611723FFFF35
:10061000670023AF1723FFFFE70263AC97000000DA
:10062000E78060DB1723FFFF6700A3AD9757FF1F2D
:100630009387877F884382801723FFFFE70223AADF
:10064000835725004111AE842A842307B10017F592
:10065000FFFF130525466C002316F10097A0FFFF4E
:10066000E780404691C4228597800000E780E0D66D
:10067000FD572310F4001306200281451305540092
:100680009720FFFFE780A0A841011723FFFF670025
:1006900043A71723FFFFE702E3A279717C003ECC5A
:1006A000B7070A003ECE7C003ED083C79500AA89DA
:1006B000AE8493F7F7073285A384F5001306A100F3
:1006C0002C0097000000E78080C80355810011448A
:1006D00097400000E780A0A915C50355A10001447B
:1006E00097B00000E780A06011CD03570500835745
:1006F000810045446318F700854597000000E780B6
:10070000E0F30144216993053900280897A0FFFF11
:10071000E780E0D3A285280897C0FFFFE78080BB71
:100720000356A10083558100280897000000E78048
:1007300040A2300801478146A6854E8597A0FFFF5D
:10074000E78040F648104AD42302810202D697D0AF
:10075000FFFFE780C09E45611723FFFF6700C39935
:100760001723FFFFE70203969757FF1F9387876BB7
:100770002A8488432E8915C5035745038357C4012E
:100780006311F7022326050223180502410597D0BD
:100790000000E780209C6306090097800000E78046
:1007A00060DB81449769FF1F93894988130A80029F
:1007B00097B0FFFFE780E0C263C4A4049757FF1F10
:1007C0009387076F9C4399C70355C4019720000086
:1007D000E780C0BD63070900228597800000E7809D
:1007E000C0A01306400E814522859720FFFFE780B9
:1007F0000092FD57231EF4001723FFFF6700C38FED
:100800003385440383A7C90A3E95035705008357E0
:10081000C4016317F700CA8597000000E78000E273
:10082000850479B71723FFFFE702C38983C79500C3
:100830004111AA8993F7F707A384F5003285AE84A6
:1008400097C0FFFFE780C0B885676378F5042A8901
:1008500097400000E780A091014401CD83D70400B8
:10086000314463882701854597000000E78080EFC9
:1008700001444E85A2864A86A68597D0FFFFE78071
:10088000609DA1679387170448003EC4230281003E
:1008900002C697D0FFFFE780808A41011723FFFF40
:1008A000670083851723FFFFE702C3819757FF1F68
:1008B00093874757804329C4014597C00000E780CC
:1008C000002181470148C1641CDC232E040323203E
:1008D00004041759FF1F1309697501449309400E59
:1008E000FD1497B0FFFFE780C0AE634FA4008145C1
:1008F00017F5FFFF1305857F97A0FFFFE780801C9A
:100900001713FFFF6700437F330534038327090B69
:100910003E958357C5016387970085459700000082
:10092000E78040E4050475BF9357050113D787009E
:10093000A380F50093170501C183A1832380E500FF
:100940002381F500A381A50082801713FFFFE70232
:1009500003792300050083C71500A300F50083C7B2
:1009600025002301F50083C73500A301F50083C7E7
:1009700045002302F50083C75500A302F50083C795
:10098000650093059500A30305002303F5002304E8
:100990000500328597000000E78040F91713FFFF3C
:1009A000670023761713FFFFE702C3714111E95473
:1009B0000DCD85CD93F9C5FF2E842A89AA84338A6B
:1009C000A900B7EA040063189A020D88854411CC87
:1009D000B7E704009C5F82972AC622866C00330525
:1009E000390197E00000E780004626854101171392
:1009F000FFFF6700637083A78A03910482979317B0
:100A00000501C183A183A38EF4FE93570501238FB3
:100A1000F4FEA183238EA4FEA38FF4FE6DB763E6DC
:100A2000D5021713FFFFE702836BB28741113686A9
:100A3000BE8536C697E00000E780E040B24641013F
:100A400036851713FFFF6700C36B814636858280AA
:100A5000838705001387F5003D05FD8793F7770829
:100A6000834607007D158606B58FA300F500630752
:100A7000B7007D17834717009D83DDB7828017136A
:100A8000FFFFE702C365B7E7040083A707093287C2
:100A90002A863A858297133515001713FFFF6700E2
:100AA000436615C181478DC11713FFFFE70223631A
:100AB000414697E00000E780003985473E851713DF
:100AC000FFFF6700036481473E8582801DCD1713B9
:100AD000FFFFE702C360414681452A849710FFFF6C
:100AE000E780E06241468145130504039710FFFF4C
:100AF000E780E0610147C1672322040438C87CC84D
:100B000005451713FFFF6700C35F014582808147DA
:100B10003DCDB5CD1713FFFFE702635CB2842E898C
:100B20001306800581452A849710FFFFE780205E29
:100B3000CA8524C4268597000000E780C0F6414698
:100B4000814522859710FFFFE780605C3044A285D5
:100B5000228597000000E780C0F293040401A2857B
:100B6000268597000000E780E0EEA68513050402C5
:100B700097000000E78000EE228597000000E780E4
:100B800020F585473E851713FFFF670083573E8595
:100B900082801713FFFFE702E3524111E9540DCDA4
:100BA00085CD93F9C5FF2E842A89AA84338AA900AA
:100BB000B7EA0400639844030D88814411CCB7E779
:100BC00004009C5F82972AC622866C003305390197
:100BD00097E00000E7802027268541011713FFFFDB
:100BE0006700835183A78A039104829793170501B5
:100BF000C183A183A38EF4FE93570501238FF4FED6
:100C0000A183238EA4FEA38FF4FE6DB765CD1713C9
:100C1000FFFFE702234BB28411E605451713FFFFE0
:100C20006700834D2A842E890145EDD93C487848D8
:100C3000B3E6E700E5D69386F7FFB3B7F6007D1776
:100C4000032A4404BA9734C87CC863050A06C1491C
:100C500013050A03B38949412295637D3601B286A3
:100C60002E86A68597000000E780A0DB7C40BE941E
:100C700064C065B7CE862E86CE8597000000E780DB
:100C800040DAC114D2944E9923220404A287930619
:100C9000040103C7070003C607038507318FA38F2D
:100CA000E7FEE398F6FE3044A28522859700000017
:100CB000E78020DD2699C1493306994063EC99000D
:100CC000A9DCA686A6851305040397000000E7802B
:100CD00040D579BF8147B306F4003307F6000347D8
:100CE000070083C5060085072D8F2380E600E39467
:100CF00037FF3044A285228597000000E78060D846
:100D0000C1145DBF014582800DC11713FFFFE702CB
:100D1000033D1306800581459710FFFFE780203FC4
:100D200005451713FFFF6700C33D014582808147DA
:100D300049C5C1C51713FFFFE702633AFC414146AD
:100D40002E84AA846399C70413860501A28781466D
:100D5000C14503C7070003C507038507298F33056E
:100D6000D600034505008506298FA38FE7FEE39291
:100D7000B6FE3044A285268597000000E78060D04B
:100D8000228597000000E78060F885473E851713AD
:100D9000FFFF67000337138507031D8E81452295EA
:100DA0009710FFFFE780A0367C40130700F813067A
:100DB0000402A2972388E70251BF3E858280171361
:100DC000FFFFE702C3316D712E84B284AA859010B3
:100DD0002800368997000000E780A0D309EDD55799
:100DE00025A050400C40280097000000E78040E21A
:100DF0007DD5FD142104F5F42C004A8597000000F0
:100E0000E78020F3814761DD3E8551611713FFFFC5
:100E10006700232F1713FFFFE702632C41112EC435
:100E200032C62C00054697000000E78080F941019A
:100E30001713FFFF6700E32C1713FFFFE702232AB6
:100E400001112A842EC602C802CA02CC02CE97E043
:100E50000000E780C023B2462A86A28508089700D2
:100E60000000E78060FB1375F50F05611713FFFFA6
:100E7000670023291713FFFFE70263267971B28702
:100E80002A8421462308B10013051101BE853AC406
:100E900036C697E00000E78000FBB246930591015B
:100EA000368597000000E78060A82285141035463B
:100EB0000C0897000000E78020F62A84224701E909
:100EC00021460C103A8597E00000E780C0F72285A4
:100ED00045611713FFFF6700C3221713FFFFE702E7
:100EE00003207171AE84AA850A85328497000000C0
:100EF000E78060BB11C90A86A6852285970000009D
:100F0000E78020B8814711E1C5473E854D61171341
:100F1000FFFF6700031F1713FFFFE70243191D714F
:100F20002A8AB289BE8435468547130511012E8C65
:100F3000B68A3A8BC28C468D2308F10097E00000F8
:100F4000E78060F010100C085285231F0100970005
:100F50000000E780C0F82A843DEDA1476313FD0837
:100F60009307900591E0E5473546E28513051101A9
:100F700013990A012308F1001359090197E00000B1
:100F8000E78060EC1357890093978A00D98F900807
:100F90000C085285231FF10097000000E78020F421
:100FA0002A8415E9A1E49387FA0091831379F90063
:100FB0003EC6631309004149668B8144C14B854D90
:100FC000B247639F970C6A868C0033855C0197E07B
:100FD0000000E78040E7228525611713FFFF6700C7
:100FE000C31093079004C9F0A547BDBF834701050F
:100FF0000947C14B2308F10083471105A58FA308BA
:10100000F10093872400814463E1FB040147140845
:101010003386E6008C08B386E400BA95DA9683C678
:10102000060083C505000507AD8E2300D600E390BA
:10103000E7FE4147639CE70490080C08528597003F
:101040000000E780C0E925D181A0B3069B00BA87E4
:101050001008B305F60090083E9603C50600034647
:10106000060085078506298E2380C500E39277FF59
:10107000998F90080C085285BE9497000000E78075
:1010800000E68947014749D12A84B1B790083E96C6
:10109000034606001408BE962380C600850759BF84
:1010A000B24785046387971481471808B306F70091
:1010B00098083E973386F900034707000346060069
:1010C0008507318F2380E600E39177FF90080C08B5
:1010D000528597000000E78080E05DF53546E285A7
:1010E000130511012308B10197E00000E780A0D5A6
:1010F000139704014183939784002183D98F10189B
:101100000C085285231FF10097000000E78020DDC6
:1011100025FD814710183387F9003E9603470700E5
:1011200003460600B306FB008507318F2380E600E7
:10113000E39277FF65A81808B306F70098083E9772
:101140003386F90003470700034606008507318F01
:101150002380E600E3E127FFCA87639E77099008B2
:101160000C08528597000000E78060D711FD814789
:101170009800B306F700900818103E973E96034774
:101180000700034606008507318F2380E600E391C0
:1011900077FF3546E285130511012308B10197E079
:1011A0000000E78040CA13970401418393978400AD
:1011B0002183D98F10180C085285231FF100970046
:1011C0000000E780C0D1E31105EC81471018338798
:1011D000F9003E960347070003460600B306FB00EE
:1011E0008507318F2380E600E3E227FFC109410B29
:1011F000C1BB814785B79408BE9683C60600180810
:101200003E972300D700850789BF638006321713F6
:10121000FFFFE702C3E959712A84BE89B28B854773
:101220003546130511022E8B468C4289BA8A368ABE
:101230002300F10297E00000E780E0C010180C10D6
:1012400022852317010297000000E78040C9631838
:101250000512A147631FFC069307900563930900DD
:10126000E5473546DA851305110293140A01230078
:10127000F102C18097E00000E780E0BC93178A008C
:1012800013D78400D98F90080C1022852317F10200
:1012900097000000E780A0C47DE1639209049307F2
:1012A000FA00BD88918391E0C144C207C183DE8CFE
:1012B000814A3EC6414DB24763E2FA0E6286B3856B
:1012C0004B01881097E00000E78080B54DC93D557F
:1012D0007DA093079004E39609F8A54759B7834783
:1012E00001050947C14C2300F10283471105B3C72B
:1012F000F900A300F10293872900814963E1FC040E
:10130000814618103306D7008C083387D900B6956C
:1013100056970347070083C5050085062D8F2300D8
:10132000E600E390D7FE41476390E70690080C1073
:10133000228597000000E78080BA35D189A0B38666
:101340003A01BA871010B305F60090083E9603C51F
:1013500006000346060085078506298E2380C50002
:10136000E39297FF3387EC4090080C102285BA99DE
:1013700097000000E780A0B68947014741D1656129
:101380001713FFFF670063D690083E9603460600DA
:101390001410BE962380C600850779B7B247850A28
:1013A00093990A01939D8A0093D909016391570F7C
:1013B00085473546DA85130511022300F10293D9DA
:1013C000890097E00000E78000A8B3ED3D019000A0
:1013D0000C1022852317B10397000000E78020B08E
:1013E00059FD8147A68963EA970626860C084A8537
:1013F00097E00000E78020A581471810B306F700AA
:10140000100898083E973E960347070003460600DB
:101410008507318F2380E600E3E197FE639FA905EE
:1014200090080C10228597000000E78040AB21F95E
:1014300081479810B306F700900818183E973E961B
:1014400003470700034606008507318F2380E60027
:10145000E391A7FF4109C10CB9BD18089000B3067C
:10146000F7003E963387FC0003470700034606005B
:101470008507318F2380E600B5B798084E9703475C
:1014800007001C10CE972380E700850941BF8547E0
:101490003546DA85130511022300F10293D989003C
:1014A00097E00000E780209AB3ED3D0190000C101A
:1014B00022852317B10397000000E78040A2E310C4
:1014C00005EC814718089000B306F7003E96338775
:1014D000FC0003470700034606008507318F238081
:1014E000E600E391A7FF41460C084A8597E000001B
:1014F000E780609581471810B306F7001008980838
:101500003E973E9603470700034606008507318F46
:101510002380E600E391A7FF90080C102285970036
:101520000000E780C09B1DD599BD7D5582801713B3
:10153000FFFFE702C3BA01112A842E8593055100EB
:10154000328902C002C202C402C69304740097F03A
:10155000FFFFE780A03D1D46A6851305910097E09B
:101560000000E780408E10088A854A8597000000B9
:10157000E780E09619ED93071400180883C607006A
:101580000346070085070507B18EA38FD7FEE397B3
:10159000F4FE05611713FFFF6700A3B61713FFFFE3
:1015A000E70243B22E848C414111AA89838715003A
:1015B0003289914463D30700A1449757FF1F938753
:1015C000A7DD9C43A1C7C1CA8D472310F10083C783
:1015D00025004A852301F10083C73500A301F100EE
:1015E00083C745002302F10083C75500A302F10021
:1015F00083C7650093059100A30301002303F10055
:101600002304010097F0FFFFE78040320C404A8638
:101610000A8597F0FFFFE780803303280400835694
:101620004400A6881D0881470147E51642868A8541
:101630004E8597000000E780408E2A8919E5A6852F
:10164000228597B0FFFFE780A0C24A8541011713AA
:10165000FFFF670063AA4A860A8597F0FFFFE780CD
:10166000002F6DB71713FFFFE702C3A52E848C412F
:101670004111AA89838715003289914463D30700F9
:10168000A1449757FF1F938727D19C43A1C7C1C689
:101690008D472310F10083C725004A852301F100FF
:1016A00083C73500A301F10083C745002302F10081
:1016B00083C75500A302F10083C76500930591001D
:1016C000A30301002303F1002304010097F0FFFFAF
:1016D000E780C0250C404A860A8597F0FFFFE78027
:1016E000002783564400032804008A85858EC2069D
:1016F0001D08C1822312D400A68881470147E51640
:1017000042864E8597000000E78060B041011713C4
:10171000FFFF6700639E4A860A8597F0FFFFE78018
:1017200000234DBF1713FFFFE702639BB335B000E3
:10173000011185052A891315F60133651501230862
:10174000B1009305110136843AC632C03EC442C28C
:1017500097F0FFFFE780801DA2471248425593D6BD
:101760008700230BF1009305910193578800A30A8A
:10177000D100A30BF100230C010197F0FFFFE780DC
:10178000E01A3247024603280400B337E0008356CC
:1017900044009207914411C2A1444A85A68842861A
:1017A0000C0897F0FFFFE78040772A8919E5A685A6
:1017B000228597B0FFFFE780A0AB4A85056117132C
:1017C000FFFF670003941713FFFFE702A38F0111C8
:1017D0003EC68647B335B0008505AA891315F601C4
:1017E0005D8D2308B1009305110136843A89B284D6
:1017F00042C446C297F0FFFFE78040132248924858
:10180000164593578800A30AF1009305910193D7D9
:101810008800230B0101A30BF100230C110197F0A9
:10182000FFFFE780A0103247104083564400B337D3
:10183000E000920703280900914891C0A1480C08D4
:101840004E8597000000E780809CAA8401E98355BB
:1018500044004A8597B0FFFFE78080A12685056197
:101860001713FFFF67004389AA959307F00F170727
:1018700001001307E75B6317B50013C5F7FF137586
:10188000F50F828005058346F5FFB58FBA9783C7AC
:101890000700D5B70357450014419307F00F17060B
:1018A00001001306E6583697420741831395060157
:1018B0004181631BE500AD8FB29703C50700130597
:1018C00015F3133515008280850603C5F6FFA98F31
:1018D000B29783C70700D9BF1713FFFFE702238022
:1018E000B28736842E86BA86AA853E85BA8497F05A
:1018F000FFFFE7806052634F0500228597D000000C
:10190000E780E0782A86A686A285268597F0FFFFE5
:10191000E78080501703FFFF6700A37E1703FFFFD8
:10192000E702437A5D712A8BAE8A17050100130521
:10193000A54D2C00B284368ABA893E8997F0FFFF04
:10194000E780C04F2A845DE134104146DA852800E3
:1019500097F0FFFFE780404C2A8449E98547A303BD
:10196000F100A6C2930771002408BEC4A68685476D
:101970000D462C18281002DC02DED6C0BEC697F039
:10198000FFFFE78000442A8435E183477102A68681
:101990000D4693F7F7072300FA00C1473EDE2C18E7
:1019A0008947281026DCA303F10097F0FFFFE780AA
:1019B00040412A8405ED4146A6854E8597D000001A
:1019C000E78060488D47A6860D462C182810A30393
:1019D000F10097F0FFFFE780C03E2A8401E941460D
:1019E000A6854A8597D00000E780E04522856161A1
:1019F0001703FFFF670043701703FFFFE702236E23
:101A000097F70000938787A1984383C747007971B0
:101A10002A89AE84170501001305853F0C083AC4D6
:101A20002306F10097F0FFFFE78040412A8405ED8F
:101A300014104146CA85080897F0FFFFE780C03DB3
:101A40002A8415E1140815462C00081097F0FFFFB2
:101A5000E780803C2A8401E921462C08268597D01E
:101A60000000E780403E228545611703FFFF6700C5
:101A700043691703FFFFE702836697F70000938728
:101A8000E7999C477971AA842E84170501001305F4
:101A9000A5380C083EC697F0FFFFE780203A0DE915
:101AA00014104146A685080897F0FFFFE780C0366E
:101AB00005E1140811466C00081097F0FFFFE7805D
:101AC000A03519E58347F10193F7F7032300F400EC
:101AD00045611703FFFF6700C3621703FFFFE702BB
:101AE00003603688A14881470147E54697F0FFFF2C
:101AF000E780A0421703FFFF6700A3601703FFFF03
:101B0000E702E35D3688A14881470147E54697F043
:101B1000FFFFE780C06F1703FFFF6700835E1703B7
:101B2000FFFFE702C35B01112A842E850C0832C631
:101B300097F0FFFFE780803009ED324797060100FC
:101B40009386062C1008C145228597000000E78087
:101B5000E0D805611703FFFF6700A35A1703FFFFD3
:101B6000E702E3574111C1472EC032C48A850946B6
:101B70003EC23EC697F0FFFFE780A0244101170355
:101B8000FFFF670003581703FFFFE70243554111AA
:101B9000AE8613061009AA850A8502C002C202C4D5
:101BA00002C697F0FFFFE780202741011703FFFFE0
:101BB000670023551703FFFFE7026352328797063A
:101BC00001009386E6252E8693050002970000000B
:101BD000E780C0D01703FFFF6700A3521703FFFF82
:101BE000E702E34F7971C1472ACC2ED032D42C08BA
:101BF0000D4628003ECE3ED23ED602C402C602C8E2
:101C000002CA97F0FFFFE780C01B45611703FFFF83
:101C10006700234F1703FFFFE702634C0111AA84FB
:101C20002E8417050100130525208A8597F0FFFFF4
:101C3000E780C02015E514084146A6850A8597F07F
:101C4000FFFFE780601D09ED8347E1010347F101D4
:101C5000A207D98FCA07C9836177D98F2310F400EF
:101C600005611703FFFF6700C34915CD1703FFFF89
:101C7000E702E3469747FF1F9387871F90439745E7
:101C8000FF1F9385251F1745FF1F1305651A97D062
:101C90000000E78000C51745FF1F130565191703EE
:101CA000FFFF670003461745FF1F13056518828075
:101CB0008DCD1703FFFFE70283429747FF1F9387EE
:101CC000271B944301112E840A869745FF1F938595
:101CD000651A97D00000E78040C60A850294014546
:101CE00005611703FFFF6700C3417D55828017031D
:101CF000FFFFE702C33E97D00000E78080D19747FF
:101D0000FF1F23A7A71617F5FFFF1305E5C997B017
:101D10000000E780C0741703FFFF6700833E17478A
:101D2000FF1F130727179317150008433E95FD570C
:101D30002310F50082801703FFFFE702433A2A844D
:101D4000084009E51703FFFF6700A33B1C4158400B
:101D50001CC06313E5005CC08347550023200500C9
:101D6000F99BA302F50097A0FFFFE780E07CC9BFC5
:101D70001703FFFFE70203359747FF1F938787137A
:101D800098432A8411CB8347350093F7070289C70C
:101D900003550500894502971305440197B00000DB
:101DA000E780403B835504000355E4009730000072
:101DB000E780A00C485819C597A0FFFFE780C077BF
:101DC000232A04021305840397000000E780E0F64D
:101DD0008144B1499790FFFFE780E06A63CBA4029A
:101DE000834734002320040493F727FCA301F40065
:101DF00000489790FFFFE780006A131615008145A1
:101E000022859700FFFFE78080301703FFFF670000
:101E1000A32EB38734030329040385043E994A851E
:101E200097000000E78060F12304090065B783474D
:101E3000350093F7070299E3014582808357E50057
:101E4000E39CB7FEC167FD176316F6000545828067
:101E5000054599A81703FFFFE702632893170601BA
:101E6000C187B2842A8401496359F002835705006F
:101E70009DCB01456367F600034584003E953325FD
:101E8000A6001375F50F0DA01C4813171900BA977B
:101E900083D70700E38E97FA05099790FFFFE78045
:101EA000805FE343A9FE01451703FFFF6700632539
:101EB0001703FFFFE7020321AE89AA849790FFFF73
:101EC000E78020532A8497D0FFFFE780A02EAA86C0
:101ED00001471306840197050000938585E41745A3
:101EE000FF1F130565FB9790FFFFE780A0192A8964
:101EF00025C98C441304C50022859E0593F5050869
:101F000097A0FFFFE780003DCC4083877400E1810C
:101F100063DD070493E50508228597A0FFFFE780AE
:101F2000603B0D4693854400228597A0FFFFE78024
:101F3000803783D50400228597A0FFFFE780A03E6D
:101F400083D52400228597A0FFFFE780C03D03D6FC
:101F5000490083A50900228597A0FFFFE780A034F0
:101F60004A851703FFFF6700231993F5F5076DB73F
:101F70001703FFFFE702A31601112A84328532C638
:101F800097A0FFFFE780A0289780FFFFE7808031C0
:101F9000835704001747FF1F130747093246231BC7
:101FA000F100930700F8A30DF1001C471843231A12
:101FB000A1008983858BB307F740B28548083ECEE0
:101FC000231C0100230D010097000000E78080EE34
:101FD00005611703FFFF6700C3121703FFFFE70246
:101FE000630E004101453DC49304C4002685328937
:101FF000AE8997A0FFFFE780802595452A8A268530
:10200000035B040197A0FFFFE780E021268597A0EE
:10201000FFFFE780203F8D45AA8A268597A0FFFF16
:10202000E7806020268597A0FFFFE780A03D5C4801
:10203000420A135A0A01D2975CC4231864018147EB
:1020400063983A0146054D813306254193371600C2
:1020500013F5F70F1703FFFF6700030A1703FFFFCE
:10206000E702630589692A8BAE8B328AB68A81447E
:102070000144314CFD199790FFFFE780C04063CDCC
:10208000A4009790FFFFE7800043018D33B5AA00BD
:102090001703FFFF6700A3053389840383270B0021
:1020A0003E9963170A008347890085043E94E1B78F
:1020B00003560A00DE854A8533F6C9009700000002
:1020C000E780E0F16DD10545E1B71703FFFFE702B7
:1020D000030101112A847C000355E5003ECAB707BD
:1020E00007003ECC7C003ECE97200000E780200811
:1020F0002A898545480897A0FFFFE780E039994580
:10210000480897A0FFFFE780A016AA844A85972079
:102110000000E780A0082380A4009747FF1F938753
:10212000E7F09C434166130606F09396870113D7A8
:102130008701558F93D68700F18E558FA207B7067A
:10214000FF00F58FD98F11462C00138514003EC473
:1021500097D00000E78020CF5008A3820400894573
:10216000228597000000E780E0E019C9AA851305E1
:10217000840397A0FFFFE780A0323C4085073CC066
:1021800005611703FFFF6700C3F71703FFFFE702AF
:1021900003F59790FFFFE78000322A8405049790AB
:1021A000FFFFE78040303305A402F1479145330536
:1021B000F50297200000E78020BA11E56555170366
:1021C000FFFF670003F49747FF1F23ADA7CC97904D
:1021D000FFFFE780402E2A8405049790FFFFE780E9
:1021E000802C3305A4028945060597200000E7806E
:1021F000A0B669D59747FF1F23AEA7C89790FFFFEA
:10220000E780602B2A8405049790FFFFE780A029D0
:102210003304A4029747FF1F239087C89790FFFFBE
:10222000E78060292A849790FFFFE780C027930703
:1022300014003385A7029747FF1F2390A7C697076F
:102240000100938727821747FF1F232BF7C40145FF
:10225000BDB71703FFFFE702E3E6AA842E89014416
:102260009749FF1F938989DC130A80069790FFFF27
:10227000E78060236347A40001451703FFFF670061
:10228000A3E73305440383A709024A86A6853E9542
:1022900097000000E780E0B919E10504C1BF0545DA
:1022A000E9BF1703FFFFE70203E1AA8A2E8BB28B77
:1022B000368C3A8A814401448149974CFF1F938CA4
:1022C000ECD6130D80069790FFFFE780C01D63C911
:1022D000A40011E085494E851703FFFF670023E145
:1022E0003389A40383A70C025E86D6853E994A856E
:1022F00097000000E780E0B31DC19790FFFFE780E3
:10230000801B0544636D4501D2866286DA8513051C
:10231000090397000000E780A0D411C18549850416
:102320005DB71703FFFFE702E3D9C16441112A89B2
:1023300001449749FF1F938969CF130A8006FD1452
:1023400036C632C42EC29790FFFFE780C015924573
:102350002246B2466348A400014541011703FFFF2E
:10236000670083D93305440383A709023E9509C654
:1023700083473500C18B9DC791C68347350093F7CE
:1023800007028DC3630699008357E500639C27010C
:102390000357050001CB63E7E50083478500BA9743
:1023A000E3CDF5FA050469BF1703FFFFE70283D108
:1023B000C1642A8901449749FF1F938929C7130AD9
:1023C0008006FD149790FFFFE780E00D6346A400B0
:1023D0001703FFFF670043D23305440383A70902B5
:1023E0003E958357E500638A9700630499006396DE
:1023F000270197000000E780E0970504E1B7170385
:10240000FFFFE702C3CA89692A8AAE8A328BB68B7C
:102410008144174CFF1F130C6CC1930C8006314D87
:10242000FD199790FFFFE780000863C6A40017031B
:10243000FFFF670083CB3389940383270C02835506
:10244000CA015A863E994A8597000000E780609E3F
:1024500031C1814D15A03384AD038327090303D611
:102460000B00D68533F6C9003E9422859700000004
:10247000E780E0B609E9850D9790FFFFE780A000AF
:10248000E3CBADFC01A8228597000000E780E08A3D
:1024900023040400850471B71703FFFFE702A3C1FB
:1024A0004169AA8A014A174BFF1F130B2BB87D19EC
:1024B000C14B054C9790FFFFE780E0FE6346AA0002
:1024C0001703FFFF6700A3C293098006B3073A030F
:1024D00083290B02BE9983D7E900638E27016384A9
:1024E0002A01639A570103A4890301E84E859700E6
:1024F0000000E780C0BD050A75BF835704016399DA
:1025000077099304C400268597A0FFFFE78020D4B5
:1025100085452A8D2685835C040197A0FFFFE7800F
:1025200080D0268597A0FFFFE78060E8620561857F
:10253000635905048D45268597A0FFFFE780A0CE4F
:102540008945268597A0FFFFE780E0CD8945268550
:1025500097A0FFFFE78020CD8545268597A0FFFF48
:10256000E780A0CD83470500094793F7F707639AF3
:10257000E7009945268597A0FFFFE78000CCA302DE
:1025800085014848337D2D01231894016A9548C47C
:102590000040A1BF1703FFFFE70263B437E4040064
:1025A0008327041D82979747FF1F83C72795171519
:1025B000FF1F1305A5F7A300F5008327441C82978E
:1025C0008327841C81461306F00F814501458297BD
:1025D0001703FFFF6700E3B21747FF1F13070782C8
:1025E00018439745FF1F83C565919747FF1F938742
:1025F000678F83468703034697036397D500974702
:10260000FF1F238DC78E828083C587010347A703E1
:102610006317B6009747FF1F2382E78E828003C6A9
:1026200087016317C7009747FF1F2389D78C8280D4
:1026300083C68701130750026319D700930760020E
:102640001747FF1F230CF78A828083C68701130672
:1026500060026315D60093077002DDB783C7870158
:1026600055BF9747FF1F9387E787D44B0947638D73
:10267000E6081703FFFFE70283A61749FF1F1309A8
:10268000A9833E8483470900918B9DCFB7E4040062
:1026900083A7041D829783A7441C1745FF1F1305BA
:1026A0002582829783A7841C81461746FF1F034615
:1026B000268381450145829721C583470900ED9B0B
:1026C0001737FF1F230AF77E8347040093F7F70F9E
:1026D00085CB91471747FF1F2320F7829700000003
:1026E000E78080EB97000000E78040EFB7E7040049
:1026F000BC4F414691451735FF1F0345257F829703
:102700001703FFFF6700E39F82801703FFFFE702C5
:10271000039D8D4741116306F504C5476308F50223
:1027200085476310F5029737FF1F238BA77CB7E718
:102730000400BC4B930500101735FF1F0345057BB4
:10274000829741011703FFFF6700A39B8547173757
:10275000FF1F2307F77AB7E70400BC4B930500205F
:10276000E1BF9737FF1F9387E777D44B1147638DFE
:10277000E600B7E7040083A7071D8297B7E70400C8
:10278000BC4B930500044DBF05491737FF1F232598
:10279000277783C7070032C62E8493F7F70FD5D368
:1027A000B7E4040083A7041D7D141374F40F82970B
:1027B000E37689FCB245994703C61500E3F0C7FCF0
:1027C000FC4409061735FF1F1305C5738297BC48E3
:1027D000930500081735FF1F03454571829779BFA0
:1027E0001703FFFFE702A38F1737FF1F1307876F3A
:1027F0004047184B1C409736FF1F23ABF66E6316FD
:10280000E4001737FF1F2327F76E130584FE979008
:10281000FFFFE78020A7035564FF9780FFFFE78055
:10282000A06F97A0FFFFE78020D11703FFFF67008D
:10283000438D1703FFFFE702838A9737FF1F9387B4
:10284000676AD84BDC4789C797000000E78080F9AA
:1028500085471737FF1F2321F76A9737FF1F938795
:10286000E7599C43930500021735FF1F0345056890
:1028700083C787031737FF1F2302F768B7E70400F2
:10288000BC4B82971703FFFF6700A3879737FF1F93
:1028900023ACA76482801703FFFFE702A38237E41B
:1028A00004007C4CA1451735FF1F03452564829722
:1028B0007C48A1451735FF1F034545639734FF1F2B
:1028C000938444628297DC4489EB97000000E780A0
:1028D00080D91703FFFF6700238203D567FF978026
:1028E000FFFFE7806063AA896DD1D84891476310E4
:1028F000F7027C4C91451735FF1F0345255F8297F2
:102900007C4891451735FF1F0345455E829703A913
:10291000490103D409018947B7E904001737FF1FAC
:10292000232CF75C83A7091D21044204829783C7E7
:1029300084011715FF1F130565BF61191717FF1FC6
:10294000A306F7BE83A7491C418082979737FF1FD4
:102950002388075A83A7C91C814609469375F40F3B
:102960004A85829711E99737FF1F83C7A76989C7EF
:102970009700FF1FE7800028B7E70400BC4F2146FF
:10298000A1451735FF1F03456556829799B717F381
:10299000FEFFE702C37493F7052001112E8481CF57
:1029A00097000000E78020E913450420056117F334
:1029B000FEFF6700037593F70510A9CF9734FF1F3B
:1029C00093844452DC4897000000E78020C1173709
:1029D000FF1F1307A742184383C7840103478703D8
:1029E0006318F700DC4489C797000000E78080DFA8
:1029F00085471737FF1F2321F750B7E70400BC4B6B
:102A0000930500021735FF1F0345454E8297134576
:102A1000041069BF93F70508BDC79737FF1F83C729
:102A2000774EE91719469735FF1F9385C54D130556
:102A3000D10093F4F70F1739FF1F0349A94C97C032
:102A40000000E780404093970401C1831737FF1FC0
:102A50001307C74B231DF100231CF1009737FF1FFD
:102A6000938747483ACE3ACAD8432306010009CB98
:102A7000DC439315890154080D46E185680082976F
:102A80001345040825B793F72500A5C39737FF1F03
:102A900093874745D84B89476306F7029737FF1F4F
:102AA00083C7874113F7270011EF918B99CFB7E7C1
:102AB0000400BC4F1306000A89451735FF1F034564
:102AC000E542829713452400D5B59737FF1F9387BA
:102AD000E7329C4383C787031737FF1F2300F74262
:102AE00097000000E78060DBF1BF93F7050281CB20
:102AF00097000000E78060DA1345040245BD93F7B4
:102B0000850081CB97000000E780E0D21345840068
:102B100071BD93F7150081CB97000000E780A0B44A
:102B20001345140061B593F7450081CB9700000071
:102B3000E78060B31345440095BD93F7050495C342
:102B40009737FF1F83C7073A91CB97000000E780B4
:102B5000A0A491471737FF1F2320F73A1345040419
:102B6000B1B593F705010145E38207E49737FF1FED
:102B700093874737D84B91476310F7049737FF1F68
:102B8000938787339C4313D727008583D98F858B01
:102B900091E7B7E7040083A7071D8297B7E7040012
:102BA000FC4F91451735FF1F0345453482978547F4
:102BB0001737FF1F2322F73413450401C5BB97378E
:102BC000FF1F2381A744828017F3FEFFE7022351F2
:102BD0009737FF1F23AE07309737FF1F23AC07300F
:102BE00085471734FF1F130464211737FF1F232560
:102BF000F7301C4083C787031737FF1F2300F730C8
